:020000040800F2
:1080000098DE0020A10901082183000823830008CD
:10801000258300082783000829830008000000004A
:108020000000000000000000000000006182000865
:108030002D83000800000000958200084594010887
:10804000BB090108BB090108BB090108BB090108FC
:10805000BB090108BB090108BB090108BB090108EC
:10806000BB090108BB090108BB090108BB090108DC
:10807000BB090108BB090108BB090108BB090108CC
:10808000BB090108BB090108BB090108BB090108BC
:10809000BB090108BB090108BB090108BB090108AC
:1080A000BB090108BB090108BB090108BB0901089C
:1080B000BB090108BB090108BB090108BB0901088C
:1080C000BB090108BB090108BB090108BB0901087C
:1080D000BB090108F9980108BB0901087D9B01084B
:1080E000BB090108BB090108BB090108BB0901085C
:1080F000BB090108BB090108BB090108BB0901084C
:10810000BB090108BB090108BB090108BB0901083B
:10811000159B0108419D010815290108BB090108AB
:10812000BB090108BB090108BB090108BB0901081B
:1081300000F002F800F084F80AA090E8000C8244F5
:108140008344AAF10107DA4501D100F079F8AFF2D2
:10815000090EBAE80F0013F0010F18BFFB1A43F025
:108160000103184770E9020090E902000A444FF049
:10817000000C10F8013B13F0070408BF10F8014B86
:108180001D1108BF10F8015B641E05D010F8016BCB
:10819000641E01F8016BF9D113F0080F1EBF10F82F
:1081A000014BAD1C0C1B09D16D1E58BF01F801CB52
:1081B000FAD505E014F8016B01F8016B6D1EF9D5D5
:1081C0009142D6D3704700000023002400250026EA
:1081D000103A28BF78C1FBD8520728BF30C148BF2A
:1081E0000B607047642922F04587782922F07E874A
:1081F000732923F014830020704710B510BD0000D0
:1082000054656D636F5049443632000000000089A8
:10821000000000671FB59DE8030023F037FA23F044
:10822000DCF823F0FDFB04000020002125F098FA83
:10823000401C60600020002125F0A8FAE0601FBD0E
:1082400023F0DBFD1146FFF7E5FF02F0DFFE24F02F
:1082500075F803B4FFF7D1FF03BC11F084F90000F7
:108260001A4B19680868B0E8F00F80F309884FF0DE
:10827000000080F311884EF00D0E704700000000E2
:1082800003480068006880F3088862B600DF00BF1A
:1082900008ED00E0EFF309800C4B1A6820E9F00FBD
:1082A000106008B54FF0BF0080F3118810F03BFE5E
:1082B0004FF0000080F31188BDE808401968086895
:1082C000B0E8F00F80F30988704700BF1C0300205E
:1082D00001B44FF0BF0080F3118801BC704701B4B6
:1082E0004FF0000080F3118801BC70470B49D1F8B2
:1082F00000C04A685CF8043B1068184442F8040B5C
:108300008C4528BFA1F1DC0C8A4228BFA1F1DC0218
:10831000C1F800C04A6020F00040704730D800200B
:108320007047FEE7FEE7FEE7FEE7704770477047DD
:10833000704700000CB5002201920092524801687B
:1083400041F4803101604FF4A063016801F4003111
:1083500000910199491C0191009911B90199994223
:10836000F3D10168890302D50121009100E0009258
:108370000099012930D145490A6842F010020A608B
:108380000A6822F003020A600A6842F002020A60E8
:108390004168416041684160416841F480614160E9
:1083A000416821F47C114160416841F4E811416069
:1083B000016841F08071016001688901FCD5416864
:1083C00021F003014160416841F0020141604168D0
:1083D000C1F381010229FAD10CBDABE710B52A48DF
:1083E000016841F0010101604168294A1140416082
:1083F0000168284A11400160016821F48021016070
:10840000416821F4FE0141604FF41F018160FFF7D4
:10841000E4FF21494FF00060086010BD10B51A4A12
:10842000506800F00C011D4B1D4800290ED0042996
:108430000ED008290ED003605168194AC1F3031108
:10844000121D515C0268CA40026010BD0360F3E770
:108450000360F1E7516801F47011536803F480334D
:10846000022404EB914133B153689B0307D50D4BB4
:1084700059430160E0E70B4B59430160DCE7074BD0
:1084800059430160D8E7000000100240002002407C
:108490000000FFF8FFFFF6FE08ED00E000127A0092
:1084A0005000002000093D009A48994941609A49CE
:1084B000416070479748016941F080010161704750
:1084C0009448C068C10701D001207047410701D519
:1084D00002207047C00601D5032070470020704776
:1084E00070B50446FFF7ECFF0546012D05D111F0EC
:1084F000A3F9641EA4B2002CF4D104B9FF252846C8
:1085000070BD70B5054645F6FF763046FFF7E8FFCB
:10851000002812D17F4C206940F002002061656183
:10852000206940F0400020613046FFF7D9FF012864
:1085300003D0216921F00201216170BD70B50646AA
:108540000D46FF20FFF7CCFF00280ED1714C2069AB
:1085500040F0010020613580FF20FFF7C1FF0128B6
:1085600003D0216921F00101216170BD00887047AD
:108570002DE9F04105460E461746002407E036F87F
:1085800014102846FFF7DAFFAD1C641CA4B2BC42ED
:10859000F5D3BDE8F081C10703D030F8010C000A23
:1085A00070470088C0B2704710B50446002307E04A
:1085B0002046FFF7DBFF21F81300A41C5B1C9BB2D5
:1085C0009342F5D310BD2DE9F05F82460F46154664
:1085D000AAF10062B2F5002F52D2FFF765FF4FEA11
:1085E000D228C2F34906C6F58064A54200D82C46BD
:1085F000DFF828B137E032183BF812208A4203D165
:10860000401C80B2A042F6D3A04214D24846FFF7E5
:1086100078FF002006E0821937F810102BF81210AE
:10862000401C80B2A042F6D348464FF480623B49DA
:10863000FFF79EFF04E0224639465046FFF798FFB9
:10864000A54202D1BDE8F05F34E708F10108002639
:1086500007EB44070AEB440A281B85B24FF48064F9
:10866000A54200D82C464FF0006000EBC829421408
:108670002A494846FFF798FF00204FF6FF71C1E7EF
:10868000BDE8F09F30B504460D46002306E02046C5
:10869000FFF781FFE854641C5B1C9BB29342F6D346
:1086A00030BD70472DE9F047ADF5006D0D469046A1
:1086B00000240746A0F10060B0F5002F23D2002669
:1086C0004FF48069EA4615E06878000215F8021B4D
:1086D00008442146641CA4B22AF811004A46944278
:1086E00006D1002469463846FFF742FF07F50067C8
:1086F000B61CB6B24645E7D3002C04D022466946E4
:108700003846FFF735FF0DF5006DBDE8F087000036
:108710002301674500200240AB89EFCD18090020F6
:108720002A4908432A490860704770B50F23C27868
:1087300001260178002A1ED0254A126802F4E06260
:10874000C2F5E062120AC2F10404D3404578A540A4
:1087500082781A402A43120101F1E02181F80024B5
:10876000007800F01F018E404009800000F1E020F9
:10877000C0F8006170BD01F01F008640480980000C
:1087800000F1E020C0F8806170BD124A1140014341
:108790000F48001F016070470D4A121D002903D0C9
:1087A000116801431160704711688143116070477F
:1087B0004FF0E021042804D0086920F0040008618B
:1087C0007047086940F00400086170470000FA052E
:1087D0000CED00E080FFFF1F10B5DB4988420AD195
:1087E00044150121204606F074FF2046BDE81040E4
:1087F000002106F06EBFD54988420AD10415012137
:10880000204606F066FF2046BDE81040002106F035
:1088100060BFCF4988420AD10121CC03204606F02F
:1088200058FF2046BDE81040002106F052BF10BDA1
:1088300010B54268C74B1A400C790B6842EA042213
:10884000134343608268C44B1A40D1E90243234377
:108850004C7942EA440213438360C26A22F47002F4
:10886000097C491EC9B242EA0151C16210BD002112
:108870000160017141718160C16001210174704723
:10888000002904D0816841F001018160704781684E
:1088900021F0010181607047002904D0816841F412
:1088A000807181607047816821F4807181607047B8
:1088B000C9B2002A03D042680A4342607047426846
:1088C0008A4342607047816841F0080181607047C7
:1088D000014600208968090700D50120704781689A
:1088E00041F0040181607047014600208968490712
:1088F00000D501207047002904D0816841F4A0010F
:1089000081607047816821F4A00181607047014651
:1089100000208968490200D501207047426822F48E
:108920006042491E42EA413141607047002904D04B
:10893000416841F4006141607047416821F4006181
:108940004160704770B5072609290AD9C568A1F1A9
:108950000A0404EB4404A640B543A3401D43C5608C
:1089600007E0056901EB4104A640B543A3401D4360
:1089700005611F23072A09D2446B521E02EB8202B3
:1089800093409C4391400C43446370BD0D2A09D22F
:10899000046BD21F02EB820293409C4391400C4334
:1089A000046370BDC46A0D3A02EB820293409C439B
:1089B00091400C43C46270BD002904D0816841F429
:1089C000801181607047816821F480118160704757
:1089D000C06C80B270475C484C300068704700291A
:1089E00004D0416841F4806141607047416821F4DE
:1089F000806141607047002904D0416841F4805192
:108A000041607047416821F480514160704782683D
:108A100022F4E0420A4382607047002904D0816852
:108A200041F4004181607047816821F40041816018
:108A30007047002904D0816841F4021181607047B9
:108A4000816821F402118160704701460020896825
:108A5000890200D50120704770B5072609290AD977
:108A6000C568A1F10A0404EB4404A640B543A34041
:108A70001D43C56007E0056901EB4104A640B5430D
:108A8000A3401D430561836BC3F30154121B921C69
:108A900002EB82021F249440A34391400B43836363
:108AA00070BD826B22F44012491E42EA015181637B
:108AB000704708B500900098084400900098026044
:108AC00008BD08B500900098084428300090009830
:108AD000006880B208BD4268204B1A400A434260D9
:108AE0007047416282627047426822F01F020A4367
:108AF0004260704714490831002804D0086840F4E7
:108B0000000008607047086820F4000008607047A3
:108B10000246002012680A4200D001207047C94373
:108B20000160704710B5024600200B0A5468C9B2B4
:108B30000C401168194202D0002C00D0012010BD59
:108B4000090AC94301607047002401400028014020
:108B5000003C0140FFFEF0FFFDF7F1FFFFFD3FFF8E
:108B600001684FF6FE721140016000210160416012
:108B70008160C1607249724A0839904204D14868E4
:108B800040F00F00486070476D4A1432904204D1A3
:108B9000486840F0F00048607047694A28329042C7
:108BA00004D1486840F4706048607047644A3C32C1
:108BB000904204D1486840F4704048607047604A71
:108BC0005032904204D1486840F4702048607047A9
:108BD0005B4A6432904204D1486840F470004860B7
:108BE0007047574A7832904204D1486840F070602C
:108BF00048607047534A111F904204D1086840F002
:108C00000F00086070474F4A1432904204D1086840
:108C100040F0F000086070474A4A2832904204D180
:108C2000086840F4706008607047464A3C329042E1
:108C300004D1086840F4704008607047414A5032DF
:108C40009042FAD1086840F470200860704730B54F
:108C5000026847F6F0739A430C6A8B682343D1E9A4
:108C600004452C4323438C692343CC6923434C6A3A
:108C700023438C6A234313430360CA6842600A6833
:108C800082604968C16030BD00210160416081603F
:108C9000C160016141618161C161016241628162C2
:108CA0007047002904D0016841F00101016070475C
:108CB00001684FF6FE72114001607047002A03D030
:108CC00002680A430260704702688A430260704784
:108CD00041607047406880B2704702460020D10072
:108CE00003D518490839096802E0154908390968A7
:108CF000114200D001207047C10003D51149091F5E
:108D0000086070470E4908394860704702460020E5
:108D1000D10003D50B490839096802E00849083930
:108D20000968114200D001207047C10003D50549F0
:108D3000091F086070470249083948607047000001
:108D4000080002400804024010B59C49884209D13D
:108D50000121042006F0BDFC0021BDE810400420E4
:108D600006F0B7BC9649884209D10121082006F0D7
:108D7000B0FC0021BDE81040082006F0AABC9149D3
:108D8000884209D10121102006F0A3FC0021BDE892
:108D90001040102006F09DBC8B49884209D101216A
:108DA000202006F096FC0021BDE81040202006F0AF
:108DB00090BC8649884209D10121402006F089FCF7
:108DC0000021BDE81040402006F083BC8049884265
:108DD00009D10121802006F07CFC0021BDE8104073
:108DE000802006F076BC7B4988420AD18415012197
:108DF000204606F06EFC2046BDE81040002106F03B
:108E000068BC10BD10B50121084606F062FC0021C7
:108E1000BDE81040012006F05CBC2DE9F0410022C5
:108E2000CC7804F00F03E40601D58C7823430C784A
:108E30004FF00F0714F0FF0F4FF0010C1CD0056826
:108E40000CFA02F40E882640A64211D1960007FAC9
:108E500006F825EA080503FA06F848EA0505CE787B
:108E6000282E02D0482E02D002E0446100E00461C6
:108E7000521C082AE4D305600A88FF2A1ED94568D7
:108E8000002202F108060CFA06F40E882640A642DB
:108E900010D1960007FA06F825EA080503FA06F845
:108EA00048EA0505CE78282E00D14461CE78482EB8
:108EB00000D10461521C082AE3D34560BDE8F0816B
:108EC0004FF6FF710180022181700421C17070474B
:108ED0000246002092680A4200D001207047806854
:108EE00080B2704702460020D2680A4200D00120BA
:108EF0007047C06880B27047016170474161704738
:108F0000002A01D00161704741617047C16070471C
:108F100041F4803282618161826181698069704738
:108F200010B52D4B1A684FF68074224042EA0010AB
:108F30000843186010BD2949C8617047F0B5264C38
:108F4000002801DAE36900E06368C0F30346420DDC
:108F5000120185B2C0F301579540032F07D0C2021A
:108F60000CD50322B240934343F0706209E023F032
:108F70007062636823F07063636002E0AB4343F0A8
:108F8000706201B12A43002801DAE261F0BD62603B
:108F9000F0BD10B58A07120F0F23934021F0030490
:108FA0000D4921448C689C438C608B68904003433E
:108FB0008B6010BD0949DC31086070470008014032
:108FC000000C014000100140001401400018014055
:108FD000001C014000200140000001400000204230
:108FE00010B51C46029B9B1AA34205D3104422468F
:108FF00022F02DFA204610BD002010BD70477047AA
:109000000000000000000000000000000000000060
:109010000000000000000000000000000000000050
:1090200030B5FE4A5188814201D9322030BDD18C01
:10903000814201D25A2030BD002102EB81035B88BE
:10904000834219D84B1C02EB83035B88834213D9FC
:109050004B1C32F8214002EB810132F82350498841
:109060002D1B401A454302EB83004088401A95FBB4
:10907000F0F02044C0B230BD491CC9B20929DCD38C
:10908000002030BD2DE9F04100250024DFF8908359
:1090900040F255570A2140460AF094F8B84205D9E3
:1090A000641CA4B2A0F2555080B20BE040F24441DF
:1090B000884206D2641CA4B2A0F24440404280B26E
:1090C00000E00020304486B2012010F0D5FB6D1C7A
:1090D000EDB2FA2DDED3B6FBF4F0D2490880B6FB30
:1090E000F4F0FFF79DFFD0490880D04A1188411A5B
:1090F00000290BDDD18849B90121117151884FF642
:10910000FF73C1EB011103EA8101D180C8490883D3
:10911000BDE8F081C74A01211160C74908700120EC
:1091200010F03DBF70B5C548012505701BF074F9FE
:10913000BA4C283CA0691BF076F9A573E57370BDA5
:10914000012080F31388BE480168BE4A01F4E06143
:1091500011430160BFF34F8FFEE7F0B587B00121E7
:10916000202006F0A0FA0121042006F09CFA01213B
:10917000102006F098FA0121082006F094FA012147
:10918000402006F090FAB04810250224007AAF4E35
:1091900004280BD34020ADF818008DF81B508DF833
:1091A0001A4006A9AA48FFF738FE0AE00420ADF8E5
:1091B00018008DF81B508DF81A4006A93046FFF7AD
:1091C0002CFE4FF40040ADF814008DF817508DF8C8
:1091D0001640374605A93846FFF71FFEADF8104088
:1091E0008DF813508DF8124004A93846FFF715FE8C
:1091F0000820ADF80C008DF80F508DF80E4003A933
:109200003846FFF70AFE0126ADF808608DF80B50CE
:109210008DF80A4002A93846FFF7FFFDADF804605B
:109220008DF807508DF8064001A98A48FFF7F5FD33
:1092300007B0F0BD10B545F2555006F0F3F8052023
:1092400006F0F3F84FF47A6006F0F2F806F0F8F85A
:10925000BDE8104006F0EFB806F0EDB82DE9F05F7C
:1092600040F2053007F08DFF7B49087040F2F6258B
:10927000284607F086FF6C1EFF2807D100212846EC
:1092800007F080FF6421204607F07CFF204607F0AE
:1092900078FF0446284607F074FF704904EB00206D
:1092A0000880DFF8A4B101269BF8F302012806D953
:1092B0008BF8F362012140F2F32007F063FF684965
:1092C0005E2008800021942007F05CFF40F2D3204C
:1092D00007F057FF04464FF4357007F052FF61491D
:1092E00004EB00200881072007F04BFFFF2804D083
:1092F000082007F046FFFF2803D13E21072007F092
:1093000041FF9BF805000025FF2830D102F07DFFCA
:109310000021052007F036FF8921042007F032FFE5
:1093200002F0DDF98BF8DA509BF8090000F03F01FC
:109330008BF80910092007F025FF0024002104F50F
:10934000A17007F01FFF641CE4B2072CF6D30024C1
:10935000002104F2491007F015FF641CE4B2072C49
:10936000F6D39BF86E00012801D98BF86E509BF85C
:109370005902FF2808D19BF85A02FF2804D1C820BF
:109380008BF859028BF85A529BF87800DFF8D8A076
:1093900038B10421012812D0022820D003282AD174
:1093A00024E029468BF89B509B2007F0EBFE3146CA
:1093B0008AF800604FF45B7007F0E4FE1BE09BF856
:1093C0009B0020B98BF89B109B2007F0DBFE294601
:1093D0008AF800504FF45B7007F0D4FE0BE04FF4B6
:1093E0005B7007F0CEFE8AF8000004E08BF89B105B
:1093F0009B2007F0C7FE1D4805701D499BF89B0088
:1094000008701C49087008B11B4806701B4C207876
:1094100018F073FE1A490880227833E028000020F3
:10942000002401403C0600206601002006020020C6
:10943000CC840020A0012142427C0020EC050020C9
:109440000CED00E00400FA054D80002000140140FE
:10945000000C014000080140B803002082000020F9
:10946000A00000209A110020AB000020B7030020CC
:109470009C0000206A000020870000206900002076
:1094800096000020FD48FE4932B19BF86C20028016
:109490009BF86D00088005E09BF8712002809BF826
:1094A000700008800027002404F1B900804607F00E
:1094B00068FE28B1404607F064FE032800D2012769
:1094C000641CE4B2052CEFD3EE48012F05D00570E3
:1094D0009BF8CC00EC4910B10AE00670F8E79BF865
:1094E000CB0028B99BF8CE0010B99BF8CD00D0B1C5
:1094F000E64805709BF8CD009BF8CE2000EB0220DB
:10950000E34A80B210809BF8DB20032A05D00E705E
:109510009BF8D310012204F091F99BF80600FF2874
:1095200003D010B111E00D70F7E78BF806608BF8EF
:10953000F352D848068001460122D748FFF743F886
:109540009BF80610062007F01DFE4FF49464204699
:1095500007F017FED1490870012804D90D700021C9
:10956000204607F00FFE40F2A244204607F009FE15
:10957000CB490870022804D90D700021204607F05D
:1095800001FE002440F2A34840F2A44908EB440045
:1095900007F0F7FD074609EB440007F0F2FD07EB83
:1095A000002081B2BF4820F814100289B2F5FA7F7A
:1095B00000D8C9BB0C210180232141803721818043
:1095C0009621C180FA2101810C21404607F0DAFD85
:1095D0000021484607F0D6FD232140F2A54007F0C0
:1095E000D1FD002140F2A64007F0CCFD372140F22A
:1095F000A74007F0C7FD00214FF4956007F0C2FDBA
:10960000962140F2A94007F0BDFD002140F2AA409A
:1096100007F0B8FDFA2140F2AB4007F0B3FD00219E
:1096200040F2AC4007F0AEFD641CE4B2052CADD3B3
:1096300040F2AD47384607F0A4FD9B4C2070FF2850
:1096400004D125700021384607F09CFD40F2AE4958
:10965000484607F096FD4FF4966840F2AF47FF2862
:1096600004D1384607F08DFDFF287DD0484607F02D
:1096700088FD6060384607F084FD616841EA00209B
:109680006060404607F07DFD616841EA004060602F
:1096900040F2B14007F075FD616841EA006060602A
:1096A00040F2B347384607F06CFD044640F2B24939
:1096B000484607F066FD04EB002081B27B4801803C
:1096C0004FF6FF783C24414508D1048000214846EC
:1096D00007F058FD3C21384607F054FD40F2B547ED
:1096E000384607F04EFD8146781E07F04AFD09EB2B
:1096F000002081B26E480180414508D105800021DB
:10970000781E07F03FFD0021384607F03BFD40F290
:10971000B747384607F035FD8146781E07F031FD22
:1097200009EB002081B263480180414508D10480E3
:109730000021781E07F026FD3C21384607F022FD67
:1097400040F2B944204607F01CFD8146671E3846AA
:1097500007F017FD09EB002081B257480180414511
:109760000AD10580002100E0D2E0384607F00AFD6A
:109770000021204607F006FD40F2C547384607F0B5
:1097800000FD044640F2C449484607F0FAFC04EBE9
:1097900000204A4C80B22080404509D150202080D2
:1097A0000021484607F0EEFC2178384607F0EAFC35
:1097B00040F2C74007F0E5FC814640F2C647384614
:1097C00007F0DFFC09EB002080B26080404508D143
:1097D00066800021384607F0D5FCA178781C07F098
:1097E000D1FC40F2C94007F0CCFC04464FF4996923
:1097F000484607F0C6FC04EB0020314C80B22080C4
:109800004FF4FA67404509D127800721484607F001
:10981000B9FC217840F2C94007F0B4FC40F2CB40DB
:1098200007F0AFFC814640F2CA4007F0AAFC09EB02
:10983000002080B2608040450AD16680002140F25D
:10984000CA4007F09FFCA17840F2CB4007F09AFC99
:1098500040F2F949484607F094FC04464FF49F60F3
:1098600007F08FFC04EB0020164C80B220804045AE
:1098700030D1278007214FF49F6025E0BA030020F4
:10988000BC030020A8000020AE000020BC00002087
:10989000C60000207400002000770008910300201B
:1098A000F0020020F202002020000020FE01002033
:1098B0000002002002020020040200200602002014
:1098C000D4010020DC01002007F05CFC2178484630
:1098D00007F058FC40F2FB4007F053FC814640F291
:1098E000FA47384607F04DFC09EB002080B2608053
:1098F000404508D166800021384607F043FCA17836
:10990000781C07F03FFC9BF8B903FF2813D019E03F
:1099100065600021484607F035FC0021384607F015
:1099200031FC0021404607F02DFC002140F2B140FF
:1099300007F028FCB4E61E218BF8B91340F2B930C9
:1099400007F020FC40F2FF4007F01BFC044640F209
:10995000FE49484607F015FC04EB0020FE4C80B29F
:1099600060800327404509D167800021484607F001
:1099700009FCA17840F2FF4007F004FC4FF42E7878
:10998000404607F0FEFB8BF8B8020C2805D98BF88F
:10999000B8520021404607F0F5FB9BF8D902012898
:1099A00006D98BF8D952002140F2D92007F0EAFB02
:1099B0009BF8DC02012806D98BF8DC5200214FF419
:1099C000377007F0DFFB00240BEB040090F8F71072
:1099D000FF2906D180F8F770032104F1F70007F0A2
:1099E000D1FB641CE4B2082CEED39BF8B802192812
:1099F00005D98BF8B8520021404607F0C3FB01207F
:109A000009E00BEB000191F8BA22FF2A01D181F89D
:109A1000BA52401CC0B29BF8B812491C8142F0D81F
:109A20001B2007F0AEFB04461C2007F0AAFB04EB4A
:109A300000272F2007F0A5FB0446302007F0A1FBEC
:109A400004EB0020C54C874201D2267000E025704F
:109A5000312007F096FB0746322007F092FB07EB18
:109A60000028452007F08DFB0746462007F089FBBC
:109A700007EB0020804501D2667000E065704FF46E
:109A80005B7007F07EFB8AF80000012801D98AF894
:109A900000609BF86603B8B99BF8E1009BF87E1064
:109AA000884203D39BF87D1088420DD9C8205C46BC
:109AB0008BF8E100C821E12007F064FB94F859120B
:109AC00094F85A0218F021FBF62007F05AFB8BF8A5
:109AD000F600A348017841F007010170A148007821
:109AE00030B39BF8090040F001008BF809009E4854
:109AF00006709BF8090000F0FB018BF809100920A3
:109B000007F040FB7B2021F053FC40F25324204619
:109B100007F037FB022803D90021204607F032FB6B
:109B200040F2EF24204607F02CFBFF2809D00CE080
:109B30009BF8090000F0FE008BF809008A480570C8
:109B4000D7E70021204607F01DFB07F067FB874899
:109B5000808820B940F2E171842002F0D7F940F208
:109B60000656304607F00DFB814CE072022804D9FE
:109B7000E5720021304607F005FB40F207563046FB
:109B800007F0FFFA2073022806D925733046BDE896
:109B9000F05F002107F0F6BABDE8F09F10B5754CF4
:109BA00010212046FFF7AAF94FF4FA700FF064FE77
:109BB0002046BDE810401021FFF79EB910B50121E5
:109BC0000D2005F070FDBDE8104001216A48FFF747
:109BD000B5B970B586B0664D0120687100240026C5
:109BE00007E0641C142C01D96E7106E064200FF0AC
:109BF00043FE0DF0F0FB0028F3D16879002824D053
:109C000002A903A80DF0D7FB68460DF0DCFB04A900
:109C100005A80DF016FB0DF0DCFB5848C17846EAAC
:109C20000161827841EA0241427841EA02210078EA
:109C30000843E861411C08D10DF050FB10B950A059
:109C400021F09AF964200FF017FE06B070BD1FB521
:109C50000025009501950295FFF7BBFF444CA571C7
:109C60004C4E6F464FF001086079002812D0B6F8CC
:109C70005000401CA6F85000207C012803D00DF0B5
:109C8000C8FA40B150E0607C401CC0B26074142837
:109C900000D92574C5E05236BDF80C003081A6F815
:109CA0000A903088401C26F8520932200FF0E4FD5B
:109CB00003A80DF0AFFAB8BBB6F85400401CA6F8E4
:109CC0005400A079042807D2BDF80C1000F101025D
:109CD000A27127F8101005E004D1BDF80C00ADF812
:109CE0000800A5714FF00001084637F81020114414
:109CF00000F10100C0B20528F7D30520B1FBF0F058
:109D000025490880BDF80000F083BDF802003084CA
:109D1000BDF804007084BDF80600B084BDF80800EA
:109D2000F084708A401C7082608A3082401C80B24D
:109D30004FF46161B0FBF1F2608201FB1200A0F50B
:109D400060610F3951D10A481C300DF0B4FA28BBBC
:109D5000217F40F2772022E00E020020A80100209F
:109D6000940000206A0000206900002018110020E3
:109D700000000020000C014000043000C4820020DC
:109D80002073657420626173656C696E653A204F5B
:109D90004B000000A6860020E40100201EE007F032
:109DA000F1F9A08BC0F307214FF41E7007F0EAF918
:109DB000E069C0F3074140F2792007F0E3F9E06978
:109DC000010E40F27A2007F0DDF9FD49E0690870E4
:109DD000020A4A70020C8A70000EC870F089401C9A
:109DE000F081FFF7F6FE84F81080E0693A36C1B2E0
:109DF0003181C0F307217181C0F30741B181000EA9
:109E0000F08136F83A09C82805D17587FFF7E1FED9
:109E100084F810806574708F642802D17587FFF70D
:109E2000BDFE4FF47A700FF027FD1DE786B0FFF7F7
:109E300079F900201AF062FF00201BF093FEE04841
:109E4000D63017F00EF9DF490D200870DE491120D9
:109E50000870DE4800240470DD480470DD4DDE4EDD
:109E6000DE4F28780C2802D1FFF75CF92C70287897
:109E7000132808D1FFF756F900201AF03FFF002001
:109E80001BF070FE2C7096F82B00A0B97471787BD3
:109E900088B90120787300234FF41672D04901A8C5
:109EA00000941AF090FA024622B10023CC4901A88E
:109EB0001BF004FE7C7305200FF0DEFCD1E70026CA
:109EC000C84801250570C84F97F8D800002804D06D
:109ED000C0EB00108100C5480180DFF81493DFF863
:109EE00014A3DFF814B30024FFF7B6F9C3490878C8
:109EF00008B1401E0870087808B9C1480470DFF83E
:109F0000D48298F800000D280AD13878A9F800000A
:109F10007878A9F802000222B549BA48FEF753FB47
:109F200098F800000E280BD1B878A9F80000F8784E
:109F3000A9F80200B3480222AD491030FEF743FBF6
:109F4000B1480178012904D19AF80010491C8AF817
:109F500000109AF80010052902D904708AF8004010
:109F6000AA490878012806D1887918B1CC71401E19
:109F7000887100E0CD71A6490878012806D188795A
:109F800018B1CC71401E887100E0CD71A1490878EC
:109F9000012806D1887918B1CC71401E887100E083
:109FA000CD719D490878012806D1887918B1CC7106
:109FB000401E887100E0CD7198490878012806D1CB
:109FC000887918B1CC71401E887100E0CD7197F886
:109FD000D80050B18549088808B1401E08809048D3
:109FE00009880278114300D10570761CF6B23C2E28
:109FF00007D397F8610318B18A480178491E0170A8
:10A0000000268848007830B997F8610318B187F8BE
:10A0100061437248057198F80000102803D188F850
:10A02000004002F0F2F898F80000112807D002F082
:10A03000FAFF7D490880DBF80000B8B11FE06548F1
:10A040000470142440F26D3540F26C76AC4205D0B9
:10A05000652C03D0FF21204607F094F8641CA4B2BD
:10A06000B442F3D302F0D1F8FFF76AF897F8B902D7
:10A0700028B103F0F5F86D480571857045706C4A9C
:10A08000107801280AD16B490878401CC0B20870CA
:10A09000052803D114700C7050480571DBF80000DE
:10A0A00098B197F8631081B1401ECBF8000060B9F9
:10A0B0009B2007F066F86049087087F89B005F49AD
:10A0C00008705A4885704548C4705D490888012861
:10A0D00001D9401E08805B49088808B1401E0880ED
:10A0E000088838B997F8ED00FF2803D001215648B9
:10A0F000FEF704FF97F8ED00FF2803D10121524835
:10A10000FEF7FAFE51490888401E80B2088008B95F
:10A110004F480570DFF83C8198F8000010B1401EF0
:10A1200088F8000098F8000020B9002201214A4870
:10A1300001F04DFA98F8010010B1401E88F80100B6
:10A1400098F8010020B900220321434801F03FFAAA
:10A1500098F8020010B1401E88F8020098F802003A
:10A1600020B9002205213C4801F031FA98F803009B
:10A1700010B1401E88F8030098F8030020B90022AF
:10A180000721354801F023FA98F8040010B1401E69
:10A1900088F8040098F8040020B9002209212E480C
:10A1A00001F015FA98F8050010B1401E88F8050076
:10A1B00098F8050018B900220B2127484EE04FE01F
:10A1C000C4820020590400205704002058040020B5
:10A1D0005A040020850300204916002000000020BA
:10A1E00054060020640000204D8000207A000020EA
:10A1F00074000020B6030020880000207F030020A8
:10A200007E03002010770008B50300202C110020E9
:10A210003611002040110020541100204A11002066
:10A22000790000208403002070000020221100200B
:10A230008C000020840000206A00002066000020BE
:10A24000980300206C000020000801407C000020E2
:10A250007E000020200200201E02002001F0B7F93D
:10A2600098F8060010B1401E88F8060098F806001D
:10A2700020B900220D21F94801F0A9F9F849C88850
:10A2800010B1401EC88000E00C71F649C88810B1BA
:10A29000401EC88000E00C71F349C88810B1401E10
:10A2A000C88000E00C71F149C88810B1401EC88018
:10A2B00000E00C714FF47A700FF0DEFA14E60EB580
:10A2C000EB490120087048708870C8700871887167
:10A2D0000121E848FEF710FEE748E84900780870D9
:10A2E00007F0CFFDE64F4FF6FF75E6A33888ED2265
:10A2F000291ACDE900100A21012007F09DFB3888BA
:10A30000E2A3291ACDE90010ED220A21012007F06D
:10A3100093FB3888DEA3291ACDE90010F9223921F0
:10A32000012007F06FFB3888D7A3291ACDE9001068
:10A33000ED226721012007F07FFB3888D5A3291A79
:10A34000CDE900104FF48C720A21012007F074FB54
:10A35000B7F80090D148042141724FF00A0A002456
:10A3600047F61966DFF8348398F80900401CC0B23C
:10A3700088F80900052801D988F80940C8480078FC
:10A3800090B1012814D0022816D0032818D0042830
:10A390001AD04FF4384038803888814518D198F861
:10A3A0000110012914D049E049F289603880F3E7AF
:10A3B0004FF6E0703880EFE74FF6E0503880EBE77B
:10A3C0004FF478403880E7E747F294103880E3E7AD
:10A3D00088F80140291ACDE90010AAA3ED220A212C
:10A3E000012007F029FB3888A8A3291ACDE900101D
:10A3F000ED220A21012007F01FFB3888A4A3291AA7
:10A40000CDE90010F9223921012007F0FBFA388844
:10A410009DA3291ACDE90010ED226721012007F044
:10A420000BFB38889BA3291ACDE900104FF48C72DE
:10A430000A21012007F000FBB7F80090DFF864B2B2
:10A440009BF80000012823D0022830D0042840D0F7
:10A45000052870D007286ED006286DD008286BD04C
:10A460000B286AD00F2869D08F49087800286FD050
:10A47000002008708D49087800286AD000200870F4
:10A480008B490120087098F80900052874D038E13C
:10A49000304607F09EF8CDE900561E2285A31146EE
:10A4A000012007F0C9FA0FF007FAFEF749FE8BF812
:10A4B0000040304607F08DF8CDE900561E2280A3FB
:10A4C0001146012007F0B8FA01F09FFE02F053FC9C
:10A4D0007BE28BF800407C4890F8650001280FD0A3
:10A4E000B8B102281ED0032829D0042832D005286C
:10A4F00039D0062841D0072848D008284FD056E048
:10A500004FF4964840460FF03EF87048C0F8088077
:10A510004DE04FF4165840460FF035F86B48C0F840
:10A52000088044E04FF4164840460FF02CF8674886
:10A53000C0F808803BE042E04EE05AE05EE04FF4B5
:10A54000614840460FF01FF86048C0F808802EE0D0
:10A550006FE070E04FF4E13840460FF014F85B48CC
:10A56000C0F8088023E04FF4963840460FF00BF80F
:10A570005648C0F808801AE05FE04FF496684046FD
:10A580000FF001F85148C0F8088010E04FF49658D9
:10A5900040460EF0F8FF4D48C0F8088007E04FF441
:10A5A000615840460EF0EFFF4848C0F80880474821
:10A5B00090F82B0003288BD10FF07EF905E2444878
:10A5C0000088C1B2C0F3072017F045FE002002F05A
:10A5D00082FB8BF80040F8E13D480088C1B2C0F32F
:10A5E000072017F092FD012002F075FB8BF8004068
:10A5F000EBE117F0F9F98BF80040E6E1CDE9005600
:10A6000034A36C220A21012007F016FACDE9005686
:10A6100031A397220A21012007F00EFACDE9005656
:10A620002EA3C2220A21012007F006FA8BF800406F
:10A63000CBE101201DE7012021E72948007820B166
:10A64000012851D0142857D05BE026480022B0F9E9
:10A650000010104607F0F9FF53E000001E02002032
:10A6600006020020D4010020DC0100200E020020A0
:10A6700022110020000801406A000020660000202E
:10A6800000030020504D20203A000000504D0000F3
:10A69000322E3500504D31303A00000000000020CD
:10A6A000FC020020850300204901002081000020D9
:10A6B000480100205570646174696E6700000000F5
:10A6C00052657374617274004D8000204916002039
:10A6D0008E0000205345540046414E00535953000C
:10A6E0004C0100208E010020FE480322B0F900102A
:10A6F000012007F0AAFF04E0002211460A2007F01B
:10A70000A4FFF9480078012873D0DFF8E08398F8B7
:10A710005700E8B398F85A0098F8591000EB012157
:10A72000F0480288511A0180F1480188022008F09F
:10A73000E0FA80B298F8851059B398F8881098F824
:10A74000872001EB0221B1FBFAF1411AE9480180AF
:10A7500098F8B300F0B398F8B60098F8B51000EB8D
:10A760000120B0FBFAF1E4480088411AE348018077
:10A77000E248E3490088C88207F083FB98F80F019C
:10A7800048B398F8120198F8111100EB012101E08B
:10A7900051E05CE0DB480288511A018098F86B01B7
:10A7A000F0B398F86E0198F86D1100EB0121D648CE
:10A7B0000288511A0180D5480079142878D0D148F0
:10A7C000008807F092FBD048008807F043FCDFF8D0
:10A7D000408302E047E054E00BE098F80700A8B39C
:10A7E0008DE870000023CB4A1A210D2007F03DF9B7
:10A7F00078E007F02CFD4FF4784BCDE900B6C6A306
:10A8000067220021012007F017F9CDE900B6C4A3A3
:10A8100092220021012007F00FF9C3A3BD2200E01E
:10A820003AE0CDE900B60021012007F005F901204A
:10A8300088F80A00CBE7AB4898F8592098F85A10E6
:10A84000038803EB0222114401806DE742E098F88F
:10A85000881098F8872001EB0221B1FBFAF1084437
:10A86000A449088074E798F8B60098F8B51000EB92
:10A870000120B0FBFAF1A048008808449F490880F5
:10A8800076E7A04898F8121198F81121038803EB95
:10A8900002221144018081E79B4898F86E1198F8D4
:10A8A0006D21038803EB02221144018083E7FFE757
:10A8B000CDE900569FA3ED220A21012007F0BCF844
:10A8C000CDE900569BA34FF48C720A21012007F0BA
:10A8D000B3F87CE78DE8700000231A461A210D209A
:10A8E00007F0DFF898F8080040B18DE870000D23FC
:10A8F000934A1A21184607F0B8F807E08DE870006F
:10A900000D2300221A21184607F0CBF898F807000B
:10A9100010B1401E88F8070098F8080010B1401EDA
:10A9200088F8080087480079C00746D086498879AA
:10A9300002280ED0052837D0062835D0012833D07C
:10A940008DE870001A21D223804A084607F08DF85E
:10A950003BE0087A462808D28DE870001A21D223FD
:10A960007B4A084607F081F82FE0502808D28DE88E
:10A9700070001A21D223774A084607F076F824E0BF
:10A980005A2808D28DE870001A21D223724A08464C
:10A9900007F06BF819E08DE870001A21D2236F4A96
:10A9A000084607F062F810E08DE870001A21D22303
:10A9B0006B4A084607F059F807E08DE870001A2145
:10A9C000D223624A084607F050F84FF47A700EF02E
:10A9D00053FFC7E44FF4E1300EF05CFE614E0025FA
:10A9E0003570614F307820B1012802D0032805D09E
:10A9F00007E00120307015F082FD02E0032015F021
:10AA00007EFD002404E0FEF727FC14200EF034FF46
:10AA10003878462804D02046641CE4B29628F2D345
:10AA20003878462802D1514815F0BEFD50480570CF
:10AA30003C214E4820F08AFD3D7040F6B8300EF0C3
:10AA40001BFFCFE74FF496400EF07AFEDFF8A090A0
:10AA50004FF4C870A9F8000026490880454E01202F
:10AA60003070DFF814A1DFF814B1454800780728EA
:10AA700004D044480078012805D008E040F6B830FA
:10AA80000EF0FAFEF1E7B9F800000DF0A3FB307804
:10AA9000012808D0022809D003280AD004280BD0A6
:10AAA00007280CD081E0384D08247EE0374D07247C
:10AAB0007BE0374D112478E0364D072475E015F022
:10AAC000BFFE0024344D354FDFF8D480285D15F0EB
:10AAD000BCFE3878A87198F80000E871641CE4B2F4
:10AAE000062C5FE08C0100205C010020058900201D
:10AAF0008A01002088010020E40100206801002074
:10AB0000CC840020E8010020EA0100204C01002054
:10AB1000221100205C3403084869676800000000C7
:10AB2000566F6C74616765006F6E20525334383510
:10AB300000000000202020202020202020200000D5
:10AB40000037030820000020C82200200C5403080E
:10AB5000A4390308EC3E0308344403087C49030885
:10AB6000C44E0308E60100207C030020F47B002093
:10AB70008A030020EE010020307C00208B0300209F
:10AB800059010020050300203AEA020842EA0208BF
:10AB900032EA02084AEA02081A010020C70300202C
:10ABA000C603002092D3F64D0824F64829680160B8
:10ABB0006968416008200FF019FA002704E0FEF7E9
:10ABC0004BFB14200EF058FE9BF80000844204D08A
:10ABD00038467F1CFFB29628F1D39BF8000011285D
:10ABE00028D39AF80000612824D19AF8010003289C
:10ABF00020D19AF802000C281CD10F21E24815F050
:10AC000035FE9AF810109AF80F2001EB022189B254
:10AC100088420FD19AF806309AF805209AF8041065
:10AC20009AF8030015F02CFC23F0E2FCA9F80000D0
:10AC30000420307000208BF800001221D24820F050
:10AC400085FC4FF47A700EF017FE0EE7CF4890F8AF
:10AC500065104FF49640092928D2DFE801F0050974
:10AC60000B0F13171B1F23004FF416500EF08BBC55
:10AC70000EF089BC4FF416400EF085BC4FF46140D5
:10AC80000EF081BC4FF4E1300EF07DBC4FF49630F5
:10AC90000EF079BC4FF496600EF075BC4FF49650F0
:10ACA0000EF071BC4FF461500EF06DBC0EF06BBC39
:10ACB0000FF0A4F90DF035FA4FF40071B448FEF727
:10ACC0001DF9FFF7C3FFB34EB34CB44D307830B12C
:10ACD000401EC0B23070012801D115F097FB2078DA
:10ACE00030B12078401E2070207808B90EF0E4FDC5
:10ACF000E88A322802D2401CE88214E00020E88270
:10AD000006F08CFAA6488288A6490A8082798A7061
:10AD1000C279CA70027A0A710278A3490A7042782D
:10AD20004A70807888700A200EF0A6FDCEE708B53C
:10AD30004FF0000A08F0C8FE944D4735287869782E
:10AD400000EB012199480180A978EA7801EB022102
:10AD5000418029796A7901EB02218180A979EA7918
:10AD600001EB0221C180297A6A7A01EB022101817B
:10AD7000A97AEA7A01EB02214181297B6A7B01EB06
:10AD800002218181A97BEA7B01EB0221C18104219F
:10AD90008748FEF7B3F84FF400717D48FEF7ACF832
:10ADA000442009F020FD7D4C0020A082814E3227F6
:10ADB0004FF00109012300227F498048009709F0E4
:10ADC00082FE08B986F80090A08A401C80B2A0825A
:10ADD0000A28EFD33078012801D0002030700DF020
:10ADE000DBFCDFF8DCB1774E774FDFF8E08104253C
:10ADF000774801787748818220780B2802D2401C5E
:10AE0000207001E000202070FEF73CF972480178C4
:10AE1000491C017008F00EFA6D48007807280BD124
:10AE20000AF1010A1FFA8AFA0320BAFBF0F100FBCB
:10AE300011A008B90DF0DAFC08F0DDFB08F07FFD89
:10AE400066484078012801D116F094FDFEF704FA17
:10AE50000023E37100204D4A02EB000C9CF89E1287
:10AE6000022901D0042945D1DFF874E13EF810E051
:10AE7000BEF1010F05D094F807C0BCF1000F1AD045
:10AE800035E09BF8001049BB357087F8009088F8D2
:10AE9000005082F89B509CF89E12022908D192F82B
:10AEA0006310C1EB01114FEA810C4E49C1F800C09B
:10AEB00084F807901BE092F8B9C2BCF1000F02D0F1
:10AEC00004290CD013E04749096839B933703D7043
:10AED00088F8003082F89B308BF8003007E0337040
:10AEE0003D7088F8003082F89B308BF800303E4986
:10AEF00081F80490401CC0B20828ADD33B4992F8B9
:10AF0000F1020988081A00D5404292F8B913884224
:10AF100073DD84F80290364880F8049041884FF63B
:10AF2000FF73C1EB011103EA8101C18084F8039032
:10AF300092F86300FF2802D13C2082F8630092F867
:10AF40006300A8B1C0EB00108100264801602948C9
:10AF500080F80090357088F80050507A40F0010178
:10AF60005172092006F00EF987F800900220E07077
:10AF70001D4880F8029080F8019080F804903DE030
:10AF80001A010020AA030020307C00204D80002000
:10AF9000000C0140950300209303002000000020D6
:10AFA00018110020D4030020C9030020A4110020A0
:10AFB000001801405B010020B4010020B001002016
:10AFC000780000206A000020680000206600002051
:10AFD00059010020A68600206201002038040020CC
:10AFE000861100208800002022110020820100200C
:10AFF0000E02002069000020FFE7A370FE49A07840
:10B00000C8834FF47A700EF037FCF1E62DE9FF5F4C
:10B010000024FA490803FDF7B8FBFEF7CFFD4FF413
:10B02000A060FDF77DFBFEF717F948200EF0F0FB5E
:10B030006421F34820F08AFA40F2CF21C82007F0BB
:10B0400087FC05F0F3FF05F0D2FEFEF7F3F805F0FC
:10B05000C7FC00F044FBFEF780F808F0A5FEE94DC0
:10B0600010212846FDF748FF20212846FDF744FF20
:10B07000E54DE64995F86A000870FEF7EFF8FEF72F
:10B08000EBF8FEF7E9F80121E148FDF735FF06F09E
:10B09000EFFBE048A046A0F81080DF4995F89B0040
:10B0A0000870DE4E4FF0010986F80090DC4A072157
:10B0B000117085F87F834FF0C80B85F880B395F841
:10B0C0007F10012902D9D74981F8009095F8B9225B
:10B0D000D54912B988B181F80090087817F00DF8B9
:10B0E000D24908803278D248D2494AB195F86C20CA
:10B0F000028095F86D00088008E004200870ECE7F5
:10B1000095F87120028095F87000088095F89210EB
:10B11000C948012906D0032180F82B1095F8D800E2
:10B1200018B105E080F82B80F8E7C44880F800806B
:10B1300016F05AFCC248291991F8B2100155641C46
:10B14000E4B2072CF7D3FEF787F80125FEF784F861
:10B15000142C0AD206F0CAF8012806D0641CE4B206
:10B1600064200EF089FB002DF0D109F010FE0024C0
:10B1700040F22D36DFF8CCA2771C06EB440006F037
:10B1800000F8054607EB440005F0FBFF05EB002047
:10B190002AF81400641CE4B2032CEED3BAF80000C1
:10B1A0004FF47A744FF41675A04207D8BAF802002B
:10B1B000A04203D8BAF80400A0421DD9AAF800B0F2
:10B1C0004FF4C870AAF80200AAF804504FF0000B20
:10B1D00006EB4B001AF81B1005F0D4FF3AF81B00E1
:10B1E000010A07EB4B0005F0CDFF0BF1010B0BF053
:10B1F000FF0BBBF1030FEBD340F2333005F0C1FF7F
:10B2000006464FF44D7005F0BCFF06EB0020AAF88F
:10B21000060040F23536304605F0B3FF8246771C13
:10B22000384605F0AEFF0AEB002081B28648018067
:10B23000A1420AD94FF4FA710180F421304605F099
:10B24000A1FF0121384605F09DFF4FF4A064204680
:10B2500005F097FF6A490880FF2801D1A1F8008016
:10B260000888401C0880C1B2204605F08BFF0224EC
:10B27000CDE90048CDF8088000232A4673A175481F
:10B28000CDF80C800DF063FC0720CDE90008CDF867
:10B29000088000232A4670A17148CDF80C800DF07B
:10B2A00056FC0526CDE90068CDF8088000232A4623
:10B2B0006CA16E48CDF80C800DF049FCCDE900681A
:10B2C000CDF8088000234FF4967269A16A48CDF842
:10B2D0000C800DF03CFC6948007860B90320CDE992
:10B2E0000008CDF808800023642265A16848CDF8E5
:10B2F0000C800DF02CFCCDE90098CDF808800023DF
:10B30000642264A16748CDF80C800DF020FC06256E
:10B31000CDE90058CDF80880002340F2644262A1D4
:10B320006348CDF80C800DF012FCCDE90058CDF843
:10B330000880002340F24C425EA16148CDF80C80A9
:10B340000DF005FCCDE90048CDF808800023C822A7
:10B350005CA15F48CDF80C800DF0F9FB0DF0D5FE37
:10B3600004B00020BDE8F09F5A4D00264FF47A77D4
:10B37000287870B1401EC1B2297051B90024002252
:10B380002146554800F023F9641CE4B2032CF6D39F
:10B390002E7038460EF070FAEAE7504DDFF8409113
:10B3A000DFF84081504EDFF844A1DFF844B1514F3F
:10B3B00000243C72B8F80020397ACA40D00702D085
:10B3C000685C401C6854685C06280FD36C5419F8FC
:10B3D000010010B1401E09F8010019F8010028B958
:10B3E000D00703D000223F4800F0F1F8387A401C23
:10B3F000C0B2387203287FE0CC84002000800008AF
:10B40000A6860020000C01404D800020A7000020EF
:10B4100000080140721100206A000020690000202D
:10B420009400002085000020680000209600002085
:10B43000BA030020BC030020491600207900002038
:10B44000F40000206402002032020020496E707572
:10B45000740000002FAD0008434F4D4D3100000037
:10B46000B1AC0008434F4D4D3200000045AA000822
:10B47000434F4D4D33000000D5A900084B0100207B
:10B4800044697370616C7952656672657368000017
:10B49000BFA20008536F66747761726574696D6549
:10B4A00072000000BF9E00084D5354500000000081
:10B4B0002D9E0008576966697461736B0000000077
:10B4C00041790108564F435F5461736B00000000DF
:10B4D0004F9C0008A2000020B000002005010020C1
:10B4E000CE000020B600002002010020CB0000208A
:10B4F000B800002000000020FFF45CAF3C72BBF8F5
:10B500000020397ACA40D00702D0705C401C7054C9
:10B51000705C06280FD374541AF8010010B1401E55
:10B520000AF801001AF8010028B9D00703D0002258
:10B53000164800F04CF8387A401CC0B23872032824
:10B54000DDD342F210700EF097F932E770B5154670
:10B550000F4B18800F480078002815D1084623F0BB
:10B560007FF80D4904460860284623F079F80B4916
:10B5700005460860204623F01FF809490880284640
:10B5800023F01AF80749088270BD0000B8000020B7
:10B590008A0100205B010020B0010020B4010020DE
:10B5A000A60100207211002048437047C84000F0F7
:10B5B0000100704701238B40DBB20178002A02D0E2
:10B5C000194301707047DA4311400170704701233D
:10B5D0008B409BB20188002A02D01943018070473A
:10B5E000DA4311400180704701228A40D1B20078CD
:10B5F000084201D1002070470120704770B540F229
:10B600007F4005F0BEFDFE4D287040F2814005F000
:10B61000B8FD4FF6FF7404EA002068804FF4906094
:10B6200005F0AFFD69880844688040F2824005F06B
:10B63000A8FDF44D287040F2844005F0A2FD04EA14
:10B640000020688040F2834005F09BFD6988084433
:10B65000688040F2854005F094FDEB4D287040F283
:10B66000874005F08EFD04EA0020688040F28640A5
:10B6700005F087FD69880844688040F28E4005F037
:10B6800080FDE24D28704FF4926005F07AFD04EAE7
:10B690000020688040F28F4005F073FD69880844FF
:10B6A00068804FF4916005F06CFDD94D287040F230
:10B6B0008A4005F066FD04EA0020688040F2894077
:10B6C00005F05FFD69880844688070BD01EB0021CA
:10B6D00009B27F2801D908B27047084670472DE9A2
:10B6E000F84F6E2005F04DFDDFF8288388F86E00D6
:10B6F0000024012805D988F86E4000216E2005F04D
:10B7000041FD0025C44E40F27E47284605F039FD34
:10B71000A5F15F02A42A1FD298F86E1001EBC103B5
:10B7200003EB411106EBC10313F812C0844507D89F
:10B7300003EB42025278824202D308F805000DE082
:10B74000B64800EB8100284410F85F1C08F805108B
:10B75000284605F017FD01E008F805006D1CADB2A4
:10B76000BD42D2D398F85D00FF2801D188F85D4032
:10B77000AB4998F85D000870AB4D0222A9492846F4
:10B78000FCF712FFA74E327898F80610FE27FF2923
:10B790001CD0D9B1914205D03180012231462846D2
:10B7A000FCF711FF0025E946284605F0EAFC09F8F8
:10B7B00005006D1CADB2042DF6D39B4B9A4D9DF840
:10B7C000001010332035FF290FD01AE002229549CE
:10B7D0002846FCF7E9FE307888F80600FF2801D0FB
:10B7E0000028DFD188F80670DCE79DF80100FF280B
:10B7F00007D19DF80200FF2803D19DF80300FF2820
:10B800002ED0E1B398F80000814224D09DF80100C9
:10B8100098F8012090421ED09DF8022098F802501E
:10B82000AA4218D09DF8032098F80350AA4212D0DB
:10B83000318070801D4602227A492846FCF7C3FEFB
:10B840009DF8020030809DF8031071800222754936
:10B850002846FCF7B8FE98F8D902FF2830D036E029
:10B86000022270491846FCF79FFE307888F80000E5
:10B87000B07888F8010002226A49284600E008E012
:10B88000FCF792FE307888F80200B07888F8030060
:10B89000E1E7022263491846FCF786FE307888F813
:10B8A0000000B07888F8010002225E492846FCF7C3
:10B8B0007BFE307888F80200B07888F80300CAE789
:10B8C00088F8D942002140F2D92005F05BFC98F8B5
:10B8D0008303FF280DD188F8834388F88243002131
:10B8E00040F2823005F04EFC002140F2833005F03A
:10B8F00049FC98F883034B4D0002103D98F88213E1
:10B900000143698198F81B0098F81C10012600EB90
:10B91000012298F82F00454900EB0020824201D215
:10B920000E7000E00C7098F8310098F8322000EBAF
:10B93000022298F8450000EB0020824201D24E70AE
:10B9400000E04C7040F26D39484605F01AFC384969
:10B950000870FF2804D10C702146484605F012FCFF
:10B9600098F85C00334BFF2803D198F85B10FF294F
:10B970000AD098F85B10FFF7A9FE188098F8861394
:10B980002020FF290AD01BE01C8000215B2005F04D
:10B99000F9FB00215C2005F0F5FBEFE74F2188F86B
:10B9A0008613662188F8871388F8881388F88943F6
:10B9B00088F88A0388F88B0388F88C0388F88D034D
:10B9C00098F88E236F21FF2A11D14C2288F88E23FC
:10B9D00088F88F13772288F8902388F8914388F8A5
:10B9E000920388F8930388F8940388F8950398F8ED
:10B9F00096234FF0640BFF2A2FD14D221CE000004C
:10BA00002C11002036110020401100204A11002086
:10BA1000541100204D80002008EB020898ED020828
:10BA20005A0100207400002000770008A8010020BF
:10BA3000880300209401002088F89623652288F866
:10BA4000972388F898B388F8994388F89A0388F878
:10BA50009B0388F89C0388F89D0398F89E23FF2A8F
:10BA600011D1482288F89E23692288F89F2388F8FC
:10BA7000A04388F8A10388F8A20388F8A30388F8F4
:10BA8000A40388F8A50398F8A623FF2A12D141221F
:10BA900088F8A623752288F8A723742288F8A8239B
:10BAA00088F8A91388F8AA4388F8AB0388F8AC0390
:10BAB00088F8AD0398F88E034C2800D0EE7098F803
:10BAC000ED00FF2806D0C0EB00104FF6FF7101EA31
:10BAD0008000288198F8AE03FF2801D188F8AE4392
:10BAE00098F89702FF2811D198F89602FF280DD1F7
:10BAF000002140F2972005F045FB88F8974201218C
:10BB000040F2962005F03EFB88F8966298F83204E1
:10BB1000FF280ED1002505F2324080B2002105F049
:10BB200031FB08EB050080F832446D1CADB22E2DC0
:10BB3000F1D315F07BFE98F882004546022801D922
:10BB400085F8824095F89200012805D985F8924041
:10BB5000FA48032180F82B1040F2914005F011FBC8
:10BB6000F74900EB8000400008804FF47A72904261
:10BB700001D90A8005E0B0F5FA7F02D24FF42F70A8
:10BB8000088040F2924005F0FCFAEE490870FFF799
:10BB900035FD95F8F102FF2800D010B9A02085F8F6
:10BBA000F102E949A879087040F2944A504605F03C
:10BBB000E8FADFF8989340F29548FF2804D1404610
:10BBC00005F0DFFAFF283AD0504605F0DAFAC9F856
:10BBD0000000404605F0D5FAD9F8001041EA0020EF
:10BBE000C9F8000040F2964005F0CBFAD9F80010F1
:10BBF00041EA0040C9F8000040F2974005F0C1FA60
:10BC0000D9F8001041EA0060C9F800000021DFF80F
:10BC10004093002001EB41024FEA820801EB410210
:10BC200009EBC20208EB40032B4493F8BAC3BCF102
:10BC3000180F11D902EB400C8CF8014010E0287865
:10BC4000697840EA0120A97840EA0140E97840EAB1
:10BC50000160C9F80000D9E702EB400A8AF801C088
:10BC600093F8BB333B2B02D902F8104001E002F8F5
:10BC70001030401C80B20628D4D3491C89B2082950
:10BC8000C7D30020B3492A1892F832240A54401C22
:10BC900080B22E28F7D395F87D043238652801D379
:10BCA00085F87DB440F29A4005F06BFADFF8A8827F
:10BCB0000002A8F8000040F2994005F062FAB8F8D6
:10BCC00000100843A8F8000040F29C4005F059FA23
:10BCD000DFF888820002A8F8000040F29B4005F0DF
:10BCE00050FAB8F800100843A8F800004FF0000818
:10BCF000A14605EB080090F86712FF2907D180F8EC
:10BD0000679208F2672080B2002105F03BFA08F143
:10BD100001081FFA88F8B8F1090FEAD395F88101F4
:10BD2000FF2806D185F88191002140F2811005F0AD
:10BD300029FA95F88001FF2806D185F88091002125
:10BD40004FF4C07005F01EFA0021854ADFF8148216
:10BD5000002008EB811343F82020401C80B21028FB
:10BD6000F9D3491C89B20029F2D0744890F82B000D
:10BD7000032838D10024DFF8F0B10BF26B3A0BF155
:10BD8000D60BE1B25846FFF72FFC40B1E1B2504666
:10BD9000FFF72AFC22F064FC08EB8411C861641CE4
:10BDA000A4B2052CEDD305215846FFF71DFC50B178
:10BDB00095F8670395F86813000200B2084422F072
:10BDC00037FCC8F85C0106215846FFF70DFC50B15E
:10BDD00095F8690395F86A13000200B2084422F04E
:10BDE00027FCC8F89C0195F86403FF2812D195F848
:10BDF00065132846FF290DD180F8649380F8659378
:10BE000000214FF4597005F0BDF9002140F2653072
:10BE100005F0B8F9E8793E2805D03E21072005F065
:10BE2000B1F93E20E87195F85F0040F266341528BC
:10BE300005D1314685F86663204605F0A3F995F8EB
:10BE4000A200152805D1314685F86663204605F025
:10BE500099F94FF4187005F094F94449087095F871
:10BE60007702FF280BD195F87802FF2807D185F8D3
:10BE7000779285F8789285F8799285F87A923C4A9B
:10BE800095F86202010295F861320B431380FF2896
:10BE900001D1A2F8009040F2A144204605F0CCF870
:10BEA00034490870FF2801D0012804D80F703946A2
:10BEB000204605F0E2F840F2F644204605F0BCF8D2
:10BEC0002D4A1070012806D028B1494682F800900A
:10BED000204605F0D2F80024284E04F20150054611
:10BEE00080B205F0A9F83055FF2804D1E1B23155F0
:10BEF000A8B205F0C2F8641CA4B2042CEDD340F241
:10BF0000055005F099F83071BDE8F88F1CB5024670
:10BF10000846843A1A4CC1B2072A0ED2DFE802F072
:10BF200004323D0D48535D00A1786278CDE90021CF
:10BF30002378E279A17905F030FA1CBD491600207A
:10BF40001C020020820300208D0300201800002026
:10BF50009A8500206C850020A00100209E01002011
:10BF600000007F432C8500204D800020FC01002034
:10BF70009A010020560400204B0100204C010020B3
:10BF800018110020A1786278CDE900212378E279A8
:10BF9000C1B2A08805F001FACFE7A1786278CDE9B7
:10BFA00000212378A179C2B2A08805F0F6F9C4E790
:10BFB000A1786278CDE90021E279C3B2A179A088A5
:10BFC00005F0EBF9B9E7A078CDE900102378E27924
:10BFD000A179A08805F0E1F9AFE76078CDE900012B
:10BFE0002378E279A179A08805F0D7F9A5E710B503
:10BFF00001210F2005F0C6F80021102005F0C2F83D
:10C000000121112005F0BEF80021BDE810401220EA
:10C0100005F0B8B870B50024FE4D04F5B070295D88
:10C0200005F0B0F8641CE4B2072CF6D370BD70B50F
:10C030000024F94D24F00100295C04F11B0005F0F7
:10C04000A1F8A41CE4B2152CF4D3012424F00100BF
:10C05000285A010A04F11B0005F094F8A41CE4B26C
:10C06000162CF3D30024ED4D24F00100295C04F1DB
:10C07000310005F087F8A41CE4B2152CF4D3012498
:10C0800024F00100285A010A04F1310005F07AF881
:10C09000A41CE4B2162CF3D370BD2DE9F0410025A9
:10C0A000DFF87C830024C5EBC50000EB080605EB38
:10C0B00085073819315D00F5A17005F063F8641C3F
:10C0C000E4B2052CF5D36D1CEDB2022DEAD3BDE828
:10C0D000F08170B50024D34D04F22D10295D05F0D8
:10C0E00051F8641CE4B2152CF6D370BD2DE9F04173
:10C0F00007460024CC4D0126062F21D2DFE807F0A9
:10C100007F037F214462C948015D04F2031005F0FA
:10C1100039F8012C07D10321A02005F033F80321C1
:10C12000A12005F02FF8072C04D2002104F1B20061
:10C1300005F028F801216F2005F024F885F86F60DC
:10C140005DE0BB48015D04F2031005F01BF8012C13
:10C1500007D10221A02005F015F80221A12005F049
:10C1600011F8072C04D2002104F1B20005F00AF8FE
:10C1700004219B2005F006F803216F2005F002F84A
:10C18000032085F86F003AE0AA48015D04F203102D
:10C1900004F0F8FF012C07D10221A02004F0F2FFE7
:10C1A0000221A12004F0EEFF072C04D2002104F1AB
:10C1B000B20004F0E7FF01216F2004F0E3FF85F8EF
:10C1C0006F601CE09C48015D04F2031004F0DAFF8C
:10C1D000012C07D10221A02004F0D4FF0221A120CC
:10C1E00004F0D0FF072C04D2002104F1B20004F0C7
:10C1F000C9FF01216F2004F0C5FF85F86F60641C42
:10C20000E4B22A2CFFF478AF61E72DE9F05F5F24F8
:10C210008A4E854D4FF48177652C19D095F86E00C4
:10C2200000EBC00101EB401006EB8000204410F849
:10C230005F1C204604F0A6FF95F86E0000EBC001DD
:10C2400001EB401006EB8000204410F85F0C2855ED
:10C25000641CA4B2BC42DFD995F86E1040F2592696
:10C26000741C11B1012913D024E0C821304604F018
:10C2700089FF0021204604F085FF304604F081FF4D
:10C2800085F85902204604F07CFF85F85A0211E037
:10C29000A821304604F076FF0221204604F072FF08
:10C2A000304604F06EFF85F85902204604F069FF1D
:10C2B00085F85A0262480078FFF718FFFFF709FF78
:10C2C000FFF7EBFEFFF7B3FEFFF7A4FEFFF78FFECD
:10C2D0004F2140F2863004F055FF662140F287304E
:10C2E00004F050FF66214FF4627004F04BFF002110
:10C2F00040F2893004F046FF202140F28A3004F0F9
:10C3000041FF202140F28B3004F03CFF20214FF40C
:10C31000637004F037FF202140F28D3004F032FFCB
:10C320004C2140F28E3004F02DFF6F2140F28F300F
:10C3300004F028FF77214FF4647004F023FF0021FC
:10C3400040F2913004F01EFF202140F2923004F0C0
:10C3500019FF202140F2933004F014FF20214FF404
:10C36000657004F00FFF202140F2953004F00AFFC1
:10C370004D2140F2963004F005FF652140F29730E0
:10C3800004F000FF64214FF4667004F0FBFE00210E
:10C3900040F2993004F0F6FE202140F29A3004F089
:10C3A000F1FE202140F29B3004F0ECFE20214FF4FE
:10C3B000677004F0E7FE202140F29D3004F0E2FEB9
:10C3C000482140F29E3004F0DDFE692140F29F30AA
:10C3D00004F0D8FE00214FF4687004F0D3FE202151
:10C3E00040F2A13004F0CEFE202140F2A23004F051
:10C3F000C9FE202140F2A33004F0C4FE20214FF4F6
:10C40000697004F0BFFE202140F2A53004F0BAFEAE
:10C41000412117E0C7EA020886EA02089CEA0208FE
:10C4200088EF0208B2EA02084D800020E0EE020820
:10C430000AEF020834EF02085EEF020898ED0208E6
:10C44000A700002040F2A63004F09CFE752140F2C7
:10C45000A73004F097FE74214FF46A7004F092FE46
:10C460006F2140F2A93004F08DFE002140F2AA3085
:10C4700004F088FE202140F2AB3004F083FE20213E
:10C480004FF46B7004F07EFE202140F2AD3004F0DA
:10C4900079FE0021922004F075FE002448274FF019
:10C4A000470807EB4406B0B204F06BFEFF2809D141
:10C4B00008EB440080B2002104F064FEB0B2002119
:10C4C00004F060FE641CA4B2082CEAD3012085F8B5
:10C4D000B80201214FF42E7004F054FE0E2140F2F8
:10C4E000BA2004F04FFE0E2085F8BA0295F84D03ED
:10C4F00020274FF07208FF2875D105F24D354120F5
:10C5000028706920687085F802804C20E8706120EE
:10C51000287162206871AF71EF71A5F24D3541212C
:10C5200040F24D3004F02EFE692140F24E3004F00E
:10C5300029FE722140F24F3004F024FE4C214FF4CA
:10C54000547004F01FFE612140F2513004F01AFED5
:10C55000622140F2523004F015FE002140F25330C7
:10C5600004F010FE00214FF4557004F00BFE002182
:10C5700040F2553004F006FE002140F2563004F03F
:10C5800001FE002140F2573004F0FCFD00214FF481
:10C59000567004F0F7FD002140F2593004F0F2FD2E
:10C5A000002140F25A3004F0EDFD002140F25B30F2
:10C5B00004F0E8FD00214FF4577004F0E3FD002182
:10C5C00040F25D3004F0DEFD002140F25E3004F008
:10C5D000D9FD002140F25F3004F0D4FD00214FF47A
:10C5E000587004F0CFFD0024FE4E04F2CC4080B21F
:10C5F00004F0C7FD3055641CA4B2142CF5D3307878
:10C600004FF06F094FF0540B4FF0630AFF2801D031
:10C6100000287BD186F800B0652070706D20B07066
:10C6200086F803A086F80490432070717420B071DE
:10C6300086F8078086F808906C2070727320B072BC
:10C64000F7723773542140F2CC4004F09BFD652112
:10C6500040F2CD4004F096FD6D2140F2CE4004F052
:10C6600091FD632140F2CF4004F08CFD6F214FF427
:10C670009A6004F087FD432140F2D14004F082FD2E
:10C68000742140F2D24004F07DFD722140F2D3408B
:10C6900004F078FD6F2140F2D44004F073FD6C216A
:10C6A00040F2D54004F06EFD732140F2D64004F014
:10C6B00069FD002140F2D74004F064FD00214FF4F1
:10C6C0009B6004F05FFD002140F2D94004F05AFD68
:10C6D000002140F2DA4004F055FD002140F2DB4039
:10C6E00004F050FD002140F2DC4004F04BFD00213D
:10C6F00040F2DD4004F046FD002140F2DE4004F04F
:10C7000041FD002140F2DF4004F03CFD0024B54E25
:10C71000143604F59C6080B204F033FD3055641C7F
:10C72000A4B2142CF5D33078FF2801D000287CD196
:10C7300086F800B0652070706D20B07086F803A098
:10C7400086F8049077715020B07186F8078086F8DB
:10C750000890642070727520B07286F80BA0742067
:10C76000307354214FF49C6004F00CFD652140F2BD
:10C77000E14004F007FD6D2140F2E24004F002FDCB
:10C78000632140F2E34004F0FDFC6F2140F2E440FD
:10C7900004F0F8FC202140F2E54004F0F3FC5021C5
:10C7A00040F2E64004F0EEFC722140F2E74004F073
:10C7B000E9FC6F214FF49D6004F0E4FC642140F239
:10C7C000E94004F0DFFC752140F2EA4004F0DAFCB5
:10C7D000632140F2EB4004F0D5FC742140F2EC40C0
:10C7E00004F0D0FC002140F2ED4004F0CBFC00212D
:10C7F00040F2EE4004F0C6FC002140F2EF4004F0AD
:10C80000C1FC00214FF49E6004F0BCFC002140F20A
:10C81000F14004F0B7FC002140F2F24004F0B2FC19
:10C82000002140F2F34004F0ADFC40F2F546304602
:10C8300004F0A7FC0446771E384604F0A2FC04EB83
:10C840000020694C81B2E181A1F57F40FF3800D022
:10C8500049B99420E0810021384604F093FCA17B83
:10C86000304604F08FFCC82140F2AF3004F08AFC5F
:10C8700000214FF46C7004F085FCC82140F2B13007
:10C8800004F080FC002140F2B23004F07BFC28214F
:10C8900040F2B33004F076FC10214FF46D7004F0D8
:10C8A00071FC1E2140F2B53004F06CFC0F2140F207
:10C8B000B63004F067FC322140F2B73004F062FC7D
:10C8C00005214FF46E7004F05DFC06214FF4A87052
:10C8D00004F058FC1E2140F2511004F053FC0821D2
:10C8E0004FF4A97004F04EFC1E2140F2531004F0E6
:10C8F00049FC12214FF4AA7004F044FC1E2140F2BE
:10C90000551004F03FFC16214FF4AB7004F03AFCD4
:10C910001E2140F2571004F035FC002140F2B920EE
:10C9200004F030FC95F89702FF280DD195F8960297
:10C93000FF2809D1002140F2972004F023FC0121B7
:10C9400040F2962004F01EFC40F2E1718420FFF7D3
:10C95000DDFA00240026281990F86712FF2907D174
:10C9600080F8676204F2672080B2002104F00AFCBC
:10C97000641CA4B2092CEED3002404F5A17080B28B
:10C98000002104F0FFFB641CA4B2072CF5D30024A3
:10C9900004F2491080B2002104F0F4FB641CA4B23C
:10C9A000072CF5D3BDE8F09F2DE9F0410F4C40F284
:10C9B0005A26204694F86E10771E90F87E000029C3
:10C9C0007ED000EBC0000525B0FBF5F020307B34B5
:10C9D000C1B2E1707E2004F0D5FBA07800EBC0006E
:10C9E00006E00000C8080020640000204D80002000
:10C9F000B0FBF5F02030C1B2A1707D2004F0C2FB85
:10CA000014F8040C00EBC000B0FBF5F02030C1B20C
:10CA100004F8041C772004F0B5FB94F8660000EBE2
:10CA2000C000B0FBF5F02030C1B284F86610E12000
:10CA300004F0A8FB94F8DE0194F8DF1100EB01206C
:10CA400080B200EBC000B0FBF5F000F5A07082B240
:10CA5000110A84F8DF1184F8DE21304604F092FBDD
:10CA600094F8DE11384604F08DFBA07EE17E00EBE9
:10CA7000012080B200EBC000B0FBF5F000F5A07023
:10CA800080B2010AE176A076962004F07BFBA17EBD
:10CA9000952004F077FB207F617F00EB012080B2BE
:10CAA00000EBC000B0FBF5F000F5A07080B2010A09
:10CAB00061772077982004F065FB217F972000E0C4
:10CAC00048E004F05FFBA07FE17F00EB012080B233
:10CAD00000EBC000B0FBF5F000F5A07080B2010AD9
:10CAE000E177A0779A2004F04DFBA17F992004F014
:10CAF00049FB14F8070D617800EB012080B200EBD0
:10CB0000C000B0FBF5F000F5A07080B2010A6170C2
:10CB10002070752004F036FB14F8071B742004F015
:10CB200031FB14F8090D617800EB012080B200EBB5
:10CB3000C000B0FBF5F000F5A07080B2010A617092
:10CB40002070732004F01EFB2178BDE8F0417220B4
:10CB500004F018BB2038C0B2092500EB8000B0FB00
:10CB6000F5F07B34C1B2E1707E2004F00BFBA078BD
:10CB70002038C0B200EB8000B0FBF5F0C1B2A1706C
:10CB80007D2004F0FFFA14F8040C2038C0B200EB4A
:10CB90008000B0FBF5F0C1B204F8041C772004F06B
:10CBA000F1FA94F866002038C0B200EB8000B0FBC8
:10CBB000F5F0C1B284F86610E12004F0E3FA94F8CD
:10CBC000DE0194F8DF1100EB0120A0F5A07080B227
:10CBD00000EB8000B0FBF5F082B2110A84F8DF119F
:10CBE00084F8DE21304604F0CDFA94F8DE113846A0
:10CBF00004F0C8FAA07EE17E00EB0120A0F5A07051
:10CC000080B200EB8000B0FBF5F080B2010AE17663
:10CC1000A076962004F0B6FAA17E952004F0B2FA30
:10CC2000207F617F00EB0120A0F5A07080B200EBB7
:10CC30008000B0FBF5F080B2010A61772077982080
:10CC400004F0A0FA217F972004F09CFAE17FFA4ECD
:10CC5000A07F06EB0121084480B200EB8000B0FB0E
:10CC6000F5F080B2010AE177A0779A2004F08AFA01
:10CC7000A17F992004F086FA14F8070D617806EB7D
:10CC80000121084480B200EB8000B0FBF5F080B2D7
:10CC9000010A61702070752004F074FA14F8071B03
:10CCA000742004F06FFA14F8090D617806EB012185
:10CCB000084480B200EB8000B0FBF5F080B2010ABE
:10CCC00061702070732004F05DFA2178BDE8F041B6
:10CCD000722004F057BA10B5D84C012823D09A20FE
:10CCE00004F04FFA703484F82A00992004F049FACD
:10CCF00084F82900702004F044FA2070712004F0B8
:10CD000040FA6070752004F03CFA6071742004F001
:10CD100038FA2071732004F034FAE070722004F0C5
:10CD200030FAA07010BD40F25A2004F02AFA79348B
:10CD300084F8E10140F2592004F023FA84F8E0017C
:10CD40006C2004F01EFA04F80D0C6D2004F019FAA2
:10CD500004F80C0C962004F014FA6077952004F087
:10CD600010FA2077982004F00CFAE077972004F06E
:10CD700008FAA07710BDFCF7E3B900218438B04A67
:10CD8000072812D2DFE800F004060A080C0E100093
:10CD900091880AE0917908E0117A06E0D17904E0FF
:10CDA000117802E0517800E0917808B270474FF4B2
:10CDB0007A700CF061BD10B504F045F8802004F0E5
:10CDC000BCF804F06DF808B1002010BDFE2004F09E
:10CDD000B4F804F065F808B1002010BD04F049F87B
:10CDE000012010BD10B5044604F02DF8802004F099
:10CDF000A4F804F055F808B1002010BD3CB1F520AE
:10CE000004F09BF804F04CF828B1002010BDF3208A
:10CE100004F093F8F6E704F02CF8012010BD70B58B
:10CE20000E4604F010F8812004F087F804F038F87A
:10CE3000012004F0A3F84FF6FF7101EA002501205C
:10CE400004F09CF840EA0504002004F097F804F090
:10CE500010F83480012070BD01F00203834201D03C
:10CE60000020704721F0030150B140F2E2404143FD
:10CE7000C81701EB104000143C38108001207047A7
:10CE800044F2A4404143C81701EB10400014A0F540
:10CE900090504D3800B20A2190FBF1F01080EDE780
:10CEA00070B5054603F0CFFF812004F046F803F08B
:10CEB000F7FF08B1002070BD012004F05FF84FF6C5
:10CEC000FF7101EA0024012004F058F8204484B2E4
:10CED000002004F053F803F0CCFF022D0AD044F2F6
:10CEE000A440444357480A2100EB244090FBF1F052
:10CEF00080B270BD40F2E24044436FF03B0000EB73
:10CF00002440F5E710B503F09EFF802004F015F8EB
:10CF100003F0C6FF08B1002010BDE72004F00DF8B3
:10CF200003F0BEFF08B1002010BD03F08CFF81208C
:10CF300004F003F803F0B4FF08B1002010BD002096
:10CF400004F01CF8044603F094FFE0B210BD70B585
:10CF50000646C1F1FA0020F00EFF4FF033323A4B93
:10CF600020F070FF04460D46304620F004FF2246B4
:10CF70002B4620F053FC20F0A1FE00B270BD2DE93D
:10CF8000F0470446084621F053FB304921F01EFAD1
:10CF900021F082F920F028FA20F00EFC0646204607
:10CFA00020F0E9FE2A4F0D46044600223B4620F0C1
:10CFB00049FF20F001FC8146DFF89880DFF898A057
:10CFC000204629464246534620F028FC04460D469A
:10CFD000484621F061F922462B4620F0DBFC20F088
:10CFE000EBFB0146304621F083F921F055F98946E3
:10CFF000064600223B4621F059F804460D463046CD
:10D0000049464246534620F01DFF22462B4620F05B
:10D01000C1FC20F053FE00B2BDE8F087632140F26E
:10D02000853004F0AFB806498A8892071FD08A7904
:10D030000D2A29D212E00000C0FEFFFF4D80002023
:10D0400018110020B3EDFFFF3333C3BF00007A4453
:10D0500000A03140CDCCCCCCCCFCA240DFE802F02B
:10D0600014393B3E4144474A4D5053575B008A793F
:10D070000D2A09D2DFE802F00807090C0F12151873
:10D080001B1E21252900C8797047C8791F307047B9
:10D09000C8793B307047C8795A307047C8797830C2
:10D0A0007047C87997307047C879B5307047C879EC
:10D0B000D4307047C879F3307047C87900F2111046
:10D0C0007047C87900F598707047C87900F5A77067
:10D0D0007047C8797047C8791F307047C8793C30AD
:10D0E0007047C8795B307047C87979307047C87924
:10D0F00098307047C879B6307047C879D5307047D6
:10D10000C879F4307047C87900F589707047C879DC
:10D1100000F231107047C87900F24F10704700B527
:10D12000FFF781FFF8498881C0F3C70200F00701CB
:10D13000F648104400F23240FEF756FA08B10120DA
:10D1400000BD002000BD2DE9F043F04DEE49012661
:10D150006A7AEF4F8B794FF0040C02F0FE044FF027
:10D16000000805280FD2DFE800F00E03101E210092
:10D170000E7142F0010068724E7181F806C081F8AC
:10D1800002C0BE71BE70BDE8F08381F804C06C724D
:10D1900081F80580002BF6D081F8068081F80280A6
:10D1A000BE71BE70EFE70A200871ECE70C20087131
:10D1B0006C7281F80580002BE5D081F8068081F83B
:10D1C0000280BE71BE70DEE710B5D24A147A002C20
:10D1D00003D0127A012902D002E00722FAE70822DE
:10D1E000CA4907283AD2DFE800F039040D161F2893
:10D1F0003100521E02EB4200084490F81A0400F07D
:10D2000007032BE0521E02EB4200084490F81A0478
:10D21000C0F3C20322E0521E02EB4200084490F821
:10D220001B0400F0070319E0521E02EB4200084401
:10D2300090F81B04C0F3C20310E0521E02EB420040
:10D24000084490F81C0400F0070307E0521E02EBAC
:10D250004200084490F81C04C0F3C20358B210BD49
:10D260002DE9FC5F002714F0E1FAAA48007AE8B340
:10D27000A848007A401E00F0FF09FFF750FFA64AB9
:10D2800000287CD0A54801784478C1EB011104EB5B
:10D290008104A3490C808378C478C3EB031304EBA7
:10D2A00083034B8003794479C3EB031304EB8303BB
:10D2B0008B808379C479C3EB031304EB8303CB80A6
:10D2C000037A447AC3EB031304EB83030B81C37A21
:10D2D000807AC0EB001003EB80004881002409EB4A
:10D2E000490802EB4805285DFF2800E001E003D073
:10D2F00037E04FF00609C0E789494FF6FF7021F883
:10D30000140008EB5400814A01901044009090F8FA
:10D310001A04E10741D0C10801F0030109B3E10794
:10D320003ED000F0C70AFF2109EB4900800000EB66
:10D33000440B0BEB020080F8BA1380F8BB130BF21E
:10D34000BA3003F01FFF0BF2BB30FF2103F01AFFCE
:10D35000009880F81AA40198514600F21A4003F090
:10D3600011FF641CE4B2062CBDD3DFF89C9199F840
:10D370000000E8B300206A4901F10E0200E0D1E0AC
:10D3800031F8103022F81030401CC0B20628F5D316
:10D3900005244FF0000C00211FE000F00301BDE761
:10D3A00000F0F80ABFE7481C32F8113032F810A03C
:10D3B000534511D90127938132F8103022F81130EA
:10D3C000938922F8103015F801A06B1893F801B07A
:10D3D00005F801B083F801A0C1B2A142E3D3641EF5
:10D3E000E4B20CF1010C0CF0FF0CBCF1060F00E0F4
:10D3F00003E0D0D3002089F80000CFB30024434FCE
:10D4000008EB5402D31993F81A14E00706D0285DEC
:10D41000012817D0D8B1FF281ED01FE0285D0128B1
:10D4200003D038B1FF280AD018E001F0F80040F02E
:10D43000010113E001F0F80040F002010EE001F0FC
:10D44000F8010BE001F0C70040F0080106E001F030
:10D45000C70040F0100101E001F0C70183F81A1481
:10D4600002F21A4003F08EFE641CE4B2062CC7D30D
:10D47000284841780078C0EB001001EB8004284D6B
:10D480000E352888A04207D86888A04204D9012117
:10D490000846FFF799FEC6B26888A04207D8A88858
:10D4A000A04204D901210220FFF78EFEC6B2A8884F
:10D4B000A04207D8E888A04204D901210320FFF741
:10D4C00083FEC6B2E888A04207D82889A04204D9C2
:10D4D00001210420FFF778FEC6B22889A04207D8B0
:10D4E0006889A04204D901210520FFF76DFEC6B26C
:10D4F0006889A04204D801210620FFF765FEC6B264
:10D500003046BDE8FC5F1EE6640000204D80002030
:10D510002211002018110020FA8400205B840020D2
:10D52000AC080020BE4809EB490800EB880000F277
:10D53000BA3001784478C1EB011104EB8104B94998
:10D540000C808378C478C3EB031304EB83034B8014
:10D5500003794479C3EB031304EB83038B80837952
:10D56000C479C3EB031304EB8303CB80037A447ABF
:10D57000C3EB031304EB83030B81C37A807AC0EB04
:10D58000001003EB80004881002402EB4805285D71
:10D59000FF2832D1A3484FF6FF7120F8141021461E
:10D5A000484614F033F9E10741D0C10801F0030106
:10D5B00019B3E1073ED000F0C70AFF2109EB49008B
:10D5C000800000EB440B9648584480F8BA1380F86A
:10D5D000BB130BF2BA3003F0D5FD0BF2BB30FF21C9
:10D5E00003F0D0FD8E4908EB5400014481F81AA4E1
:10D5F00000F21A40514603F0C5FD641CE4B2062C4B
:10D60000C5D3DFF8249299F80000E8B300208549DB
:10D6100001F10E0231F8103022F81030401CC0B277
:10D620000628F7D305244FF0000C00211FE000F07E
:10D630000301BDE700F0F80ABFE7481C32F81130DB
:10D6400032F810A0534511D90127938132F81030D8
:10D6500022F81130938922F8103015F801A06B18C8
:10D6600093F801B005F801B083F801A0C1B2A1425E
:10D67000E3D3641EE4B20CF1010C0CF0FF0CBCF11E
:10D68000060FD2D3002000E001E089F80000CFB3FC
:10D690000024634F08EB5402D31993F81A14E007DF
:10D6A00006D0285D012817D0D8B1FF281ED01FE072
:10D6B000285D012803D038B1FF280AD018E001F016
:10D6C000F80040F0010113E001F0F80040F0020121
:10D6D0000EE001F0F8010BE001F0C70040F0080196
:10D6E00006E001F0C70040F0100101E001F0C701C1
:10D6F00083F81A1402F21A4003F044FD641CE4B2E9
:10D70000062CC7D3494841780078C0EB001001EBE4
:10D710008004444D0E352888A04207D86888A0426E
:10D7200004D900210120FFF74FFDC6B26888A0424E
:10D7300007D8A888A04204D900210220FFF744FDA1
:10D74000C6B2A888A04207D8E888A04204D9002120
:10D750000320FFF739FDC6B2E888A04207D8288920
:10D76000A04204D900210420FFF72EFDC6B228896B
:10D77000A04207D86889A04204D900210520FFF7FC
:10D7800023FDC6B26889A04204D800210620FFF715
:10D790001BFDC6B23046FFF7D6FC99F80100864261
:10D7A00004D02349012008718870487089F801600D
:10D7B000BDE8FC9FF0B5034619481A4CC51844341F
:10D7C00095F86702FF2824D0002658B1411E012792
:10D7D00005290BD2C9B21748FDF706FF012803D06F
:10D7E000E65416E0E65414E0E75412E01249062825
:10D7F00006D1B1F90020002A01DDE75400E0E6542B
:10D80000072806D1B1F90200002801DDE75400E045
:10D81000E65495F86702002801D16420E054F0BD79
:10D820004D800020AC08002064000020181100206A
:10D830002211002018020020EE0000202DE9F04106
:10D84000FC4C0023A370E370FC4D3C24FA4F1826D7
:10D8500005EB8203002904D0012939D0022968D1BF
:10D8600057E0B0FBF4F104FB110197F802C06144EA
:10D87000C9B2B1FBF4FCB1FBF4F804FB1811D97088
:10D88000B0FBF4F104FB1101401A80B2B0FBF4F0DC
:10D89000B0FBF4F104FB1101614497F801C061444D
:10D8A000C9B2B1FBF4FCB1FBF4F804FB1811997098
:10D8B000B0FBF4F0397860440844C0B2B0FBF6F134
:10D8C000B0FBF6F406FB1400587005F8221030E0A7
:10D8D000B978D970B0FBF4F104FB110197F801C0DD
:10D8E0006144C9B2B1FBF4FCB1FBF4F804FB1811BC
:10D8F0009970B0FBF4F0397860440844C0B2B0FBD2
:10D90000F6F1B0FBF6F406FB1400587005F822108F
:10D910000FE0B978D9707978997039780844C0B235
:10D92000B0FBF6F1B0FBF6F406FB1400587005F8F6
:10D930002210D8783B2801D13A20D870BDE8F08178
:10D9400010B5BC4BBD49BC4A002814D011F820408A
:10D95000DB789C422FD101EB80001378417899420B
:10D9600027D181785378994221D1C0789178884223
:10D970001BD8012010BD08789B78984213D14878B5
:10D98000137898420DD188785378984207D1C87897
:10D990009178884201D8012010BD002010BD0020E0
:10D9A00010BD002010BD002010BD002010BD0020C3
:10D9B00010BD002010BD002010BD2DE9F14FDFF893
:10D9C000748298F80C0001285AD10024814608F18D
:10D9D0003E0B4FF0000A08F11A06994F4DE0651C06
:10D9E000E8B2FFF7ADFF012801D1315D11B1012887
:10D9F0002CD041E097F8DB00032813D017F8CB0FA9
:10DA0000797800EB012080B2A8F8240006F8049091
:10DA1000397ACB3F0122FFF711FF97F8DB0002288C
:10DA20000DD029E006F80490EAB23BF8140000217A
:10DA3000FFF704FF7F483B3000F80490EDE706F85D
:10DA400004A088F80AA088F80CA015E0305D012831
:10DA500012D197F8DB00032814D017F8CD0F79788E
:10DA600000EB012080B2A8F8240006F804A0B979E0
:10DA7000CD3F0122FFF7E2FEECB200988442AED324
:10DA8000BDE8F88F6B48423030F8140030B106F82A
:10DA900004A0EAB20021FFF7D1FEEDE706F80490FA
:10DAA000EAB23BF814000021FFF7C8FEE4E7D21CFD
:10DAB000884205D1D1B25F4800221830FDF787BDFA
:10DAC000D1B25C4801221830FDF781BD10B5044683
:10DAD000002903D05749002032310855554801220A
:10DAE00021461830FDF773FDE41CE1B251480022D5
:10DAF000BDE810401830FDF76ABD10B504464D482A
:10DB00002630015D4F48005D821C91420DD9494885
:10DB1000002221461030FDF75AFD214645480122DA
:10DB2000BDE810401230FDF752BD801E81420DDA73
:10DB30004048012221461030FDF749FD21463D486D
:10DB40000022BDE810401230FDF741BD39480022E7
:10DB500021461030FDF73BFD214636480022BDE846
:10DB600010401230FDF733BD2DE9F04F89B0044667
:10DB7000334EDFF8C09096F86B00002807D00128DC
:10DB800044D0314F02287ED0032810D1AAE099F862
:10DB9000050006280CD096F8AE03022815D00128FF
:10DBA00013D02046FFF7A9FF0120FFF7A6FFC1E031
:10DBB0002048012200211030FDF709FD1D480022F8
:10DBC00011461230FDF703FDB4E00120FFF795FF89
:10DBD00096F8AE0302280CD016480122002110301E
:10DBE000FDF7F5FC1348002211461230FDF7EFFC5B
:10DBF000DAE71048002211461030FDF7E8FC0D4826
:10DC0000012200211230FDF7E2FCCDE70120FFF7F1
:10DC100074FF99F80400C8B106480022114610307C
:10DC2000FDF7D5FC0348012200211230FDF7CFFC9F
:10DC300017E028E0A200002018110020F9080020B9
:10DC40004D800020B2030020BE03002001220021ED
:10DC5000FE48FDF7BCFCFD4800221146801CFDF784
:10DC6000B6FC99F80B0070B3401E89F80B00002237
:10DC70001146F648FDF7ABFCF44800221146801C23
:10DC8000FDF7A5FC56E096F89F02052804D096F80B
:10DC90009E02052807D00AE07888012801D00025D7
:10DCA00005E0012503E0388801280DD000256DB17D
:10DCB00000221146E548FDF78AFCE44801220021D4
:10DCC000801CFDF784FC35E00125F0E701220021EE
:10DCD000DE48FDF77CFCDD4800221146801CFDF784
:10DCE00076FC27E00221DA48FDF77EFC10B901201E
:10DCF00089F8070096F89F02052804D096F89E023E
:10DD0000052807D00AE07888012801D0002505E021
:10DD1000012503E0388801285DD00025F5B30122F4
:10DD20000021CA48FDF753FCC84800221146801C58
:10DD3000FDF74DFCA020A0EB4407C548C349D438EB
:10DD4000C44AC05D253104EB440B02EB4B080026AE
:10DD500028B3062856D010F808000855C81C12F839
:10DD60001B200255DFF8E4A20AF1160A0AF10F019E
:10DD70001AF80400095D0AF10905884204D305F187
:10DD80000901095D884224D9B148D43890F8790056
:10DD9000022801D004283DD8214601E01DE028E0FA
:10DDA000B9F81200FDF702FC30B1A8481AF80410C7
:10DDB0002830005D81420CD32146B9F81000FDF7F0
:10DDC000F5FB38B3A1481AF804102530005D8142F4
:10DDD00020D92E5569E10125A0E7002211469B4874
:10DDE000FDF7F5FB994801220021801CFDF7EFFBB0
:10DDF000A0E79648642228300255964810F81B0088
:10DE00000855AFE70E55934810F81B208F4828306F
:10DE10000255A7E72146B9F81000FDF7C7FBD0B3BC
:10DE20000021A1208A4AA0EB4400D43ADFF824E282
:10DE3000105C05AB08E0D25D01EB4B0C724412F8AC
:10DE40000C205A54491CC9B2814AD43A8842F2D8AB
:10DE50000022C0F1060C06E003EB020B022100F8E1
:10DE60000B10521CD2B29445F6DC1AF804004FF0A5
:10DE7000030E032802D802460AF804E01AF8040048
:10DE80009DF819C0CDF820C0ACF1020C604503DA52
:10DE9000062129551BE06FE09DF81410884201D936
:10DEA0002E5514E0002103EB010B9BF801B05845FF
:10DEB00009D913F801B0ABF1020B584503DA01F1AF
:10DEC000010B05F804B0491CC9B20429EBD39DF835
:10DED00014108B1E984207DB884205D8295D012962
:10DEE00002D009B1012129559DF815108B1E9842C9
:10DEF00008DB884206D8295D012903D0022901D018
:10DF0000022129559DF816108B1E984208DB884285
:10DF100006D8295D022903D0032901D005F804E0C1
:10DF20009DF817108B1E984208DB884206D8295DA1
:10DF3000032903D0042901D0042129559DF8181084
:10DF40008B1E984208DB884206D8295D042903D03D
:10DF5000052901D005212955604509DB089988422A
:10DF600006D8295D052903D0062901D006212955A7
:10DF7000032801D10AF804202146B9F81200FDF760
:10DF800015FBE8B30020324905AAD439C95D04E085
:10DF900018F800301354401CC0B28142F8D8002059
:10DFA0006623C1F1060705E002EB000C01F80C3016
:10DFB000401CC0B28742F7DC9DF819701AF80400C3
:10DFC00007F1020C604502D90C21295514E09DF897
:10DFD0001410884201D22E550EE0002153185B78B0
:10DFE000984205D2535C9B1C984201D9CB1D2B55FE
:10DFF000491CC9B20429F1D39DF81410884200E0ED
:10E0000053E008D3891C884205D8295D072902D02E
:10E0100009B1072129559DF81510884209D3891C9B
:10E02000884206D8295D072903D0082901D0082194
:10E0300029559DF81610884210D3891C88420DD8A6
:10E04000295D08290AD0092908D005E0B20000207E
:10E050002181002005090020092129559DF817106C
:10E06000884209D3891C884206D8295D092903D032
:10E070000A2901D00A2129559DF81810884209D390
:10E08000891C884206D8295D0A2903D00B2901D0B2
:10E090000B212955B84208D3604506D8285D0B28C6
:10E0A00003D00C2801D00C202855FE4F0DF11C0A7E
:10E0B000385D0AF804002146B9F81800FDF776FA31
:10E0C00078B12146B9F80E00FDF770FA48B9385D0D
:10E0D000B8B1401C3855F348002221461A38FDF7E4
:10E0E00076FA04F1030808F0FF01B9F81800FDF70B
:10E0F0005DFA70B32146B9F80E00FDF757FAD8B1B2
:10E1000027E0285D062805D92146B9F81600FDF755
:10E110004DFA70B1285D401E0628DCD22146B9F8C0
:10E120001400FDF743FA0028D5D1385D401C38555E
:10E13000D1E707203855CEE7385D072815D008B15C
:10E14000401E3855D74808F0FF0100221A38FDF765
:10E150003EFA285D0D286ED2DFE800F06D091E3A08
:10E16000586E8BA4B8D5F6EFEE003E55EAE7385D61
:10E17000401E06280BD2CB48002221461A38FDF754
:10E1800026FA385D22460121FFF791FC2EE101219C
:10E190002046FFF79BFC29E1385D811E05290BD243
:10E1A000C048002221461A38FDF711FA385D224690
:10E1B0000221FFF77CFC19E1012804D0012120464F
:10E1C000FFF784FC12E100212046FFF77FFC0DE100
:10E1D000385DC11E04290BD2B248002221461A38EC
:10E1E000FDF7F5F9385D22460321FFF760FCFDE0FD
:10E1F000022806D0012804D001212046FFF766FC42
:10E20000F4E000212046FFF761FCEFE0385D011FDC
:10E2100003290BD2A348002221461A38FDF7D7F96B
:10E22000385D22460421FFF742FCDFE00121204651
:10E23000FFF74CFCDAE0C0E0385D411F02290BD249
:10E240009848002221461A38FDF7C1F9385D224668
:10E250000521FFF72CFCC9E0401E032804D800214B
:10E260002046FFF733FCC1E001212046FFF72EFCDA
:10E27000BCE0385D062807D0401E04280DD80021D8
:10E280002046FFF723FCB1E08648002221461A38D9
:10E29000FDF79DF906203855A8E001212046FFF73B
:10E2A00015FCA3E0385D06280BD97E4800222146E4
:10E2B0001A38FDF78CF9385D22460721FFF7F7FB86
:10E2C00094E001212046FFF701FC8FE0385D07282C
:10E2D0000DD974484FF000022146A0F11A00FDF755
:10E2E00076F9385D22460821FFF7E1FB7EE005D193
:10E2F0004FF000012046FFF7E9FB77E001212046BF
:10E30000FFF7E4FB72E0385D08280DD965484FF04F
:10E3100000022146A0F11A00FDF759F9385D2246A6
:10E320000921FFF7C4FB61E009D0072807D00121CC
:10E330002046FFF7CBFB59E02EE019E004E0002176
:10E340002046FFF7C3FB51E0385D09280BD955483B
:10E35000002221461A38FDF73AF9385D22460A2193
:10E36000FFF7A5FB42E000212046FFF7AFFB3DE0B1
:10E37000385D0A280BD94B48002221461A38FDF790
:10E3800026F9385D22460B21FFF791FB2EE0002194
:10E390002046FFF79BFB29E0385D0B2808D9414850
:10E3A000002221461A38FDF712F90C2038551DE0DD
:10E3B00000212046FFF78AFB18E03A480022214658
:10E3C0001A38FDF704F9385D38B1364808F0FF0116
:10E3D00001221A38FDF7FBF808E0285D385531486E
:10E3E00008F0FF0100221A38FDF7F1F81AF80400CE
:10E3F000395D884219D02B490120093108704870D5
:10E4000088702848012221462438FDF7E0F80A20C8
:10E4100089F800000220CDE900060296002364225C
:10E4200021A1244803960AF092FB385D30BB1AF80C
:10E430000400DFF87080411EA8F10608A8F1030A65
:10E4400006291CD2DFF870B09BF8660048B10122A3
:10E450002146A8F11800FDF7BAF89BF8660008F805
:10E4600004009BF8670048B10E48012221461C3881
:10E47000FDF7ADF89BF867000AF804002AE00728CA
:10E4800028D3DFF834B09BF8660048B10548012274
:10E4900021461C38FDF79BF89BF866000AF804003B
:10E4A0000CE00000D4000020537461746553776958
:10E4B0007463680069B300084D8000209BF8670012
:10E4C00040B101222146FB48FDF781F89BF8670027
:10E4D00008F8040099F8010000280ED1A9F8186086
:10E4E000A9F81460A9F816602878072800D32E70C0
:10E4F000285D3855012089F8010009B0BDE8F08F8A
:10E500002DE9FF4F81B081464D460024DFF8A883F6
:10E51000DFF8A0B308F1D6000BF1270BA24600905C
:10E5200084B198F8CD0098F8CE1000EB012604983D
:10E5300000F00F010398052919D2DFE801F00D0F53
:10E540001113170098F8CB0098F8CC1000EB0126B7
:10E55000029801094846EEE7002508E0642506E038
:10E56000054604E0322101EB500500E04508D148A2
:10E5700008300555002739460098FDF735F8012881
:10E5800007D108EB070090F8B910032901D190F8E2
:10E590008B511CB17F1CFFB2052FECD398F8D31020
:10E5A000012902D0022904D006E0C6EB061086003D
:10E5B00002E04FF461604643642206FB05F0B0FBC5
:10E5C000F2F0BC4F80B22A3727F81400C5F164037B
:10E5D0007343B3FBF2F23B1D23F8142088B185B1DD
:10E5E0001BF80420012A0CD1A3F142020126167364
:10E5F000621CD2B2FFF722F9A7F1240006550BF8EE
:10E6000004A037F8140000B11DB9AA48801D00F815
:10E6100004A0641CE4B2022C82D305B06EE72DE99D
:10E62000F34F83B00026DFF88C92DFF890A209F157
:10E630001E094FF47A7BA04A9019029010F8B74F48
:10E64000007B072815D004987100005DC84000F0D9
:10E650000300A021984AA1EB44010191575CA1213C
:10E66000A1EB440112F8018095490978012902D0F3
:10E670000FE00398EDE7904991F8B720012A01D106
:10E6800006B9022091F8B810012902D1012E00D15B
:10E69000022030B101287DD0022804D0032801D106
:10E6A0005EE00025C1E08348824912302131005DDF
:10E6B000095D884231D217B919F80410D1B119F89F
:10E6C000041004EB4405514407EB4502114411F8D2
:10E6D000011C081A5946FCF767FF0AEB450107EBD6
:10E6E0000802114411F8011C90FBF1F55D4500D9B9
:10E6F0005D469AE004EB440508EB4501514411F8EE
:10E70000011C081A5946FCF74FFF0AEB450141442A
:10E7100011F8011C90FBF1F5E8E766492431095D29
:10E7200088421BD919F8041004EB440501EB0A02D6
:10E730006FF0060101EB4501515C401A5946FCF7A8
:10E7400033FF0AEB4501394411F8011CC1F16401A2
:10E7500090FBF1F55D4568D95D4666E0002564E013
:10E760005448544912302131005D095D884235D248
:10E77000F7B119F8041004EB4405514407EB4502C6
:10E78000114411F8011C081A5946FCF70DFF0AEB59
:10E79000450100E048E007EB0802114411F8011CB4
:10E7A00090FBF1F505F5FA755D453ED95D463CE017
:10E7B00019F8041004EB4405514408EB45021144D8
:10E7C00011F8011C081A5946FCF7EEFE0AEB450148
:10E7D000414411F8011C90FBF1F5E3E73549243180
:10E7E000095D88421ED919F8041004EB440501EBB9
:10E7F0000A026FF0060101EB4501515C401A4FF42B
:10E80000FA71FCF7D1FE0AEB4501394411F8011CFD
:10E81000C1F1640190FBF1F505F5FA755D4504D988
:10E820005D4602E0002500E05D46029890F8C300D6
:10E83000072827D004984021B140005D084000B36C
:10E840001C481C4912302131005D095D884239D2D3
:10E85000D7B119F8041004EB4405514407EB450205
:10E86000114411F8011C081A4FF4FA71FCF79CFED0
:10E870000AEB450108EB0702114411F8011C90FB5B
:10E88000F1F542E00020DAE719F8041004EB440542
:10E89000514408EB4502114411F8011C081A59466D
:10E8A000FCF782FE0AEB4501414411F8011C90FB84
:10E8B000F1F52AE0B60000204D8000200509002077
:10E8C0005D010020FE49095D88421DD919F8041038
:10E8D00004EB440501EB0A026FF0060101EB450170
:10E8E000515C401A4FF4FA71FCF75EFEF54A01994B
:10E8F000515C4FF0FF32514402EB4502895CC1F19B
:10E90000640190FBF1F500E00025EF48007838B98C
:10E91000022C05D1ED480078012823D0EC48058869
:10E920005D4500D95D46029890F87B0011280CD017
:10E93000022842D0032848D0042857D028461FF088
:10E940008FFEE44901EB86114862761CF6B2022E76
:10E95000FFF471AEDB4A0023DF4992F8C3000228BE
:10E960004DD04EE099F80000062811D8DB48018808
:10E97000DB480088091AD24812380078C0F16400D8
:10E9800048436421B0FBF1F0D649098845180EE0F0
:10E99000D2480188D2480088091AC948123800783C
:10E9A00048436421B0FBF1F0CE4909884518CD48B1
:10E9B00000888542B4D20546B2E768081FF050FED1
:10E9C000C44901EB86114862BFE705EB85000621CB
:10E9D000B0FBF1F0C8301FF043FEBE4901EB8611D9
:10E9E0004862C14A9042B0DD4A62AEE7C5F57A702E
:10E9F0001FF036FEB74901EB86114862A5E70C8887
:10EA00001CB1032803D1488808B9B248436292F880
:10EA1000C400022801D10A8822B1032804D1488801
:10EA2000002801D1AB484366F7E530B5A549062873
:10EA300013D091F87C10A34A4C1F642392F863030F
:10EA400092F86223801A0C2C32D2DFE804F009110C
:10EA50001919191919191919222691F87B10EAE7C1
:10EA6000A249B1F90010484390FBF3F000B230BD69
:10EA70009F49B1F90010484390FBF3F000B230BD5C
:10EA8000954AC91F32F91110484390FBF3F000B2C8
:10EA900030BD9848B0F9000030BD9749098809B2E7
:10EAA000891A4FF47A72514391FBF0F000B230BDF5
:10EAB000002030BD2DE9F04F8BB000250195834833
:10EAC0008F49804F02788D48002A06D097F86C2035
:10EAD000028097F86D00088005E097F871200280A9
:10EAE00097F87000088000242046FFF73DF8641C6A
:10EAF000E4B2032CF8D37248DFF8C4A13838AAF185
:10EB0000060A007A01280BD197F8A0008AF80000C5
:10EB100097F8C800C0EB00108100AAF132004184D0
:10EB2000684A9AF8000002F51C71654E02F5B07251
:10EB30000E36CDE90921DFF8CC91DFF8CCB1A6F192
:10EB40002008062828D899F80010C319C1EBC10283
:10EB500002F203129A5C3280D1B10999415C0591AD
:10EB600017F8A01F084498F8001010F80B00401A7E
:10EB70006421FCF719FD797817F8A029114411F8E0
:10EB80000B1090FBF1F0C4B2642C2ED964242CE05D
:10EB90000A99415C0591E3E799F80010C1EBC102C5
:10EBA000131897F8A120C2F106029B1A3B4493F870
:10EBB00003313380E9B3811A394491F8601105912A
:10EBC000514998F80020891F405C6421101AFCF715
:10EBD000EBFC97F8A01011F80B10C1F1640190FB49
:10EBE000F1F0C4B2642C00D964243548DFF818A1D0
:10EBF000801F0AF1060A4078062832D899F80010DA
:10EC000041B34249415C71800999415C039117F815
:10EC10009E1F084498F8011010F80A00401A642159
:10EC2000FCF7C2FC797817F89E29114411F80A10F4
:10EC300000E009E090FBF1F000F0FF0BBBF1640F86
:10EC400035D94FF0640B32E0811A394491F87012D3
:10EC50000591B5E72E49415C71800A99415C0391A9
:10EC6000D5E799F8001049B397F89F10C1F1060154
:10EC7000411A394491F82621728091F8601103916C
:10EC800098F8011010F80B00081A6421FCF78CFCAE
:10EC900097F89E1011F80A10C1F1640190FBF1F091
:10ECA00000F0FF0BBBF1640F01D94FF0640B044877
:10ECB0001549801F0C31807808912BE046E0000058
:10ECC000DA0000204D8000200A01002069000020A9
:10ECD000140100202C850020861100200E01002048
:10ECE000100100201201002000007A448E01002053
:10ECF000960000208C01002088010020BA0300202B
:10ED0000BC0300206A000020040900207381002059
:10ED10002C83002006282BD899F8001019B3FC4941
:10ED2000415CB18017F89C1F01440898085C98F872
:10ED30000210401A6421FCF737FC387879789C3F40
:10ED400001440898085CB4FBF0F02DE097F89F10A0
:10ED5000C1F10601411A394491F8DF22728091F81D
:10ED6000701203918CE7EA490E31415CB180D9E71A
:10ED700099F8001041B397F89D10C1F10601411AAE
:10ED8000394491F81213B18098F8021010F80A0073
:10ED9000081A6421FCF708FC97F89C200899515C3C
:10EDA000C1F1640190FBF1F097F8DB00DFF864A398
:10EDB000C0B30121002002AA052816DA3B1893F8F7
:10EDC000B930032B0AD019E097F89D10C1F1060164
:10EDD000411A394491F82013B180D5E7012902D0B6
:10EDE000012150540AE00021FBE73B1893F87630EC
:10EDF000112B03D1012965D001215054401C00B2D0
:10EE00000728D9DB9DF808001AF80000F0B39DF838
:10EE100009001AF80000D0B3039B5A461946584619
:10EE2000FFF76EFB0024DFF8ECB24FF0010A0BF1A4
:10EE3000070BB848005D032861D004286BD00BF89D
:10EE400004001BF80400214636F81000FCF7AEFB66
:10EE50000246B04821463238FCF7B9FB641CE4B2E4
:10EE6000072CE6D3AB48AC4E52388079C0B3A948E2
:10EE7000523890F8200001900024381990F8B90019
:10EE800001280DD002280BD0214601E01CE02FE024
:10EE900001A8FCF7A9FB1FF0E3FB06EB8411486215
:10EEA000641CE4B2052CE8D301210020DFF864B231
:10EEB000ABF1380B052860D23A1892F8B920032A32
:10EEC00048D068E0002198E79DF809001AF8000092
:10EED00038B15A462046039B0599FFF711FBA1E77D
:10EEE00025E0059B224619462046FFF709FB99E7D6
:10EEF00022465846059B0399FFF702FB92E798F8D4
:10EF0000000098F80110884202D20BF8045098E7EC
:10EF10000BF804A095E798F8000098F801108842D3
:10EF200002D90BF804508CE70BF804A089E7002401
:10EF300078485238B0F820B02BFA04F000F0010005
:10EF40001FF08EFB06EB84114862641CE4B2052CB2
:10EF5000F2D3A9E7012908D001211BF80120012AD9
:10EF600005D006EB8012556215E00021F5E706EBAF
:10EF700080134FF07E525A620DE03A1892F87620D4
:10EF8000112A08D1C9B100211BF80120012A16D08D
:10EF900006EB80125562401CC0B207288AD30024B9
:10EFA00004F1B700079002F0ECF803280DD00798A1
:10EFB00002F0E7F8042816D022E00121E4E706EB8E
:10EFC00080134FF07E525A62E5E798F8000098F8F7
:10EFD0000110884203D2381980F8B75010E0381970
:10EFE00080F8B7A00CE098F8000098F8011088426B
:10EFF00003D9381980F8B75002E0381980F8B7A063
:10F00000641CE4B2022CCBD34248DFF808A152388A
:10F01000AAF1060A407980B1062829D0AAF11A027D
:10F020001178062953D899F80000E0B33B48085CF2
:10F030008DF8100004F00F0058E0BAF800003230EC
:10F0400000B2AAF800004FF47A71884201DDAAF8F4
:10F050000050BAF80200323800B2AAF802000028C4
:10F0600001DAAAF802104FF4FA700AF005FC17E171
:10F0700097F8A602042817D0AAF8005097F8A7021C
:10F08000042817D0AAF80250BAF900104FF47A7089
:10F09000814201DDAAF80000BAF90210814201DDC7
:10F0A000AAF80200FCE00BE00620FFF7BEFCAAF87D
:10F0B0000000E3E70720FFF7B8FCAAF80200E3E747
:10F0C00016480E30085C8DF8100020090EE099F803
:10F0D0000000E0B197F8A100C0F10600081A38441A
:10F0E00090F82D018DF8100004F00F0097F89F3074
:10F0F0005178C3F10603CB1A062922D899F80030BB
:10F10000D3B1064BDB1DC95C8DF8111021E007E07F
:10F110005F830020F40000202C8500207A810020ED
:10F12000200997F8A130C3F10603C91A394491F8B0
:10F130003B118DF81010D9E7B34BC95C8DF8111055
:10F1400007E099F8001081B1D91991F834118DF8C0
:10F1500011109178062914D899F800205AB1AA4ABA
:10F160002032895C8DF8121018E0D91991F8E61256
:10F170008DF81110EDE7A44A3332895C8DF8121036
:10F180000CE099F80020EAB197F89D20C2F1060240
:10F19000891A394491F806138DF8121004A9FFF763
:10F1A0003EFA9A4805210690FCF71EFAA8B197F896
:10F1B000670397F86813000200B208441FF038FA9A
:10F1C000F0610CE097F89D20C2F10602891A3944DB
:10F1D00091F819138DF81210E0E78D48F0610621BF
:10F1E0000698FCF701FA50B197F8690397F86A138B
:10F1F000000200B208441FF01BFAF06501E08448E9
:10F20000F065844CA07901284AD197F8B70004A989
:10F210004FF06409095CC1F3011149B101292CD0F7
:10F2200004F13503DA1C022904D0032927D114E0A4
:10F23000E58324E018F80010125C914203D9881A83
:10F240004000E0831BE0185C814204D2C1F132002F
:10F250004000E08313E0E58311E018F80010125C31
:10F26000914201D9E1830AE0185C814203D2C1F1E5
:10F270006400E08303E0E58301E0A4F81E90072129
:10F280000698FCF7B1F908B1607BE083B4F91E0081
:10F29000052801DAE58303E05F2801DDA4F81E906C
:10F2A0000024DFF87481381990F8BE00012802D1DB
:10F2B0005A49097861B1022802D1B8F8001039B171
:10F2C000032802D1B8F8021011B1042804D006E0D6
:10F2D00006EB841045622DE097F8DB1011B105288C
:10F2E0000AD00CE09BF80000012823D106EB841122
:10F2F0004FF07E5048621DE097F8DB1011B10628F0
:10F300000DD017E021464648FCF76EF99BF8001037
:10F3100008401FF0A5F906EB841148620AE097F84F
:10F32000DB00022806D13B48807A012802D106EB97
:10F3300084104562641CE4B2052CB4D30020354A25
:10F340004FF07E51537A3C1894F8DC40022C04D1E3
:10F35000012B19D006EB80146562401CC0B2052851
:10F36000F1D30024507900281AD0294D002006EB53
:10F37000841151F82020AA420AD051F820001FF031
:10F380001BF92AF8140007E006EB80146162E4E739
:10F39000401CC0B21028ECD3641CE4B2002CE5D0B1
:10F3A0000BB0BDE8F08F1B4832300078011F0229F6
:10F3B00002D80A30C0B27047C11F022902D8C01E4D
:10F3C000C0B27047A0F10A010229FAD8C01DC0B22C
:10F3D000704770B50F4E0021308AFCF7E7F80446FD
:10F3E0000A4DD63D95F8A10000B900240021708A8D
:10F3F000FCF7DCF828B1A41CE4B295F8A00000B931
:10F400000024204670BD00003383002023810020AB
:10F4100000007F43A2000020861100206900002028
:10F42000180200200D49086070470C494860704779
:10F430000A498860704709494AF6AA20086070475F
:10F4400006494CF6CC400860704701460020034A4C
:10F45000D2680A4200D0012070470000003000400E
:10F46000B448016841F0010101604168B24A1140AD
:10F4700041600168B14A11400160016821F48021B6
:10F480000160416821F4FE0141604FF41F01816079
:10F490007047A8490A6822F480320A600A6822F498
:10F4A00080220A60B0F5803F07D0B0F5802F03D1ED
:10F4B000086840F4A02008607047086840F4803075
:10F4C000086070470346002059099A4A01290AD06A
:10F4D00002290AD0516A03F01F02012393400B4214
:10F4E00000D0012070471168F5E7116AF3E718B5FD
:10F4F000002000904FF4A0643120FFF7E3FF009953
:10F50000491C00910099A14201D00028F4D031207B
:10F51000FFF7D8FF08B1012018BD002018BD854AAB
:10F52000116821F0F80141EAC00010607047844979
:10F53000086070477F4B5A6822F47C1208431043DE
:10F54000586070477E49086670477A4A516821F0D2
:10F5500003010143516070477648406800F00C0099
:10F560007047744A516821F0F001014351607047BF
:10F57000704A516821F4E0610143516070476D4A5F
:10F58000516821F4605141EAC00050607047694AF7
:10F59000002903D0517A014351727047517A814357
:10F5A000517270476649D83108607047614A5168A6
:10F5B00021F440410143516070475E4900222031EF
:10F5C0000A7001F82029012805D0042802D105205D
:10F5D00081F820007047012081F8200070475949C8
:10F5E0000860704753490A6A02430A6270475549E6
:10F5F00044390860704710B54E4A516801F00C015B
:10F60000514B002927D0042927D0082927D003608F
:10F61000516801F0F00109094C4B5C5C0168E14064
:10F620004160546804F4E064240A1C5D21FA04F487
:10F630008460546804F46054E40A1B5DD940C160DE
:10F64000526802F44042920B404B1B1F9A5CB1FB84
:10F65000F2F1016110BD0360DAE70360D8E7516899
:10F6600001F47011536803F48033022404EB9141D8
:10F6700033B153689B0307D5354B59430160C7E746
:10F68000334B59430160C3E72F4B59430160BFE738
:10F69000284A002903D051690143516170475169DB
:10F6A000814351617047234A002903D09169014386
:10F6B0009161704791698143916170471D4A0029AA
:10F6C00003D0D1690143D1617047D1698143D161D0
:10F6D0007047184A002903D0D1680143D1607047B0
:10F6E000D1688143D1607047124A002903D0116963
:10F6F00001431161704711698143116170471149DC
:10F700004039086070470E49C86470470949C8719C
:10F7100070470848416A41F0807141627047014674
:10F720000020044A92680A4200D001207047014933
:10F7300088727047001002400000FFF8FFFFF6FEDD
:10F74000000042428004424200127A00260100205A
:10F7500000093D004D4A002903D011880143118062
:10F76000704711888143118070474848001D018807
:10F7700041F01001018070474448001D018821F0CC
:10F7800010010180704741481C3000883F49183102
:10F79000098840EA0140704700B50246FFF7E5FFDF
:10F7A0003A49100C18310880081D02805DF804EBFE
:10F7B000E2E700B50246FFF7D8FF3449C2F3034041
:10F7C00008310880081D02805DF804EBD4E700B51D
:10F7D0000246FFF7CAFF2D49100C20310880081D92
:10F7E00002805DF804EBC7E7284810300088000766
:10F7F000010B2648143000880843704770B5002478
:10F80000224D2D1D06E0641CE4B264200AF034F899
:10F810001E2C02D828888006F5D570BD70B500244E
:10F820001A4D2D1D288820F00800288006E0641C51
:10F83000E4B264200AF020F81E2C02D828880007C1
:10F84000F5D570BD01460020104A121D12880A42EB
:10F8500000D0012070470D49091D0A8882430A80A3
:10F8600070470A49091D0988C2B21140074A128827
:10F87000024202D009B101207047002070470349BD
:10F88000091D0A8882430A80704700000028004052
:10F8900010B5FE4988420AD1C41401212046FFF761
:10F8A00018FF2046BDE810400021FFF712BFB0F15D
:10F8B000804F0CD0F649884213D101210220FFF776
:10F8C00013FF0021BDE810400220FFF70DBF01210A
:10F8D0000846FFF709FF0021BDE810400120FFF7AF
:10F8E00003BFEC49884209D101210420FFF7FCFE47
:10F8F0000021BDE810400420FFF7F6BEE64988422B
:10F9000009D101210820FFF7EFFE0021BDE81040DA
:10F910000820FFF7E9BEE149884209D10121102002
:10F92000FFF7E2FE0021BDE810401020FFF7DCBE2B
:10F93000DB49884209D101212020FFF7D5FE0021B3
:10F94000BDE810402020FFF7CFBED64988420AD13B
:10F95000441401212046FFF7BCFE2046BDE81040BC
:10F960000021FFF7B6BED04988420AD10121CC045C
:10F970002046FFF7AEFE2046BDE810400021FFF70D
:10F98000A8BECA4988420AD101210C052046FFF7CA
:10F99000A0FE2046BDE810400021FFF79ABEC449F2
:10F9A00088420AD101214C052046FFF792FE2046ED
:10F9B000BDE810400021FFF78CBEBE49884209D146
:10F9C00001214020FFF790FE0021BDE810404020BB
:10F9D000FFF78ABEB849884209D101218020FFF78C
:10F9E00083FE0021BDE810408020FFF77DBEB349B3
:10F9F00088420AD1841501212046FFF775FE204672
:10FA0000BDE810400021FFF76FBEAD4988420AD122
:10FA100001210C042046FFF75CFE2046BDE81040A3
:10FA20000021FFF756BEA74988420AD101214C04A4
:10FA30002046FFF74EFE2046BDE810400021FFF7AC
:10FA400048BEA14988420AD101218C042046FFF713
:10FA500040FE2046BDE810400021FFF73ABE10BD31
:10FA600030B50288894C8F4DA0420DD0A8420BD0F2
:10FA7000B0F1804F08D0864B984205D0854B984214
:10FA800002D0854B984203D122F070034A881A4372
:10FA9000824B984206D0824B984203D022F44073A6
:10FAA000CA881A4302808A8882850A880285A04211
:10FAB0000AD0A84208D0824A904205D0814A90429A
:10FAC00002D0814A904201D1097A018601218182C6
:10FAD00030BD30B5028C22F001020284028C838892
:10FAE000048B24F0700424F003050C882C4322F0CE
:10FAF00002020D8915434A882A43644DA8420BD05F
:10FB0000684DA84208D06E4DA84205D06D4DA84260
:10FB100002D06D4DA8420FD122F008054A892A4330
:10FB200022F004058A882A4323F4807323F40073A7
:10FB30008D891D43CB892B4383800483C9888186AB
:10FB4000028430BD70B5028C22F010020284028C57
:10FB50008388048B24F4E04424F440760D884FF627
:10FB6000FF7404EA0525354322F020020E8904EAD9
:10FB7000061616434A8804EA02123243434EB04244
:10FB800002D0484EB04217D122F080024E8904EADA
:10FB90000616164326F040068A8804EA021232430B
:10FBA00023F4806323F400638E8904EA86061E43EF
:10FBB000CB8904EA8303334383800583C9880187A3
:10FBC000028470BD70B5028C22F480720284028CB3
:10FBD0008388848B24F0700424F003040D8825436B
:10FBE00022F400720E894FF6FF7404EA06261643CB
:10FBF0004A8804EA02223243244EB04202D0294EFF
:10FC0000B04217D122F400664A8904EA0222324344
:10FC100022F480668A8804EA0222324323F4805365
:10FC200023F400538E8904EA06161E43CB8904EAA6
:10FC30000313334383808583C9888187028470BD21
:10FC400070B5028C22F480520284058C8288838BEA
:10FC500023F4E04323F440760C884FF6FF7303EA65
:10FC60000424344325F400550E8903EA06362E4356
:10FC70004D8803EA05353543044EB04202D0094EA3
:10FC8000B04226D122F480468A891FE0002C014030
:10FC90000004004000080040000C0040001000403C
:10FCA0000014004000340140004C0140005001406D
:10FCB0000054014000180040001C0040002000409B
:10FCC00000400140004401400048014003EA821224
:10FCD000324382808483C988A0F84010058470BDB7
:10FCE000828B22F440628283828B4FF6FF7303EA99
:10FCF00001210A4382837047F0B5048C24F48054B8
:10FD00000484868B048C4FF6FF7505EA013726F4D0
:10FD1000734605EA0222324305EA03331343F74AE6
:10FD200090420ED0F64A90420BD0B0F1804F08D0EE
:10FD3000F44A904205D0F44A904202D0F34A9042ED
:10FD400005D124F40051394341F4805104E024F4F6
:10FD500002420A4342F4805183830184F0BD828BC6
:10FD600022F00C028283828B0A4382837047F0B5B3
:10FD7000048C24F480740484858B048C4FF6FF7704
:10FD800007EA012625F0F30507EA031313432B4383
:10FD9000DA4A90420ED0DA4A90420BD0B0F1804F4E
:10FDA00008D0D84A904205D0D74A904202D0D74ACC
:10FDB000904205D124F40071314341F4807104E094
:10FDC00024F420620A4342F4807183830184F0BDED
:10FDD000028B22F440620283028B4FF6FF7303EA28
:10FDE00001210A4302837047F0B5048C24F010040B
:10FDF0000484068B048C4FF6FF7505EA011726F480
:10FE0000734605EA0333334305EA02221A43BB4B28
:10FE100098420ED0BA4B98420BD0B0F1804F08D028
:10FE2000B84B984205D0B84B984202D0B74B984295
:10FE300005D124F02001394341F0100104E024F001
:10FE4000A0030B4343F0100102830184F0BD028B39
:10FE500022F00C020283028B0A430283704770B5C2
:10FE6000048C24F001040484058B048C25F0F30534
:10FE70004FF6FF7606EA031313432B439F4A904243
:10FE80000ED09F4A90420BD0B0F1804F08D09D4ACF
:10FE9000904205D09C4A904202D09C4A904205D1A3
:10FEA00024F002020A4342F0010104E024F00A02B5
:10FEB0000A4342F001010383018470BD70B5054619
:10FEC0000C468E48854209D08D48854206D0B5F152
:10FED000804F03D08B48854200D08B4820886188B2
:10FEE000A288238958B1042811D0082817D02846A1
:10FEF000FFF702FFE1882846BDE87040F0E628469B
:10FF0000FFF7ADFFE1882846BDE870409FE728462F
:10FF1000FFF76AFFE1882846BDE8704058E72846A9
:10FF2000FFF725FFE1882846BDE8704017E72DE977
:10FF3000F04107460C46002501266188002900D1C2
:10FF40000225A288012A00D102262088238988B1AF
:10FF50003846FFF749FFE1883846FFF739FF238924
:10FF6000324629463846FFF77AFFE1883846BDE831
:10FF7000F0416CE73846FFF772FFE1883846FFF73B
:10FF800066FF2389324629463846FFF72DFFE18870
:10FF90003846BDE8F0411BE710B50A884B88CC888D
:10FFA0001A438B8823431A430B891A434B89898947
:10FFB0001A430A43A0F8442010BD4FF6FF71818018
:10FFC00000210180C18041800172704700210180C1
:10FFD00041808180C180018141818181C1817047DF
:10FFE00000210180418001228280C180018170470F
:10FFF0000021018041808180C18001814181818116
:020000040801F1
:100000007047002904D0018841F001010180704748
:10001000018821F0010101807047002905D030F8E6
:10002000441F41F400410180704730F8441FC1F380
:100030000E0101807047002A03D082890A43828121
:10004000704782898A438281704781827047114359
:10005000A0F848107047002A03D082890A438281A1
:10006000704782898A4382817047018921F00701A4
:1000700001817047028922F070020A4302817047B1
:1000800000B503461846FFF7F5FF188940F0070052
:10009000188100BD70B50D4604461146602D0CD088
:1000A00001222046FFF7DBFE29462046FFF7E2FF4C
:1000B000208940F00700208170BD01222046FFF713
:1000C00093FEF1E730B50489E4B24FF6FF7505EA17
:1000D000032313430B432343038130BD10B5044670
:1000E0002046FFF7EFFF208920F0070040F00700CF
:1000F00020F0700040F07000208110BD002C014005
:10010000003401400004004000080040000C0040A2
:1001100010B504462046FFF7D5FF208940F4804003
:100120002081EAE7018582827047028822F070020E
:100130000A430280704770B50589048B068C25F050
:1001400007050D434FF6FC410C4040F201110C43F2
:1001500026F022064FF6FF7101EA031111433143E5
:1001600005810483018470BD028B22F070020A4372
:1001700002837047028B22F4E0424FF6FF7303EADA
:100180000121114301837047828B22F070020A43E0
:1001900082837047828B22F4E0424FF6FF7303EABA
:1001A0000121114381837047002904D0018841F067
:1001B000800101807047018821F080010180704733
:1001C000002904D0818841F0040181807047818832
:1001D00021F0040181807047002904D0818841F01A
:1001E000080181807047818821F008018180704773
:1001F000002904D0818841F0010181807047818805
:1002000021F0010181807047028B22F008020A432D
:1002100002837047028B22F400624FF6FF7303EAF9
:100220000121114301837047828B22F008020A43A7
:1002300082837047828B22F400624FF6FF7303EAD9
:100240000121114381837047028B22F004020A438B
:1002500002837047028B22F480624FF6FF7303EA39
:100260000121114301837047828B22F004020A436B
:1002700082837047828B22F480624FF6FF7303EA19
:100280000121114381837047028B22F080020A43CF
:1002900002837047028BC2F30E024FF6FF7303EA2C
:1002A0000121114301837047828B22F080020A43AF
:1002B00082837047828BC2F30E024FF6FF7303EA0C
:1002C0000121114381837047028C22F002020A430C
:1002D00002847047028C22F008020A4302847047AD
:1002E000028C22F020024FF6FF7303EA0111114342
:1002F00001847047028C22F080024FF6FF7303EAFC
:100300000111114301847047028C22F400724FF6F0
:10031000FF7303EA0121114301847047028C22F428
:1003200000624FF6FF7303EA012111430184704715
:10033000028C22F400524FF6FF7303EA013111439D
:100340000184704710B501238B40048C9C430484C6
:10035000038C8A4013430384CFE610B504238B40FB
:10036000048C9C430484038C8A4013430384C4E6B6
:1003700030B500F1180301248C40058CA543058499
:10038000002911D008290FD0091FC1F34E001844CD
:10039000016821F4E041016001684FF6FF7303EA50
:1003A00002221143016030BD03EB5100016821F0CE
:1003B0007001016001681143016030BD002904D063
:1003C000018841F0020101807047018821F002019B
:1003D00001807047002904D0018841F004010180A8
:1003E0007047018821F0040101807047002904D082
:1003F000818841F0800181807047818821F08001EF
:1004000081807047028822F00802028002880A4335
:1004100002807047828822F07002828082880A43BC
:1004200082807047028922F00702028102890A4312
:1004300002817047028922F08002028102890A4308
:10044000028170478184704781857047818670473B
:100450000187704781877047A0F840107047028875
:1004600022F44072028002880A4302807047808E24
:100470007047008F7047808F7047B0F8400070471A
:10048000808C7047008D704702460020128A0A4215
:1004900000D001207047C943018270470246002006
:1004A000138A0B4092890A40002B02D0002A00D008
:1004B00001207047C94301827047000010B5E1492F
:1004C00088420AD101218C032046FFF702F9204619
:1004D000BDE810400021FFF7FCB8DB4988420AD193
:1004E00001214C042046FFF7FFF82046BDE81040EC
:1004F0000021FFF7F9B8D54988420AD101218C04BF
:100500002046FFF7F1F82046BDE810400021FFF734
:10051000EBB8CF4988420AD10121CC042046FFF72D
:10052000E3F82046BDE810400021FFF7DDB8C949D7
:1005300088420AD101210C052046FFF7D5F8204654
:10054000BDE810400021FFF7CFB810BD30B585B031
:1005500004460D46208A4CF6FF710840E9880143A5
:100560002182A0894EF6F3110840A9882A891143F7
:100570006A8902431143A181A08A4FF6FF410840D6
:10058000A9890143A1826846FFF735F8AD48844246
:1005900001D1039800E00298A189090408D500EB75
:1005A000C00101EB001029684900B0FBF1F007E041
:1005B00000EBC00101EB001029688900B0FBF1F0ED
:1005C0006422B0FBF2F109010B096FF018056B43CF
:1005D00000EB8300A3891D044FF0320307D503EB22
:1005E000C000B0FBF2F000F00700084306E003EBA8
:1005F0000010B0FBF2F000F00F000843208105B0BE
:1006000030BD4FF41651016000218180C18001810D
:100610000C2242818181704710B5038A4FF2FF029C
:1006200013400A884C8822438C88C9880C43224393
:100630001A43028210BD0021018041808180C18067
:100640007047002904D0818941F4005181817047AD
:10065000818921F400518181704710B540F66A13F9
:10066000C1F3421301F01F040121A140012B07D067
:10067000022B07D014303AB102680A43026010BD61
:100680000C30F8E71030F6E702688A43026010BDCC
:10069000002A03D0828A0A4382827047828A8A4370
:1006A00082827047028A22F00F020282028A0A4383
:1006B00002827047828922F40062828182890A4321
:1006C00082817047002904D0818941F00201818133
:1006D0007047818921F0020181817047028A22F0EE
:1006E00020020282028A0A4302827047002904D053
:1006F000018A41F4804101827047018A21F48041DE
:1007000001827047C1F30801818070478088C0F37F
:1007100008007047818941F0010181817047028B97
:10072000D2B20283028B42EA012101837047028B1D
:1007300002F47F420283028B0A430283704700293E
:1007400004D0818A41F0200181827047818A21F0A2
:10075000200181827047002904D0818A41F0100174
:1007600081827047818A21F01001818270470029BF
:1007700004D0818A41F0080181827047818A21F08A
:10078000080181827047002904D0818941F4004129
:10079000818170478189C1F30E01818170470029F1
:1007A00004D0818A41F4006181827047818A21F4FA
:1007B000006181827047828A22F004028282828AEA
:1007C0000A4382827047002904D0818A41F00201E5
:1007D00081827047818A21F002018182704702463E
:1007E000002012880A4200D0012070478A05C943C0
:1007F0000180704770B5002440F66A12C1F34213BD
:1008000001F01F05012606FA05F2012B0CD0022B80
:100810000DD0838A1340090A8E40008830400BB106
:1008200000B10124204670BD83891340F3E7038A99
:100830001340F0E740F66A120A0A01219140C943C9
:1008400001807047003801400044004000480040EB
:10085000004C00400050004010B50120FEF74FFF53
:10086000BDE810400020FEF74ABF204908607047ED
:100870001E49091F086070471C4984310860704791
:100880001B4A118821F46071014311807047184A96
:10089000118821F07F0101431180704708B5144A87
:1008A0002C3A104400900098016008BD08B510492A
:1008B0002C39084400900098008808BD0B489C30F3
:1008C0000068C0B270470A480830018841F0010151
:1008D000018070470548A0300068C0B270470448E6
:1008E0000830018841F002010180704704860D4202
:1008F0002C6C004010B501210C072046FEF7F4FED9
:100900002046BDE810400021FEF7EEBE21490862F6
:1009100070472049086170471F4A116821F0E001C3
:100920000143116070471B49A031086070471A4BA2
:100930001A6822F0030202431A601848026842F063
:1009400004020260012905D020BF016821F00401E2
:100950000160704730BFF8E70F48016841F00401BB
:100960000160016841F0020101600C48016841F03A
:100970000401016030BF704701460020064A5268FA
:100980000A4200D00120704703490A6842EA800009
:100990000860704700000E420070004010ED00E05B
:1009A0000948804709480047FEE7FEE7FEE7FEE703
:1009B000FEE7FEE7FEE7FEE7FEE7FEE7044805493F
:1009C000054A064B70470000DD83000831810008AE
:1009D00098D8002098DE002098DA002098DA0020CD
:1009E0007FB5B14CA088ADF80C0048258DF80F50AC
:1009F00002268DF80E6003A92068F8F70EFA208A07
:100A0000ADF808008DF80B508DF80A6002A9E06877
:100A1000F8F703FAA08BADF804008DF807508DF8B5
:100A2000066001A9A069F8F7F8F9208DADF800007B
:100A30008DF803508DF802606946606AF8F7EDF9A9
:100A40007FBD70B5984D583DB5F85C10A86DF8F7AE
:100A50003FFA964C18B3207820F004002070B5F8C7
:100A60006810686EF8F734FAF0B1207820F00200D0
:100A70002070B5F87410286FF8F72AFAC8B12078FA
:100A800020F001002070B5F88010E86FF8F720FA28
:100A9000A0B1207820F008002070207870BD207868
:100AA00040F004002070DAE7207840F00200207067
:100AB000DFE7207840F001002070E4E7207840F084
:100AC00008002070E9E72DE9F047012008F0B4FEA6
:100AD000FFF7B7FF0446754EDFF8D481093E4FF0AB
:100AE000000770794FF0010534EA000015D098F83E
:100AF0007F00032811D0F5706E48077098F8ED005C
:100B00006D49C0EB00104FF6FF7202EA80000880CA
:100B100018B101216948F8F7EFF9F078684B01281E
:100B200076D1717931EA040072D098F87A000228FF
:100B30006ED0F77063480570634A64201070B1711D
:100B400062480770187801280FD072784FF00D0CAA
:100B500005204FF00E0962B3012951D002293DD082
:100B6000042960D0082976D169E03079172801D0AE
:100B7000182803D108290AD0042908D001290DD04A
:100B8000022908D004290CD008290FD10CE0192023
:100B9000B07237715FE01820B07207E01720B072B2
:100BA00004E01620B07201E01520B072B07A307106
:100BB00051E001294FD002294DD0042902D0082943
:100BC00049D105E086F80AC07570B570307042E012
:100BD00086F80A907570B57030703CE0B278012AE2
:100BE00004D0022A05D0032A06D007E00A22B272F6
:100BF00004E01122B27201E01222B27230702AE0D7
:100C0000B278012A05D0022A06D0032A07D008E0CC
:100C100032E00922B27204E00F22B27201E0102227
:100C2000B272307017E086F80AC07570B278032A85
:100C300002D2521CB27000E0B57030700BE086F842
:100C40000A907570B278012A02D9521EB27001E082
:100C50000322B2703070042908D0082906D0022976
:100C600004D0012902D098F8790028B918480770F3
:100C7000F571B5811748077074710C2C11D1187873
:100C800078B998F87F0001280BD0032809D0307A72
:100C9000411C31721E2802D91320B0721D70BDE8AC
:100CA000F0873772FBE7000008F002083F010020E0
:100CB0004D800020840000206C00002000080140CE
:100CC0008C000020860000209D0000209E00002057
:100CD000900000209F00002038B5BB4C208FADF85D
:100CE000000048208DF803006946606BF8F795F81E
:100CF000218F606BF8F700F938BD38B5B24C208F02
:100D0000ADF8000010208DF8030003208DF80200DC
:100D10006946606BF8F781F8218F606BF8F7ECF8A3
:100D200038BD08B50820ADF8000010208DF803008C
:100D300003208DF802006946A448F8F76EF808BD54
:100D400008B50820ADF8000048208DF8030069467A
:100D50009E48F8F762F808BD9B4A002803D0918DA1
:100D6000906AF8F7C9B8918D906AF8F7C7B8964AB3
:100D7000002803D0118F506BF8F7BEB8118F506B5D
:100D8000F8F7BCB89048018F406BF8F7A1B88E48CF
:100D9000818D806AF8F79CB8F8B58B4C0121606AA8
:100DA000FEF781FCA08DADF8000010258DF80350F2
:100DB00003268DF802606946A06AF8F72EF8A18D27
:100DC000A06AF8F799F80121206BFEF76CFC208FE0
:100DD000ADF800008DF803508DF802606946606B35
:100DE000F8F71BF8218F606BF8F786F8F8BDF8B5B7
:100DF00001210820FEF757FC4FF48065ADF8005044
:100E000010268DF8036003248DF80240704F694668
:100E10003846F8F702F829463846F8F76DF8012108
:100E20000820FEF740FC6D00ADF800508DF803601F
:100E30008DF8024069463846F7F7EFFF29463846F5
:100E4000F8F75AF8F8BD10B5FFF757FF0120FFF784
:100E50008EFF0120FFF780FF042008F0EDFC00204A
:100E6000FFF785FF042008F0E7FCBDE810400020F4
:100E700072E710B5FFF741FF0020FFF76DFF00207C
:100E8000FFF775FF042008F0D7FC0120FFF764FF8F
:100E90000120FFF76CFFBDE81040042008F0CCBC37
:100EA00010B500240120FFF762FFFFF715FF0120B6
:100EB00008F0C2FC0120FFF74FFF012008F0BCFC46
:100EC00007E0641CA4B2FA2C03D9FFF7D2FF01207B
:100ED00010BDFFF757FF0028F3D1FFF73DFF0020BB
:100EE00010BD10B50020FFF737FFFFF706FF002009
:100EF000FFF73DFF022008F09FFC0120FFF72CFFC9
:100F0000022008F099FCBDE81040002024E710B54D
:100F10000020FFF721FFFFF7F0FE0120FFF727FF7A
:100F2000022008F089FC0120FFF716FF022008F0DC
:100F300083FCBDE8104000200EE770B50546FFF7C2
:100F4000DCFE0020FFF708FF0024E809FFF70FFF91
:100F50006806050E022008F06FFC0120FFF7FCFE7A
:100F6000022008F069FC0020FFF7F6FE022008F0DE
:100F700063FC641CE4B2082CE7D370BD70B5064670
:100F80000024FFF7A9FE00250020FFF7E5FE022060
:100F900008F052FC0120FFF7DFFE6006040EFFF7A9
:100FA000F1FE08B1641CE4B2012008F045FC6D1CA0
:100FB000EDB2082DE8D31EB1FFF793FF204670BDB8
:100FC000FFF7A5FFFAE70000B0EF020800080140B4
:100FD000000C014038B5704CE06B002815D054F877
:100FE0003C0F0121FEF75FFB2089ADF800001020C7
:100FF0008DF8030003208DF8020069466068F7F75A
:101000000CFF21896068F7F777FF38BD624AD16B22
:1010100000290AD020B1B2F84410106CF7F76CBF69
:10102000B2F84410106CF7F769BF704710B5FFF7BE
:10103000B3FEBDE81040CDE710B50446FFF703FF4F
:10104000200AA02101EB4000C0B2FFF776FFFFF7B6
:1010500027FFE0B2FFF771FFFFF722FFFFF7F3FE74
:10106000A120FFF76AFFFFF71BFF0020FFF786FFB5
:101070000446FFF7FEFE204610BD70B504460D463F
:101080000020FFF7C3FFFFF7DEFE200AA02101EBDF
:101090004000C0B2FFF751FFFFF702FFE0B2FFF7D9
:1010A0004CFFFFF7FDFE2846FFF747FFFFF7F8FE6E
:1010B000FFF7DFFE0120FFF7A9FFBDE87040052024
:1010C00008F0DABB2DE9F04106460D46174600242C
:1010D00009E0E00025FA00F0C1B2301980B2FFF754
:1010E000CCFF641CE4B2BC42F3D3BDE8F0812DE92F
:1010F000F04102460E4600200024971908E0050240
:10110000381B401E80B2FFF797FF2844641CE4B2EE
:10111000B442F4D3E9E710B5FF20FFF78DFF55285F
:101120000AD05521FF20FFF7A8FFFF20FFF784FF1B
:10113000552803D0012010BD002010BD002010BD97
:1011400070B504460E46154608E02046641CA4B25D
:10115000FFF772FF06F8010B6D1EADB2002DF4D142
:1011600070BD70B506460D46144606E02978304637
:10117000FFF783FF761CB6B26D1C641EA4B2F5D2D5
:1011800070BD59E7054A1278012A03D0B72802D06A
:10119000B82800D071E77047B0EF02084401002082
:1011A000704730B56423B0FBF3F4E4B2B0FBF3F561
:1011B00003FB1500132C01D96430C0B200EB90037F
:1011C0000724B3FBF4F504FB1533A44D1A440D4476
:1011D00015F8015C2A4492B2800703D1032901D299
:1011E000521E92B2B2FBF4F004FB102030BD810716
:1011F00001D0002070476421B0FBF1F201FB120125
:1012000009B1012070474FF4C871B0FBF1F201FB46
:10121000120008B100207047012070472DE9F04707
:10122000FEF7B1FA06468E4FB6FBF7F38D488E4DAA
:101230000188994233D0038040F2B2744FF4B778FA
:101240004FF4B6790FE02046FFF7D1FF38B14345A0
:1012500002D3A3F5B77304E0641CA4B205E0A3F2C3
:101260006D13641CA4B24B45EDD8AC800024DFF8AC
:10127000EC8108F10C080CE0A888FFF7B8FF08B172
:10128000012C2FD018F80400984204D81B1A641CB3
:10129000A4B21C2BF0D2641CAC715B1CEB71B6FBCE
:1012A000F7F007FB10604FF46161B0FBF1F22A70B8
:1012B000B0FBF1F201FB12033C22B3FBF2F36B70C3
:1012C000B0FBF1F301FB1300B0FBF2F102FB1100E4
:1012D000A870EA79A979A888FFF763FF287200202F
:1012E000BDE8F0871D2BD6D31D3BD0E770B5002499
:1012F0000420FFF7DBFA45F25005A8423FD0012158
:101300004FF0C050FEF7DAF90120FFF7FFFAFFF7C0
:10131000A3FA0120FEF751F908E0641CE4B20A20A8
:1013200008F0AAFAC82C01D3012070BD4120FEF7B5
:10133000C9F80028F1D0FA2C01D3012070BD4FF478
:101340008070FEF74FF90120FEF751F9FEF756FACB
:10135000FEF764FA01210846FEF7FCF9FEF74EFAA3
:10136000FEF703FA47F6FF70FEF723FAFEF746FA98
:10137000FEF702FA29460420FFF790FA07E0FEF78D
:101380004DFA01210846FEF7E5F9FEF737FAFFF7B7
:1013900007FFFFF743FF002070BD2DE9F05F064611
:1013A000DDF828A0894690460024A6F2B270822873
:1013B00002D30120BDE8F09F40F2B2752B4FDFF859
:1013C000B0B008E02846FFF712FF08B13C4400E047
:1013D0005C446D1CADB2B542F4D3A9F1010909F02A
:1013E000FF070025DFF87490DFF874B009F10C09ED
:1013F0000FE019F8050040F2A321484304EBC014A4
:101400003046FFF7F4FE10B1012D00D15C446D1C95
:10141000ADB2BD42EDD3A8F1010840F2A32008FB14
:1014200000F804EBC810C3EB4311C1EB032100EB40
:101430000110CAEB0A1100EB81000B99441801213D
:101440004FF0C050FEF73AF90120FFF75FFA20464F
:10145000FEF7A2F9FEF7D2F90020ABE796EF0208FB
:101460008051010046010020181100200085E20192
:101470008033E10170B5FA4B0024C3F88041F94A8A
:101480000125127A042A02D3F74A156001E0C3F855
:1014900088510022C3F88441060602D5C3F88C5156
:1014A00001E0C3F88C41C3F884514006000E521C81
:1014B000D2B2082AEED30020C3F884410A0602D52E
:1014C000C3F88C5101E0C3F88C41C3F8845149063C
:1014D000090E401CC0B20828EED3C3F8805170BD7D
:1014E000C0F30722C1B21046C4E730B5DC4A00237E
:1014F000C2F88031DB49097A042902D3DA490B604A
:1015000001E0C2F8883100210124C2F884310506C7
:1015100002D5C2F88C4101E0C2F88C31C2F8844196
:101520004006000E491CC9B20829EED3C2F880411A
:1015300030BD30B5CA4A0024C2F88041C9490123F0
:10154000097A042902D3C8490B6001E0C2F8883146
:101550000021C2F88441050602D5C2F88C3101E0B1
:10156000C2F88C41C2F884314006000E491CC9B251
:101570000829EED3C2F8803130BD2DE9F043814611
:101580008846C2F30724D5B2C3F30726DFB22A2068
:10159000FFF7ABFF0020FFF7CCFF4846FFF7C9FF7E
:1015A0000020FFF7C6FF4046FFF7C3FF2B20FFF7E1
:1015B0009CFF2046FFF7BDFF2846FFF7BAFF3046E5
:1015C000FFF7B7FF3846FFF7B4FFBDE8F0432C2024
:1015D0008BE72DE9F0410746002240F23F13EF214F
:1015E0001046FFF7CAFF00254FF4A07600243846C6
:1015F000FFF776FF641CF02CF9D36D1CB542F5D3D0
:10160000BDE8F08100B52820FFF76FFF10205DF8DE
:1016100004EB6AE710B51120FFF767FF782008F0A8
:101620002BF9BDE8104029205FE770B58F4C0125EC
:101630002560052008F020F90020E0630A2008F06A
:101640001BF9E563782008F017F91120FFF74DFF2B
:10165000782008F011F9CF20FFF747FF0020FFF7AF
:1016600068FFC320FFF765FF3020FFF762FFED2022
:10167000FFF73BFF6420FFF75CFF0320FFF759FFF4
:101680001220FFF756FF8120FFF753FFE820FFF7F6
:101690002CFF8520FFF74DFF1020FFF74AFF792030
:1016A000FFF747FFCB20FFF720FF3920FFF741FF6F
:1016B0002C20FFF73EFF0020FFF73BFF3420FFF711
:1016C00038FF0220FFF735FFF720FFF70EFF20203D
:1016D000FFF72FFFEA20FFF708FF0020FFF729FFA1
:1016E0000020FFF726FFC020FFF7FFFE2220FFF7B4
:1016F00020FFC120FFF7F9FE1120FFF71AFFC520D8
:10170000FFF7F3FE3D20FFF714FF2020FFF711FF46
:10171000C720FFF7EAFEAA20FFF70BFF3620FFF7EE
:10172000E4FEC820FFF705FF3A20FFF7DEFE552054
:10173000FFF7FFFEB120FFF7D8FE0020FFF7F9FE0C
:101740001320FFF7F6FEB620FFF7CFFE0A20FFF7C3
:10175000F0FEA220FFF7EDFEF620FFF7C6FE012007
:10176000FFF7E7FE3020FFF7E4FEF220FFF7BDFEB3
:101770000020FFF7DEFE2620FFF7B7FE0120FFF76F
:10178000D8FEE020FFF7B1FE0F20FFF7D2FE3F208A
:10179000FFF7CFFE2F20FFF7CCFE0C20FFF7C9FE8E
:1017A0001020FFF7C6FE0A20FFF7C3FE5320FFF705
:1017B000C0FED520FFF7BDFE4020FFF7BAFE0A208D
:1017C000FFF7B7FE1320FFF7B4FE0320FFF7B1FECB
:1017D0000820FFF7AEFE0320FFF7ABFE0020FFF767
:1017E000A8FEE120FFF781FE0020FFF7A2FE002007
:1017F000FFF79FFE1020FFF79CFE0320FFF799FEE6
:101800000F20FFF796FE0520FFF793FE2C20FFF731
:1018100090FEA220FFF78DFE3F20FFF78AFE0520F5
:10182000FFF787FE0E20FFF784FE0C20FFF781FEF6
:101830003720FFF77EFE3C20FFF77BFE0F20FFF7EF
:1018400078FE1120FFF751FE782008F015F82920C6
:10185000FFF74BFEBDE87040322008F00DB80000E5
:10186000008022424D8000209881214280812242C6
:1018700010B5FF48002101604160C160C163A0F55F
:10188000C070FC4A127A042A02D3FB48016001E0CE
:10189000C0F88811FFF7C9FEF848407820B1BDE8CC
:1018A00010404FF6FF7094E6BDE8104047F619600F
:1018B0008FE62DE9F05FDDE90A78002809D0F04CC9
:1018C00010261825322B1AD02E2B15D0352B15D0DB
:1018D00015E0EC4C302660252D2B07D0202B08D0AE
:1018E000303B03EBC30004EB801408E004F5B45470
:1018F00005E004F5C65402E0303400E06034881995
:10190000401E00F0FF0C5319C8B25B1E6146FFF782
:1019100034FE7543E81705EB5070C0F3CF0900267D
:1019200019E000254FEA182A4FEA172B2078E840E3
:10193000C00704D0F9B25846FFF79CFD04E008F058
:10194000FF015046FFF796FD6D1CADB2082DEDD39B
:10195000641C761CB6B24E45E3D3BDE8F09F2DE97A
:10196000F05FDDE90A7800281CD0C54D90351826B7
:101970002424203B03EBC30000EB400005EB800573
:101980008819401E00F0FF0C1319C8B25B1E614697
:10199000FFF7F3FD7443E01704EB5070C0F3CF0979
:1019A00000262CE0B74D302660242D2B07D0202BAD
:1019B00008D0303B03EBC30005EB8015E0E705F5ED
:1019C000B455DDE705F5C655DAE700244FEA182AD5
:1019D0004FEA172B2878E040C00704D0F9B25846E8
:1019E000FFF748FD04E008F0FF015046FFF742FD15
:1019F000641CA4B2082CEDD36D1C761CB6B24E4507
:101A0000E3D3AAE72DE9FC470746DDE90A890C463E
:101A100016461D4609E0B2B2A1B23846CDE90089AA
:101A2000FFF747FF37B10F346D1C2B78002BF2D135
:101A3000BDE8FC871F34F7E72DE9FC470746DDE9E1
:101A40000A890C4616461D4609E0B2B2A1B23846D4
:101A5000CDE90089FFF783FF2FB117346D1C2B7878
:101A6000002BF2D1E4E71F34F8E770B51646049A6C
:101A700001FB00F4A5B254181844401EC1B2641E04
:101A8000D8B22346FFF779FD002407E036F81400AA
:101A9000C1B2000AFFF7EEFC641CA4B2AC42F5D35D
:101AA00070BD2DE9F041089E069A01FB00F4A5B235
:101AB00054181844401EC1B2641ED8B22346FFF722
:101AC0005CFD0024370A05E0F1B23846FFF7D2FC8E
:101AD000641CA4B2AC42F7D392E52DE9FF5F8046C7
:101AE0000020B8F1010F06D0B8F1020F05D0B8F10F
:101AF000030F05D103E06C2702E0972700E0C2271F
:101B0000DFF8789147F6196509F102094FF6FF767B
:101B100019F80830142B12D00A2200244FF0640C5C
:101B20004FF47A7B4FF0200A022B12D0032B10D0F7
:101B3000042B0ED0002B7CD0012B7AD068E1CDE9AC
:101B4000006551A33A460A210120FFF775FFBDE861
:101B5000FF9F4CF25030814200D3014642F2107098
:101B6000814229D3B1FBF0F330338DF80830B1FB5B
:101B7000F0F300FB1310B0FBFBF030308DF80900E0
:101B8000B1FBFBF00BFB1010B0FBFCF030308DF81C
:101B90000A00B1FBFCF00CFB1010B0FBF2F030308F
:101BA0008DF80B00B1FBF2F002FB101030308DF815
:101BB0000C008DF80D4083E0594522D3B1FBFBF0BA
:101BC00030308DF80800B1FBFBF00BFB1010B0FBC0
:101BD000FCF030308DF80900B1FBFCF00CFB10106C
:101BE000B0FBF2F030308DF80A00B1FBF2F002FBEE
:101BF000101030308DF80B008DF80CA08DF80D40D2
:101C00005EE064291DD3B1FBFCF030308DF8080094
:101C1000B1FBFCF00CFB1010B0FBF2F030308DF893
:101C20000900B1FBF2F002FB101030308DF80A0011
:101C300000E04EE08DF80BA08DF80CA08DF80D4063
:101C40003EE00A292BD3B1FBFCF00CFB1010B0FBDB
:101C5000F2F030308DF80800B1FBF2F002FB10100A
:101C600030308DF809008DF80AA08DF80BA011E036
:101C7000808122424D800020988121424A0100202B
:101C8000B80B0308B8F002082020202020202020D4
:101C9000202000008DF80CA08DF80D4010E0B1FB65
:101CA000F2F002FB101030308DF808008DF809A01A
:101CB0008DF80AA08DF80BA08DF80CA08DF80D40C2
:101CC000CDE9006502AB3A466A210120FFF7B4FE78
:101CD0009EE0012B01D013B106E0252004E0FE4870
:101CE00090F86E0030B346202E23594524D3B1FB23
:101CF000FBF030308DF80800B1FBFBF00BFB10104F
:101D0000B0FBFCF030308DF80900B1FBFCF00CFBAF
:101D10001010B0FBF2F030308DF80A008DF80B3067
:101D2000B1FBF2F002FB101030308DF80C008DF892
:101D30000D404AE04320D7E764291DD3B1FBFCFBEB
:101D40000BF1300B8DF808B0B1FBFCFB0CFB1B1C3E
:101D5000BCFBF2FC0CF1300C8DF809C08DF80A3098
:101D6000B1FBF2F302FB131130318DF80B108DF83B
:101D70000C008DF80D4028E00A2913D3B1FBF2FCCA
:101D80000CF1300C8DF808C08DF80930B1FBF2F37E
:101D900002FB131130318DF80A108DF80C008DF80C
:101DA0000D4012E04FF0300C8DF808C08DF809306E
:101DB000B1FBF2F302FB131130318DF80A108DF8EC
:101DC0000B008DF80C408DF80DA0DFF810B39BF8D8
:101DD000000080B1C248007868B18DF808A08DF885
:101DE00009A08DF80AA08DF80BA08DF80CA08DF835
:101DF0000D408DF80EA0CDE9006502AB3A466A2190
:101E00000120FFF719FE9BF8000008B9B54844709F
:101E100019F8080088B1012818D002281FD003281B
:101E200026D004287FF493AECDE90065AEA33A46F0
:101E30000A210120FFF700FE89E6CDE90065ACA389
:101E40003A460A210120FFF7F7FD80E6CDE900655B
:101E5000A9A33A460A210120FFF7EEFD77E6CDE976
:101E60000065A7A33A460A210120FFF7E5FD6EE6CB
:101E7000CDE90065A4A33A460A210120FFF7DCFD65
:101E800065E670B50124A24D285D052824D2DFE85F
:101E900000F0030A11171D009E48008881B22046F9
:101EA000FFF71BFE1CE09C48008881B22046FFF72C
:101EB00014FE15E0994801882046FFF70EFE0FE05A
:101EC000974801882046FFF708FE09E095480188F9
:101ED0002046FFF702FE03E000212046FFF7FDFD4C
:101EE000641CE4B2032CCFD970BD7FB542F20F71F0
:101EF000884200D908464FF47A73642200240A21EC
:101F0000984220D3B0FBF3F530358DF80850B0FB84
:101F1000F3F503FB1503B3FBF2F330338DF809300F
:101F2000B0FBF2F302FB1302B2FBF1F230328DF898
:101F30000A20B0FBF1F201FB120030308DF80B00EB
:101F40008DF80C4040E02023642819D3B0FBF2F553
:101F500030358DF80850B0FBF2F502FB1502B2FBEC
:101F6000F1F230328DF80920B0FBF1F201FB1200E2
:101F700030308DF80A008DF80B308DF80C4023E0DE
:101F80000A2812D3B0FBF1F230328DF80820B0FBF2
:101F9000F1F201FB120030308DF809008DF80A30A3
:101FA0008DF80B308DF80C400EE0B0FBF1F201FB28
:101FB000120030308DF808008DF809308DF80A30A5
:101FC0008DF80B308DF80C40574858490278098835
:101FD0004FF6FF70401A82B1012A17D0022A1ED094
:101FE000032A25D0042A2CD0CDE9000102ABED2232
:101FF0007E210120FFF720FD7FBDCDE9000102AB6E
:10200000ED227E210120FFF717FD7FBDCDE9000104
:1020100002ABED227E210120FFF70EFD7FBDCDE951
:10202000000102ABED227E210120FFF705FD7FBDFF
:10203000CDE9000102ABED227E210120FFF7FCFC7F
:102040007FBDCDE9000102ABED227E210120FFF72B
:10205000F3FC7FBD7FB542F20F71884200D908467C
:102060004FF47A73642200240A21984220D3B0FBF3
:10207000F3F530358DF80850B0FBF3F503FB15038D
:10208000B3FBF2F330338DF80930B0FBF2F302FB0F
:102090001302B2FBF1F230328DF80A20B0FBF1F2FC
:1020A00001FB120030308DF80B008DF80C406DE014
:1020B0002023642846D3B0FBF2F530358DF8085064
:1020C000B0FBF2F502FB1502B2FBF1F230328DF8F3
:1020D0000920B0FBF1F22BE04D80002080000020B1
:1020E00081000020221100204C55583A00000000C9
:1020F00054656D3A0000000048756D3A000000001C
:10210000434F323A00000000564F433A00000000AF
:102110004C0100208E0100208C010020880100204D
:102120006801002080010020FC0200200003002044
:1021300001FB120030308DF80A008DF80B308DF85D
:102140000C4023E00A2812D3B0FBF1F230328DF8B4
:102150000820B0FBF1F201FB120030308DF80900CD
:102160008DF80A308DF80B308DF80C400EE0B0FB86
:10217000F1F201FB120030308DF808008DF80930C3
:102180008DF80A308DF80B308DF80C40F848F9497D
:102190004FF48C72037809884FF6FF70401A7BB1B8
:1021A000012B15D0022B1BD0032B21D0042B27D0C1
:1021B000CDE9000102AB7E210120FFF73DFC7FBD90
:1021C000CDE9000102AB7E210120FFF735FC7FBD88
:1021D000CDE9000102AB7E210120FFF72DFC7FBD80
:1021E000CDE9000102AB7E210120FFF725FC7FBD78
:1021F000CDE9000102AB7E210120FFF71DFC7FBD70
:10220000CDE9000102AB7E210120FFF715FC7FBD67
:102210001CB547F61964012808D00094D6A3C22241
:10222000002101200194FFF707FC1CBD0094D2A3FC
:102230006C22002101200194FFF7FEFB0094CEA345
:102240009722002101200194FFF7F6FB1CBD3EB54B
:1022500047F619654FF6FF7467208DE831000023BB
:102260001A462D21EF20FFF71CFC92208DE831004B
:1022700000231A462D21EF20FFF713FCBD208DE827
:10228000310000231A462D21EF20FFF70AFC3EBD46
:102290002DE9FF4764250A2320244FF0000C4FF45A
:1022A0007A77202A29D02E264FF0300900297ADBB0
:1022B000B94279DB91FBF7F030308DF8080091FBE3
:1022C000F7F007FB101090FBF5F030308DF80900A7
:1022D00091FBF5F005FB101090FBF3F030308DF81A
:1022E0000A008DF80B6091FBF3F003FB1010303007
:1022F0008DF80C008DF80D20B1E0B9421EDB91FB8A
:10230000F7F030308DF8080091FBF7F007FB101064
:1023100090FBF5F030308DF8090091FBF5F005FBEE
:10232000101090FBF3F030308DF80A0091FBF3F0C1
:1023300003FB101030308DF80B0045E064291BDBE7
:1023400091FBF7F007FB101090FBF5F030308DF8A3
:10235000080091FBF5F005FB101090FBF3F0303016
:102360008DF8090091FBF3F003FB101030308DF86D
:102370000A008DF80B4027E00A2916DB8DF808408B
:1023800091FBF5F005FB101090FBF3F030308DF869
:10239000090091FBF3F003FB101030308DF80A00B8
:1023A0008DF80B4010E05DE015E000290CDB8DF8A6
:1023B000084091FBF3F003FB101030308DF809005A
:1023C0008DF80A408DF80B408DF80C408DF80D40CB
:1023D0008DF80EC0A7E064291BDB91FBF5F03030CF
:1023E0008DF8080091FBF5F005FB101090FBF3F061
:1023F00030308DF809008DF80A6091FBF3F003FB93
:10240000101030308DF80B008DF80C208DF80D4039
:1024100025E00A2912DB91FBF3F030308DF808003B
:102420008DF8096091FBF3F003FB101030308DF84C
:102430000A008DF80C208DF80D4010E08DF8089002
:102440008DF8096091FBF3F003FB101030308DF82C
:102450000A008DF80B208DF80C408DF80D408DF89A
:102460000EC060E048424FF02D0811F57A7F24DC61
:102470008DF8088090FBF7F130318DF8091090FB52
:10248000F7F107FB110191FBF5F130318DF80A10DE
:1024900090FBF5F105FB110191FBF3F130318DF863
:1024A0000B108DF80C6090FBF3F103FB1100303042
:1024B0008DF80D008DF80E2033E011F1640F1DDC56
:1024C0008DF8088090FBF5F130318DF8091090FB04
:1024D000F5F105FB110191FBF3F130318DF80A1094
:1024E0008DF80B6090FBF3F103FB110030308DF899
:1024F0000C008DF80D208DF80E4012E08DF808804C
:102500008DF809908DF80A6090FBF3F103FB110040
:1025100030308DF80B008DF80C208DF80D408DF8C3
:102520000E408DF80FC047F619604FF6FF71CDE9E8
:10253000001002ABC22200210120FFF77DFABDE8A6
:10254000FF877CB50E4647F619654FF6FF740346C4
:102550006C2200210120CDE90045FFF76DFA3346DA
:10256000972200210120CDE90045FFF765FA7CBDE7
:10257000FC0200200003002020202020202020201A
:102580002020202020202020000000002DE9F04104
:1025900086B0044647F617664FF47847CDE90176D2
:1025A000ED20002300901A461E21EF20FFF779FA54
:1025B0000021D14DCF4B03A82A7803F11E0C14B192
:1025C000012C07D00CE001EB020813F8088000F89A
:1025D000018005E001EB02081CF8088000F801808A
:1025E000491CC9B20A29EAD300248DF81640CDE966
:1025F000007603ABED221E210120FFF71DFA28789B
:10260000192804D2401C287006B0BDE8F0812C7057
:10261000FAE70EB555224FF6FF71002809D0CDE933
:102620000021029108218B2300220846FFF739FA86
:102630000EBDCDE9002147F61960029008218B23D9
:1026400000220846FFF72DFA0EBD2DE9FC5F064675
:102650000D4647F619684FF6FF770A2E23D04FF044
:102660000A0A4FF064094FF47A7B002D7CDB2C467C
:10267000CDE90078A1A3202206210120FFF7DCF993
:102680005D4561DB94FBFAF004B2642C38DB94FB0B
:10269000F9F03030CDE90078C3B2052227210020BF
:1026A000FFF75DF934E0CDE9007894A320220621FC
:1026B0000120FFF7C1F9CDE9007820230522272169
:1026C0000020FFF74CF9CDE900782023052257219F
:1026D0000020FFF744F9CDE9007820230522972157
:1026E0000020FFF73CF90020FFF793FFCDE90078C9
:1026F00082A33822D6210120FFF79EF9BDE8FC9F76
:10270000CDE900782023052227210020FFF727F9B3
:1027100094FBF9F009FB104090FBFAF03030CDE962
:102720000078C3B2052257210020FFF718F994FB67
:10273000FAF00AFB10403030CDE90078C3B2052230
:1027400097210020FFF70BF95D4532DA642D0CDB91
:1027500094FBF9F03030CDE90078C3B2052227218F
:102760000020FFF7FCF808E024E0CDE90078202302
:10277000052227210020FFF7F2F894FBF9F009FB6E
:10278000104090FBFAF03030CDE90078C3B205225A
:1027900057210020FFF7E3F894FBFAF00AFB104002
:1027A0003030CDE90078C3B2052297210020FFF731
:1027B000D6F86FE0684204B2642C37DB94FBF9F082
:1027C0003030CDE90078C3B2052227210020FFF781
:1027D000C6F894FBF9F009FB104090FBFAF030309A
:1027E000CDE90078C3B2052257210020FFF7B7F8E2
:1027F00094FBFAF00AFB10403030CDE90078C3B208
:10280000052297210020FFF7AAF8CDE900783CA324
:10281000202206210120FFF70FF9CDE9007837A328
:10282000202228210120FFF707F933E0CDE90078C5
:102830002023052227210020FFF791F894FBF9F0CF
:1028400009FB104090FBFAF03030CDE90078C3B2BC
:10285000052257210020FFF782F894FBFAF00AFBCB
:1028600010403030CDE90078C3B205229721002016
:10287000FFF775F8CDE9007820A32022062101207A
:10288000FFF7DAF8CDE900781DA3202228210120E6
:10289000FFF7D2F80EB1012E08D15D4503DD00200F
:1028A000FFF7B7FE02E00120FFF7B3FE5EB1012E95
:1028B0007FF424AFCDE9007812A33822D62101207D
:1028C000FFF7BAF81AE7104890F86E0040B1CDE96A
:1028D00000780EA33822D6210120FFF7ADF80DE7CE
:1028E000CDE900780AA33822D6210120FFF7A4F809
:1028F00004E700007CF002084A01002020000000EC
:102900002D000000250000004D8000204600000042
:102910004300000010B5254C01212046FDF7B4FD11
:10292000012803D122490A68521C0A6021490888FB
:1029300042F21072904203D20A88521C0A8001E0CF
:10294000002008802046BDE810400121FDF7A3BD0E
:102950007FB504460D4601211020FCF7AFFEADF80F
:102960000840ADF804500020ADF80A00ADF80600AC
:102970000E4C01A92046FDF773F836218DF80010A2
:1029800001218DF8011003228DF802208DF803102B
:102990006846F5F7CAFE012211462046FDF74BFBBB
:1029A00001212046FDF72DFB7FBD000000100040F7
:1029B00054010020EE050020FD49097A05290BD2BB
:1029C000FC4A20B1883291881068F6F795BA8832AF
:1029D00091881068F6F792BAF74A18B102211046AA
:1029E000F6F78ABA02211046F6F788BAF049097A52
:1029F00005290BD2EF4A20B1943291881068F6F77E
:102A00007BBA943291881068F6F778BAEA4A18B11E
:102A100001211046F6F770BA01211046F6F76EBA9A
:102A2000E349097A05290BD2E24A20B1A032918804
:102A30001068F6F761BAA03291881068F6F75EBAAE
:102A4000DD4A18B110211046F6F756BA102110468B
:102A5000F6F754BAD649097A05290BD2D54A20B1DE
:102A6000AC3291881068F6F747BAAC32918810689A
:102A7000F6F744BAD04A18B108211046F6F73CBA26
:102A800008211046F6F73ABAC949097A05290BD246
:102A9000C84A20B1B83291881068F6F72DBAB8321A
:102AA00091881068F6F72ABAC34A18B10421104673
:102AB000F6F722BA04211046F6F720BA2DE9FC41B8
:102AC000F220ADF8040000258DF8075002248DF89F
:102AD0000640BA4E01A93046F6F79FF94FF00308B9
:102AE000ADF804808DF807508DF80640B44F01A969
:102AF0003846F6F792F9ADF804808DF807508DF856
:102B00000640DFF8C08201A94046F6F786F9A848DA
:102B10001025007A052816D21C20ADF804008DF887
:102B200007508DF8064001A94046F6F776F9C02017
:102B3000ADF804008DF807508DF8064001A9304625
:102B4000F6F76BF915E03F20ADF804008DF807505B
:102B50008DF8064001A99848F6F75FF90C20ADF80A
:102B600004008DF807508DF8064001A94046F6F79D
:102B700054F94FF40076ADF800608DF803508DF8ED
:102B8000024069463846F6F748F901213046FCF71D
:102B90008AFDBDE8FC8110B586B04FF40040FCF71B
:102BA00005FD01214802FCF77EFD002001908DF813
:102BB00008008DF809004FF4602103910490012072
:102BC0008DF81400804C01A92046F5F731FE012153
:102BD0002046F5F755FE2046F5F775FE2046F5F739
:102BE00077FE0128FAD02046F5F779FE2046F5F762
:102BF0007BFE0128FAD006B010BD2DE9F04705464E
:102C0000042B06D0062B04D0842B05D0862B03D0B2
:102C100004E04FF4FA7001E04FF47A70DFF890C1ED
:102C200005F114036344DC7E1B7F04EB032340F2B5
:102C3000FF34664FA14203DBBB6718B2BDE8F087E3
:102C400001EB81014E0096FBF0F10CB2CAB1611CA0
:102C500005EB41016144CA7E097F02EB012305EBCC
:102C600044016144CA7E097F02EB01255D1B00FB24
:102C700014636B4393FBF0F000EB01201044B86742
:102C800033E005EB4401614411F8312F497802EB40
:102C90000122611C05EB4101614491F8315091F82A
:102CA000328005EB0821A2EB01091BF0D9FC82461A
:102CB00048461BF0BDFC814630461BF0B9FC064679
:102CC000601C1BF0B5FC51461BF0DEFC31461BF0CE
:102CD000B1FD49461BF0D8FC51461BF077FB1BF0B9
:102CE0006BFC00EB08202844B867B7F8780000B206
:102CF000A4E730B52E4B0A281DD0354C1A1834F9EC
:102D0000105092F8F72005FB021101EB81014900F8
:102D1000521C91FBF2F10A2291FBF2F302FB131316
:102D2000052B00DB0A3191FBF2F324F8103091FB04
:102D3000F2F000B230BD254A907A052800D2D18544
:102D400093F86000B2F92E3003FB0011401C91FB98
:102D5000F0F0D085EDE710B512224FF4E1641329AD
:102D600007D0142949D01B4B997C814268DD20464D
:102D700010BD194B997C814201DD204610BD521EC9
:102D800052B29C5C2144814234DD081A64214843DC
:102D9000995C90FBF1F0042A20DB121F02EBC201C8
:102DA00001EB021100EB8100C0F30E0020E00000F7
:102DB0004D800020B0EF02080018014000080140DB
:102DC000000C014000100140002401405801002087
:102DD0005E110020CEEA0208E1EA020802EBC2011D
:102DE00001EB021100EB8100C0F5C87040F4004017
:102DF00000B210BD002AC2D148E00921FE4B5A8A18
:102E0000824202DD4FF4AF7010BD491E49B233F863
:102E100011402244824210DD101AC0EB0010400025
:102E200033F8112090FBF2F0C1EB011100EB4100EF
:102E3000C0F30E00463000B210BD0029E5D125E0F8
:102E4000521E52B29C5C214481421DDD081A64214D
:102E50004843995C90FBF1F0042A09DB121F02EB56
:102E6000C20101EB021100EB8100C0F30E0009E08A
:102E700002EBC20101EB021100EB8100C0F5C8704A
:102E800040F4004000B210BD002AD9D1DB4810BD8B
:102E90002DE9F0410746DA48B0F90050B0F9024098
:102EA000281B1BF0C5FBD74E31461BF08FFA80461E
:102EB000C8204443684200EB800004EBC0001BF0D4
:102EC000B7FB31461BF082FACF4C21461BF0DCFBEE
:102ED000054638461BF0C4FB41461BF0D5FB29468E
:102EE0001BF006FA21461BF071FA1BF065FB00B2DD
:102EF000BDE8F0812DE9F05F1F4640F2062301FB9B
:102F000003F5C24B4FF47A794FF0640E93F87D3499
:102F1000002848D00E2846D063284AD040F26F3CA3
:102F200001FB0CF64FF49668DFF8D4A201FB08FC15
:102F3000DFF8D882AAF1460A40F2FF3B98F80880F1
:102F40009AF801A0802836D08B2834D001283ED0B2
:102F50000B283CD00D283AD002285FD0822868D0B8
:102F6000032872D0052870D007286ED008286CD0AE
:102F700009286AD00A2868D0832871D085287FD094
:102F800087287DD088287BD0892879D08A2877D057
:102F9000042870D084286ED006286DD086286BD087
:102FA0000C286AD0F2E095FBF9F0434393FBFEF264
:102FB000ECE00A46EAE0B8F1050F02D2BAF1000FE0
:102FC00002D09CFBFBF2E1E096FBF9F2DEE0012887
:102FD00017D00D281AD088B21321FFF7BCFE0104C8
:102FE00002D5C0F30E004042884991F86E1031B10D
:102FF00000EBC000052190FBF1F000F5A070C219B4
:10300000C4E088B20221FFF7A6FEE8E788B21421E7
:10301000FFF7A1FE4628E2DA4620E0E708461AF06C
:10302000AAFE7B4A7B4B1AF00DFF1AF047FE0246C0
:10303000ACE008461AF09FFE774A784B1AF002FF80
:103040001AF03CFE0246A1E0FFE7B1F5F17F0ADC91
:10305000052806D0082804D00A2802D0012295E0CD
:103060000EE0002292E0032808D0072806D00928A5
:1030700004D001228AE01DE049E075E0002285E0ED
:103080004FF4FA73994209DC852805D0882803D0CB
:103090008A2801D0012279E0002277E0994275DD8B
:1030A000832805D0872803D0892801D001226DE02C
:1030B00000226BE0042802D0842803D00AE095FBAC
:1030C000F9F207E0B8F1050F02D2BAF1000F0CD007
:1030D0009CFBFBF2534393FBFEF1494A0A3204285E
:1030E000127805D084280AD00FE096FBF9F2F1E7B8
:1030F000042309B20020FFF780FD044605E0842385
:1031000009B20020FFF779FD0446E2193EE00628E7
:1031100002D0862803D00AE095FBF9F207E0B8F167
:10312000050F02D2BAF1000F0CD09CFBFBF2534307
:1031300093FBFEF1324A0A320628527805D08628DF
:103140000AD00FE096FBF9F2F1E7062309B200205E
:10315000FFF753FD044605E0862309B20020FFF780
:103160004CFD0446E21911E008461AF004FE2C4A10
:103170002C4B1AF067FE1AF0A1FD4FF4C87188427B
:1031800000DA084680B2FFF783FE024610B2BDE8BF
:10319000F09F811E0B2911D2DFE801F00B10100601
:1031A00006060606060606001F49401F31F91000F4
:1031B000704713484638B0F95400704700207047F4
:1031C0008008704770B505460C4602212846F5F781
:1031D000A6FC0523012221462846F5F7B3FB012171
:1031E0002846F5F788FB02212846F5F791FC0028D0
:1031F000F9D028461AE00000F4EA0208E883FFFF4D
:103200009E01002000002043000020414D8000204E
:1032100039B4C876BE9FBA3FC1CAA145B6F3BD3F17
:103220005C8FC2F5285CDF3F86110020BDE870404E
:10323000F5F7CEBB70B50F21FE48FFF7C3FF80B294
:10324000FFF7BEFF01B20A20FFF753FDFA4DFB4C1A
:1032500095F85F1013291BD014291ED0042921D002
:1032600080B20221FFF777FD208700EBC001052225
:1032700091FBF2F101F5A07109B2618795F86E201A
:10328000EF4E92B1022086F82D00A4F8541011E000
:1032900080B21321FFF75FFDE6E780B21421FFF74C
:1032A0005AFDE1E7B4F94E00DEE7012186F82D1062
:1032B000A4F854003C34208B608321880844208388
:1032C0003C3CDD480021D530F8F78EF938B195F84F
:1032D000800395F87F1300EB0120E08670BD95F820
:1032E0005F00A8B1022817D0132815D0042817D0E2
:1032F000D449032850D0102856D011285CD0122869
:1033000067D0421F072A76D831F81200E08679E0AC
:10331000B4F85400E08675E0B4F85400E08671E03B
:10332000E07878B196F8290048B32B3694F902205A
:103330007078317800EB0120B4F856101144081A67
:10334000E0865FE096F8290060B12B3694F9022000
:103350007078317800EB0120B4F856101144081A47
:10336000E0864FE02B36B4F85610707894F90220BE
:103370000844317802EB01210844E08642E02B3614
:10338000B4F85610707894F902200844317802EBB2
:1033900001210844E08635E0B1F90000B4F9541089
:1033A00008444010E0862DE0B1F90000B1F90210A8
:1033B00008444010E08625E0B1F90000B1F9022090
:1033C000B1F9041010440844032190FBF1F0E086A9
:1033D00018E0B1F90000B1F902201044B1F904205D
:1033E000B1F9061011440844C11700EB9170801028
:1033F000E08607E0FFE7012809D015280AD0B4F8D5
:103400005400E08695F8A20015280FD01AE008882D
:10341000E086F7E795F82703FFF7BBFE034695F82C
:103420002803FFF7B6FE181AE086EBE795F82703A6
:10343000FFF7AFFE034695F82803FFF7AAFE181A18
:10344000A4F85200B4F936107F48814200DAE086D1
:10345000B4F9361040F6B83081427FF73FAFE086CE
:1034600070BD10B50D2828D00ADC0D283DD2DFE84C
:1034700000F02C242C242C24242424242424340060
:10348000862812D00EDC83280FD006DC0E281CD034
:1034900080280AD0822828D107E0842805D08528F2
:1034A00023D102E0873804281FD80120FFF79EFAB5
:1034B000BDE810400020FFF77FBA0120FFF796FA21
:1034C000BDE810400120FFF777BA0020FFF78EFA21
:1034D000BDE810400120FFF76FBA0020FFF786FA21
:1034E000BDE810400020FFF767BA10BD10B50828EE
:1034F0005DD2DFE800F0040F1A25303B4651002072
:10350000FFF7C2FA0020FFF7A5FABDE8104000203F
:10351000FFF786BA0020FFF7B7FA0020FFF79AFA04
:10352000BDE810400120FFF77BBA0020FFF7ACFA9E
:103530000120FFF78FFABDE810400020FFF770BAB6
:103540000020FFF7A1FA0120FFF784FABDE8104040
:103550000120FFF765BA0120FFF796FA0020FFF778
:1035600079FABDE810400020FFF75ABA0120FFF7B2
:103570008BFA0020FFF76EFABDE810400120FFF73C
:103580004FBA0120FFF780FA0120FFF763FABDE888
:1035900010400020FFF744BA0120FFF775FA012020
:1035A000FFF758FABDE810400120FFF739BA10BD07
:1035B00002462149092A08D2DFE802F00705080B74
:1035C0000E1114171A0091F89E02704791F89F028D
:1035D000704791F8A002704791F8A102704791F8E6
:1035E000A202704791F8A302704791F8A4027047B5
:1035F00091F8A50270472DE9F84F104E0027776724
:103600000024DFF830800B214046FFF7DBFD716FAF
:1036100008447067022006F02FF9641CE4B2142CF1
:10362000F1D3706F4FF0140BB0FBFBF040F6E441A8
:1036300048430BE0002401404D8000205801002049
:1036400005890020861100200CFEFFFF000B70672B
:10365000F08740F276214FF6FF7988420CD340364E
:10366000A0F27620706309EA8000308071880844F7
:10367000B080403EFE4988823220FE4900900123FE
:103680000022081F01F01FFADFF8ECA348B9B06D63
:103690001AF092FFA6F84E00F06D1AF08DFFAAF80E
:1036A00010000025002408214046FFF78BFD05444B
:1036B000022006F0E1F8641CE4B2142CF3D31420C9
:1036C000B5FBF0F0ED494FF0010B0979090723D55F
:1036D0001AF0C6FFEA491AF0D7FFEA491AF076FE57
:1036E000E9491AF0D1FFE9491AF070FE1AF080FF9B
:1036F00080B23085DE494883DE4920310A88801A4D
:10370000002809DDC88838B981F804B04888C0EBC2
:10371000001009EA8000C8800025002409214046E5
:10372000FFF750FD0544012006F0A6F8641CE4B242
:10373000142CF3D31424B5FBF4F064214843000B9C
:1037400000EB4000708505214046FFF73BFDD04966
:1037500080080880317BCF4D632301BB717B79B139
:10376000F16E0A18F266316F491C3167142923D9AA
:10377000B2FBF4F1B166726E914211D98A1A10E06F
:10378000F16E0144F166306F401C306714281DD97A
:1037900086F80DB0B1FBF4F07066F766376715E098
:1037A000521A052A04D286F800B086F80CB001E05F
:1037B00071662B80F7663767716E091A082901D385
:1037C000706603E086F800B086F80CB0307838B93F
:1037D000306EB0F5C27F03D2401C30662B8012E001
:1037E000AD4C0225207820B1022806D0012807D050
:1037F00009E001F03BFD257005E084F800B002E02F
:1038000001F034FD2570A54890F8D912F1B340F2CB
:10381000DB20FDF7B6FC0002B08640F2DA20FDF7AF
:10382000B0FCB18E0844B086B6F934004FF47A7417
:10383000A04200DDB486B6F93400002800DAB7866D
:103840002436B6F91010B6F92A00F9F798FB308142
:1038500001214046FFF7B6FC00B243F6D0014843D1
:103860000014F08404214046FFF7ACFC00B243F69C
:10387000D0014843001430850C214046FFF7A2FCDC
:10388000C0EBC0004000B0FBF4F000E01DE0308071
:103890000D214046FFF796FCC0EBC0004000B0FB96
:1038A000F4F080B2708036F824190F2901D80F285F
:1038B0003CD9F07A0A2801D2401DF072F07A0A2829
:1038C00001D386F804B0BDE8F88F90F80001744C7D
:1038D000A0B1BAF910100920FFF70BFA2080718E01
:1038E0000820FFF706FA80B23086624A2832118833
:1038F000411A00290EDDD18821B10BE0BAF8100081
:103900002080ECE782F804B05188C1EB011109EA8C
:103910008101D18042F21071884201D9481E30865F
:103920002088604909880844B0867DE7F07A08B1AC
:10393000401EF072F07A0028C5D13771C3E730B568
:103940000021594A4B4B5C3B8EE092F82840012CF9
:1039500071D192F8234004F0F00482F82340F1B1D1
:10396000012921D0022924D0032927D004292AD0D3
:1039700005292DD0062931D0072934D0082937D080
:1039800009293AD00A293DD00B2940D00C2943D02F
:103990000D2946D00E2949D00F294DD050E0B3F95A
:1039A0003600642460434BE0B3F934006424604380
:1039B00046E0188E4FF47A74604341E0188A4FF461
:1039C0007A7460433CE0988B4FF47A74604337E03C
:1039D00027484FF47A740088604331E0D88B4FF465
:1039E0007A7460432CE0188C4FF47A74604327E0BB
:1039F000588A4FF47A74604322E0988A4FF47A74BC
:103A000060431DE0D88A4FF47A74604318E0188B45
:103A10004FF47A74604313E0588B4FF47A74604328
:103A20000EE0588C4FF47A74604309E0D8894FF463
:103A30007A74604304E014E0188D4FF47A746043A4
:103A400069B192F829408CB392F82C4092F82B502F
:103A500004EB05246FF018056C4300EB8400C2F8FA
:103A60001E00491CC9B22E321029FFF46EAF30BDC2
:103A7000CC840020B401002072110020200000201E
:103A800000803B4500F07F450000C84200007C42BA
:103A900034020020360200202E0200204D8000203B
:103AA000920000206E00002005890020FFE792F8B8
:103AB0002C4092F82B5004EB052404EBC40505EBD5
:103AC000041400EB8400CAE710B5FEF7F7FFBDE869
:103AD0001040FFF760B8014600208A1E0B2A0BD267
:103AE000DFE802F00B0A0A060606060606060600CE
:103AF000A748491F30F911007047A648B0F9540093
:103B000070472DE9F041A34A00209071A04E012199
:103B10005A3E3578002D06D173880C2B02D93172AC
:103B2000917100E030729C4B012D93F86E400CD1E6
:103B300093F87154A54202D03172917100E0307255
:103B4000B5790DB1307200E03172914F503F3E4671
:103B50003D7876882DB90C2E02D93972917100E02A
:103B60003872012D0FD193F872C4A44502D0397276
:103B7000917100E0387297F806C0BCF1000F01D0D7
:103B8000387200E03972DFF808C2ACF1460C9CF8DC
:103B9000007057B9BCF80280B8F1020F03D98CF855
:103BA0000810917101E08CF80800012F11D193F8F1
:103BB0007374A74203D08CF80810917101E08CF85F
:103BC00008009CF8064014B18CF8080001E08CF85D
:103BD0000810DFF8BCC1ACF1320C64469CF80070F0
:103BE00064883FB90E2C03D08CF80810917101E065
:103BF0008CF80800012F0FD1152C03D08CF8081079
:103C0000917101E08CF808009CF8064014B18CF822
:103C1000080001E08CF80810DFF874C1ACF13C0C2E
:103C200064469CF8007064883FB90E2C03D08CF871
:103C30000810917101E08CF80800012F0FD1152CAC
:103C400003D08CF80810917101E08CF808009CF802
:103C5000064014B18CF8080001E08CF80810D47903
:103C60003CB993F8B770022F02D01172917100E045
:103C70001072012C07D193F8B840022C02D01172B7
:103C8000917100E01072002D05D193F8A230B3427B
:103C900003D051729171BDE8F0815072FBE770B5AD
:103CA000FFF72FFF3C4E96F86F04012838D1384CAF
:103CB0003A49463CA4F11405B4F90400B5F90430BE
:103CC000374A984203DA04200870107002E000209E
:103CD00008701070287818B9A878FFF7FCFEA88043
:103CE0002B4D503D287818B9A878FFF7F4FEA8802E
:103CF000207818B9A078FFF7EEFEA08096F870043F
:103D000001280DD1224923483C390A780AB9828E0C
:103D10008A801F4932390A78002A01D1808E888032
:103D200070BDF0B51C4C0125002194F86F24194892
:103D3000012A0AD041714079012805D11948028829
:103D4000428004F89E1F6570F0BD82790AB141710E
:103D5000F1E7114BDFF838C094F870645A7C9B7C13
:103D6000ACF15A0C02EB0322BCF904300CF114073D
:103D70009A1AB7F904301EB19A4207DD4571DAE7A5
:103D80009A4201DD4571D6E74171D4E74171D2E72E
:103D900086110020580100204D8000206A0000207C
:103DA000660000209600002008B501210820FBF7DE
:103DB0007AFC3020ADF8000010208DF803000220BE
:103DC0008DF802006946FE48F5F727F808BD0B4656
:103DD0001146012B07D0022B07D0032B07D0042B51
:103DE00007D1FCF739BBFCF731BBFCF731BBFCF763
:103DF00031BB704730B40346F24AF34CF348127AB1
:103E0000062B27D2DFE803F026191D030E21042A12
:103E100004D320460A4630BC0121D8E70A4630BC0C
:103E20000321D4E7042A04D320460A4630BC0221E9
:103E3000CDE70A4630BC0421C9E70A4630BC01215F
:103E4000C5E70A4630BC0221C1E70A4630BC012161
:103E5000DF48BCE730BC7047DD4B002804D04FF48E
:103E60007A7203211846B2E7002203211846AEE712
:103E7000D74B002804D04FF47A7202211846A6E7E7
:103E8000002202211846A2E72DE9F84F8346D148C7
:103E9000421C02F1010A00789AF800101278BBF176
:103EA000080F57D2DFE80BF056040F1B27333F4BA8
:103EB000002500F0010601F0010402F00107A84608
:103EC0004FF0010946E00125C0F34006C1F340046C
:103ED000C2F340074FF002084FF003093AE0022511
:103EE000C0F38006C1F38004C2F380074FF00408DA
:103EF0004FF005092EE00325C0F3C006C1F3C0044E
:103F0000C2F3C0074FF006084FF0070922E004256E
:103F1000C0F30016C1F30014C2F300174FF00808F5
:103F20004FF0090916E00525C0F34016C1F340140F
:103F3000C2F340174FF00A084FF00B090AE00625BC
:103F4000C0F38016C1F38014C2F380174FF00C0841
:103F50004FF00D09B74247D19E484146801E008967
:103F6000F7F724FB0090A6B100200099884220D0EA
:103F70008EB1002297484146801DF7F728FB9548EF
:103F80009049009A083042B1294491F842114155B4
:103F900007E00120E9E70122ECE7294491F8491103
:103FA0004155405D28B18B4801224946801DF7F7F5
:103FB0000EFB884D4946AD1E2889F7F7F7FA002811
:103FC00012D185F801B007B90124BBF1080F0BD25B
:103FD000DFE80BF00A040C131A21282F9AF80000CE
:103FE00064F300008AF80000BDE8F88F9AF800003A
:103FF00064F341008AF80000F6E79AF8000064F3E1
:1040000082008AF80000EFE79AF8000064F3C3002A
:104010008AF80000E8E79AF8000064F304108AF8D0
:104020000000E1E79AF8000064F345108AF8000008
:10403000DAE79AF8000064F386108AF80000D3E704
:104040002DE9F84F6448DFF894810078002823D0E8
:104050000124DFF880A14FF000090AF1020AAAF159
:104060000106F51EAF1C2046FFF70EFF68780028FA
:1040700077D0012803D09AF80010CA0772D0387898
:104080003178401C60F3000131709AF8000020F094
:1040900001008AF80000DEE0B8F90000C82815DA4F
:1040A0004FF47A710120FFF7A5FE00210220FFF7EF
:1040B000A1FE00210320FFF79DFE00210420FFF751
:1040C00099FE00210520FFF795FE61E0B0F5C87F5D
:1040D00015DA00210120FFF78DFE4FF47A710220DE
:1040E000FFF788FE00210320FFF784FE0021042053
:1040F000FFF780FE00210520FFF77CFE48E0B0F5C9
:10410000167F15DA00210120FFF774FE002102203E
:10411000FFF770FE4FF47A710320FFF76BFE00216A
:104120000420FFF767FE00210520FFF763FE2FE064
:10413000B0F5487F17DA00210120FFF75BFE002170
:104140000220FFF757FE00210320FFF753FE4FF434
:104150007A710420FFF74EFE00210520FFF74AFE8A
:1041600016E07AE027E000210120FFF743FE00215E
:104170000220FFF73FFE00210320FFF73BFE002156
:104180000420FFF737FE4FF47A710520FFF732FE67
:104190000F4CB8F8002002212046FFF718FEB8F8AF
:1041A000022003212046FFF712FEBDE8F84F4FF42E
:1041B000FA7005F061BB022801D08A071CD50FE018
:1041C000000C01404D8000200004004000340140FC
:1041D0000008004018020020A7000020EE00002088
:1041E000387832784010401C60F34102327021F080
:1041F00002008AF800002EE0032801D04A070BD500
:10420000387832788010401C60F38202327021F0DE
:1042100004008AF800001EE0042801D00A070BD52C
:1042200038783278C010401C60F3C302327021F03D
:1042300008008AF800000EE0052801D0C8060AD55B
:10424000387832780011401C60F30412327021F08B
:1042500010008AF8000085F80190641CE4B2062C76
:10426000FFF401AFDFF8B4A3DFF8B4B30AF1D6006E
:104270009AF86A100090062916D00024214600986A
:10428000F7F7B2F980B30AEB040090F8B9000328FD
:1042900030D02146E348F7F7A7F918B300222146AA
:1042A000E148F7F787F925E0E048007838B1287849
:1042B000C0070DD0E9880120FFF79CFD4DE00021EB
:1042C0000120FFF797FD287800F0FE00287044E0F9
:1042D0004FF47A710120FFF78DFD297841F001013B
:1042E00029703AE00122DAE7FFE7D249D04801EB32
:1042F0008411C8619BF8000001281FD19AF853026D
:10430000022802D001280DD013E02146CA48F7F751
:104310006BF928B100222146C348F7F74BF908E0B2
:104320000122F8E72CB98AF8D6900021D620FCF7B4
:1043300029FF042C02D103208BF80000641CE4B296
:10434000052C9BD33078C00717D000210120FFF740
:1043500051FD287800F0FE0028703078800723D4C3
:10436000287880071BD44FF47A710220FFF742FDB2
:10437000297841F0020129701EE02878C00704D096
:10438000E9880120FFF736FDE7E74FF47A71012055
:10439000FFF730FD297841F001012970DDE7E98858
:1043A0000220FFF727FD07E000210220FFF722FD92
:1043B000287800F0FD0028703078400711D4287864
:1043C000400709D44FF47A710320FFF713FD2978D1
:1043D00041F0040129700CE0E9880320FFF70AFD91
:1043E00007E000210320FFF705FD287800F0FB001F
:1043F00028703078000711D42878000709D44FF4CA
:104400007A710420FFF7F6FC297841F00801297041
:104410000CE0E9880420FFF7EDFC07E00021042010
:10442000FFF7E8FC287800F0F70028703078C00625
:1044300011D42878C00609D44FF47A710520FFF70B
:10444000D9FC287840F0100028700CE0E98805209D
:10445000FFF7D0FC07E000210520FFF7CBFC287810
:1044600000F0EF0028709BF8000001280DD19AF8A9
:104470005302022809D1012205210098F7F79AF882
:10448000012206210098F7F795F805210098F7F723
:10449000ABF880B39BF80000012803D19AF85302CF
:1044A000022811D09AF8670300029AF868130844AA
:1044B00000B29AF87B1079B111290DD082B2022195
:1044C0005E48FFF784FC26E09AF8560200029AF84C
:1044D0005512084400B2ECE7012805D00022022161
:1044E0005648FFF774FC16E04FF47A7202215348E5
:1044F000FFF76DFC0FE0FFE79AF87B00A8B10128F9
:104500001ED004281CD011280FD0B8F8002002219A
:104510004A48FFF75CFC06210098F7F765F8E8B316
:104520009BF80000012824D027E03878800603D5C6
:104530000120FFF79DFCEEE70020FFF799FCEAE77A
:104540009AF86F0401280DD19AF87404B8F9001094
:1045500000EB8002B1EB420F04DA00EB8000400078
:10456000A8F80000B8F8002002213448FFF72FFC1B
:10457000D1E79AF85302022815D09AF8690300028D
:104580009AF86A13084400B29AF87C1089B19AF834
:104590007B1011290DD082B2032100E019E0BDE8A3
:1045A000F84F264813E49AF857020102084400B273
:1045B000EAE7012805D0BDE8F84F002203211F4893
:1045C00005E4BDE8F84F4FF47A7203211B48FFF76A
:1045D000FEBB9AF87C0068B1012816D0042814D0DC
:1045E000112807D0B8F80220BDE8F84F032113487E
:1045F000FFF7EDBB3878400603D5BDE8F84F012042
:104600002AE4BDE8F84F002026E4B8F80220BDE80F
:10461000F84F03210948FFF7DABB00004D80002066
:1046200079000020B8830020190200206A000020D1
:1046300000007F432C850020A1820020000800405C
:1046400010B5FCF75AFB0120FCF791FB012005F0A7
:10465000F3F80120FCF780FB012005F0EDF80020C5
:10466000FCF785FB0A2005F0E7F80020FCF774FB57
:10467000BDE810400A2005F0DFB810B5FCF73DFB9F
:104680000020FCF769FB012005F0D6F80020FCF7BC
:104690006EFB012005F0D0F80120FCF75DFB0A203D
:1046A00005F0CAF80120FCF762FBBDE810400A20C3
:1046B00005F0C2B870B50546FCF71FFB80242C42FC
:1046C00003D10020FCF753FB02E00120FCF74FFB75
:1046D000052005F0B1F80120FCF73EFB052005F0B0
:1046E000ABF80020FCF738FB012005F0A5F86408C2
:1046F000002CE4D1BDE87040FCF7D2BB70B5044695
:104700000025FCF71DFB4FF47A7607E0641EE4B247
:1047100001D2042070BD304605F08EF8FCF737FB5F
:104720000028F3D0284670BD2DE9F04105460E461D
:104730001746002028700120FCF719FBFCF7CCFA83
:1047400080240120FCF708FB012005F075F83846AD
:10475000FFF7D4FF8046032005F06EF8FCF7E1FA7E
:10476000FCF710FB10B12878204328700020FCF7DC
:10477000F3FA012005F060F86408002CE1D1FCF7A1
:10478000BCFABEB10120FCF7F2FA012005F054F8A2
:104790000120FCF7E1FA052005F04EF80020FCF7B7
:1047A000DBFA0120FCF7E3FA142005F045F8404657
:1047B000BDE8F0810020FCF7DAFAE6E710B5FFF774
:1047C0003FFF0020FFF776FF002803D1BDE810402F
:1047D00006206FE710BD0000F9494000087040F066
:1047E000010048707047F7E7FFF747BF70B505460F
:1047F000FF20002340F2311410E0EA5C5040082210
:10480000060603D584EA4000C0B201E04006000E6F
:10481000521ED2B2002AF3D15B1CDBB28B42ECD326
:1048200070BD10B51446FFF7E1FFA04201D0022091
:1048300010BD002010BD7CB504460D46002101A826
:10484000FFF772FF28B9002211460DF10500FFF7AE
:104850006BFF20B9002229466846FFF765FF28B99B
:104860009DF80020022101A8FFF7DBFF9DF805104D
:104870009DF8042041EA022121807CBD10B5FFF79C
:10488000DFFECF484078BDE81040FFF713BF70B59A
:104890000446200AFFF70EFF0546E0B2FFF70AFFC5
:1048A000284370BD10B5FFF7CBFEC5480078BDE8C2
:1048B0001040FFF7FFBEF8B50646FFF7F3FF0546C9
:1048C0004FF45E50FFF7E3FF40EA050414B9FFF729
:1048D000D5FF04462CB9642200216846FFF7ABFFE0
:1048E000044634B9002201210DF10200FFF7A3FFB5
:1048F0000446FFF779FF34B9BDF80200BDF8001097
:1049000040EA014030602046F8BD70B50546FFF72B
:10491000C9FF044624B94FF22D30FFF7B8FF044613
:1049200014B9FFF7ABFF04462CB900220121284639
:10493000FFF781FF0446FFF757FF204670BD10B513
:10494000FFF7B0FF044624B943F24100FFF79FFF91
:104950000446FFF749FF204610BD10B519F080FE50
:10496000984919F091FE984919F08EFEBDE8104063
:10497000964919F02BBD10B519F072FE944919F043
:1049800083FE914919F080FE904919F01FFDBDE8A2
:104990001040904919F04EBF2DE9FC41074688466A
:1049A00016461D46FFF77EFF0446200005D196B14E
:1049B000012E0AD0022E02D0802494B120E042F2CF
:1049C0001640FFF764FF0446F7E742F20B40FFF79B
:1049D0005EFF0446F1E74FF41050FFF758FF04461E
:1049E000EBE74FF47A7606E0FFF748FF04462CB178
:1049F000304604F021FF6D1EEDB2F5D205B9042456
:104A000064B90022114601A8FFF715FF05460022F0
:104A100001216846FFF70FFF40EA0504FFF7E4FEB7
:104A200054B9BDF80400FFF7A6FF3860BDF80000D8
:104A3000FFF793FFC8F800002046BDE8FC812DE990
:104A4000FC4106460F4615469846FFF72BFF0446E5
:104A50002CB995B1012D0AD0022D02D0802494B139
:104A600014E042F61040FFF712FF0446F7E742F663
:104A70000D40FFF70CFF0446F1E742F60640FFF752
:104A800006FF0446EBE7FFF7F9FE04462CB9424661
:104A9000002101A8FFF7CFFE04462CB90022012116
:104AA0006846FFF7C8FE0446FFF79EFE4CB9BDF806
:104AB0000400FFF760FF3060BDF80000FFF74DFF16
:104AC00038602046B9E730B4029C002B04D0012B9B
:104AD00005D0802030BC7047234630BCAFE723466A
:104AE00030BC59E770B505460E46FFF7DBFE0446BD
:104AF0002CB97DB3012D2ED0022D04D08024FFF7D8
:104B000073FE204670BD052E22D2DFE806F00309B1
:104B10000F151B0042F22F00FFF7B9FE0446EEE727
:104B200042F22D10FFF7B3FE0446E8E742F22B20D5
:104B3000FFF7ADFE0446E2E742F22930FFF7A7FE99
:104B40000446DCE742F22A70FFF7A1FE0446D6E7EE
:104B50008024D4E726E0052E22D2DFE806F0030900
:104B60000F151B0042F22400FFF791FE0446C6E732
:104B700042F22610FFF78BFE0446C0E742F22020E7
:104B8000FFF785FE0446BAE742F22230FFF77FFEC8
:104B90000446B4E742F22170FFF779FE0446AEE71F
:104BA0008024ACE7052E2FD2DFE806F003161C2286
:104BB000280042F23200FFF76AFE04469FE7000039
:104BC000280200200000C8420000204100FF7F476B
:104BD00000002F430000E14342F23010FFF757FE80
:104BE00004468CE742F23620FFF751FE044686E782
:104BF00042F23430FFF74BFE044680E742F2377052
:104C0000FFF745FE04467AE7802478E77CB5054641
:104C10000E46FFF747FE044624B94FF46040FFF705
:104C200036FE044614B9FFF729FE04462CB90022CB
:104C3000114601A8FFF7FFFD04462CB9002201210F
:104C40006846FFF7F8FD04464CB9BDF80400FFF7CD
:104C500092FE2860BDF80000FFF77FFE3060FFF78E
:104C6000C3FD20467CBD10B5FFF71CFE044624B9E9
:104C700043F26D00FFF70BFE0446FFF7B5FD20463B
:104C800010BD10B5FFF70EFE044624B943F26600CE
:104C9000FFF7FDFD0446FFF7A7FD204610BD70B5E8
:104CA000FFF700FE054643F2A200FFF7F0FD40EAE1
:104CB0000504FFF799FD1CB94CF2503004F0BCFD1F
:104CC000204670BD10B5244C4FF080502060234822
:104CD00004F0B2FDA0142060BDE810404CF250304A
:104CE00004F0AABD38B5010A8DF800108DF8010056
:104CF00002216846FFF77AFD04469DF80000FFF7A1
:104D0000D9FC18B99DF80100FFF7D4FC002802D1A6
:104D10002046FFF7CFFC38BD10B5114919F0E8FA6D
:104D2000104919F053FB104919F0AEFC19F060FC62
:104D300080B210BD10B50D4919F048FB0A4919F0B1
:104D4000A3FC19F055FC80B210BD03480838006878
:104D5000C0F3802070470000100C0140A0860100C5
:104D60000000344200002F4300FF7F470000C8428C
:104D70000A1A00D5524292B2642A07D8052A05D9E8
:104D8000401A062290FBF2F0084400B270472DE969
:104D9000F84301211020FAF786FC4020ADF800000E
:104DA00010208DF8030003208DF80200F94C6946AD
:104DB0002046F4F732F840212046F4F79DF840F2FF
:104DC00029394846FCF7DDF9F34C207040F22A38C7
:104DD0004046FCF7D6F9607040F22B373846FCF7B6
:104DE000D0F9A0707E1C3046FCF7CBF9E07020783B
:104DF0001425FF2804D1257014214846FCF7C2F978
:104E00006078FF2805D11E2060701E214046FCF707
:104E1000B9F9A078FF2805D13720A070372138468E
:104E2000FCF7B0F9E078FF2805D16420E070642138
:104E30003046FCF7A7F9D84824384571BDE8F88317
:104E40002DE9F04F89B080460D464FF07E5427463D
:104E50002646D248D54940444144CDE90710D449BB
:104E6000CF4A29440691D349CE4B05EB0109D249DB
:104E7000DFF834C305EB010AC849491E05EB010BF5
:104E8000B0F5B50F7FD20698CC49B0F5000F1CD80D
:104E9000CB480190CB480290CB4803902046049029
:104EA0000E46BE494046494219F0C4FC314619F04D
:104EB0008DFA0746BE4E28467642314619F0BAFCB6
:104EC000314619F083FA0646DCE0B9F59C0F1CD296
:104ED000BD4801904FF07E500290BC480390049270
:104EE0000E46AE494046494219F0A4FC314619F03D
:104EF0006DFA0746AF492846C94319F09BFCAC49F7
:104F0000494219F063FA0646BCE04FF44810824566
:104F10001AD2AE4801900292AD48039004930E4617
:104F20009E494046494219F085FC314619F04EFA37
:104F30000746A1492846C94319F07CFC9C494942CF
:104F400019F044FA06469DE083451AD2A048019024
:104F50000293A0480390CDF810C00E468F494046FA
:104F6000494219F067FC314619F030FA07468B497F
:104F70002846494219F05EFC8D49494219F026FA4B
:104F800006467FE0FFE707984FF4481E704579D842
:104F9000864906984942B0F5000F1CD8894801900F
:104FA0008D4802904FF07E5003908C480490814EC3
:104FB0004046F64319F03EFC314619F007FA074621
:104FC0007B4E28467642314619F034FC314619F0C2
:104FD000FDF9064656E0B9F59C0F1AD24FF07E5007
:104FE00001907E48029003927D480490714E4046A5
:104FF000F64319F01FFC314619F0E8F9074631462F
:10500000284619F017FC6A49494219F0DFF90646AB
:1050100038E07046824519D201927148029003939C
:1050200070480490634E4046F64319F003FC314645
:1050300019F0CCF9074660492846C94319F0FAFB34
:105040005B49494219F0C2F906461BE0834519D273
:10505000019364480290CDF80CC063480490554E0B
:105060004046F64319F0E6FB314619F0AFF9074622
:105070004A492846494219F0DDFB4D49494219F099
:10508000A5F9064659490898884231D80698B0F1E2
:10509000997F2DD83946029819F0F6FA0446394618
:1050A0004FF07E5019F0C6FB0590019919F0ECFA0B
:1050B000214619F01DF900903946049819F0E4FAD8
:1050C00004460399059819F0DFFA214619F010F902
:1050D000314619F0D9FA044631464FF07E5019F0A6
:1050E000A9FB009919F0D0FA214619F001F90446FC
:1050F0002F49DFF8FCC0491E3E4A3F4B3F4E404F10
:10510000A5F500002944E04522DDBD4204D8B5F5EF
:10511000000F01DA1446A5E03A4A904201D21C463B
:10512000A0E03948814201D22B4C9BE037488145B1
:1051300001D22A4C96E03648824501D2284C91E0B3
:10514000834501D2274C8DE0B54200DD264C89E035
:10515000DFF848E0CEF1000EF04563DABD4204D836
:10516000B5F5000F01DA14467CE0264A904201D2E0
:105170001C4677E02448814201D2114C72E023485A
:10518000814501D2104C6DE02148824542D20F4C3E
:1051900068E000000010014050020020000038BC10
:1051A000CDCC4C3FF6281C3F6666E63E0080DDBB5A
:1051B000000038BDFFFFB7BCFFFF69BC00007A43A9
:1051C0007B14CE3F8FC2B53F6666A63FA4707D3F7D
:1051D00014AE473F0AD7233F0000A03F7B146E3F29
:1051E0003333333F713D0A3FF628DC3E00808C00AC
:1051F0000080544466661640CDCCCC3F0000FA4394
:105200000000C8C200004842FFFF7F00FFFF4D00C2
:10521000FFFF3100834501D2FB4C23E0B54221DD85
:10522000FA4C1FE0FA48FB49404488421AD2FA4837
:10523000854217DAB54215DDBD4201D9144611E0A9
:1052400001D21C460EE00898B0F5B50F01D2F34C20
:1052500008E00798B0F5481F01D2F14C02E0E045A4
:1052600000DBF04C09B02046BDE8F08F2DE9FF5F70
:10527000DFF8B4A39AF8020000287DD00AF12807CD
:105280009AF804003C1F07F1080B4FF000090028B2
:1052900073D09AF8000000286FD0BAF81800DFF831
:1052A0008C83642869D9BAF81C001421B0FBF1F092
:1052B00019F0D6F90546CAF820004146284619F0EB
:1052C000E3F9DB4919F0ACFA294619F07FF819F037
:1052D0008FF980B2AAF8160018F064FDD54E0022AE
:1052E000334618F057FB18F067FA05463968DBF8C3
:1052F0000000FFF7A5FD294619F0C6F90290BAF89B
:10530000160018F04FFD0022334618F043FB18F04A
:1053100053FA05467968DBF80400FFF791FD29464A
:1053200019F0B2F90190029818F0B6FFC24AC34BC7
:1053300018F088FD05460E46019818F0ADFF2A4684
:10534000334618F043FD3ED2BAF8100019F088F940
:105350000090BAF8160019F083F90390029919F039
:1053600093F9414618F0C4FFB14E0146304619F09A
:105370002DF80546019901E06FE024E0039819F04B
:1053800083F9414618F0B4FF0146304619F01EF883
:10539000294619F04FFAAA4919F076F9009918F040
:1053A000A7FF19F025F980B2AAF81000BAF8121078
:1053B00022780B1A521F934201DB814203D2AAF8D2
:1053C0001C108AF80090BAF81A00BAF80880404514
:1053D00001D9AAF81A809AF80300401CC0B28AF8D2
:1053E00003009AF805600125B0420FD38AF80450F3
:1053F0008AF803909348B0F9000019F019F9386061
:10540000BAF8180019F02CF9CBF80000AAF81E80A1
:105410008D499AF8030021F81080711E88420BD143
:105420008848B0F9000019F003F97860BAF818005C
:1054300019F016F9CBF80400BAF80E005746401CD4
:1054400080B2AAF80E0041F2883240F2FF31904259
:1054500016D9787801280CD012E0BAF80800AAF81A
:105460001A00AAF81E00AAF81C0077490880BDE8B7
:10547000FF9F87F80190A7F80E90788BB883798307
:10548000F889B0F5117F06D9387820B9A7F80E90C1
:10549000788BB88379833879002878D0B98B3B46EC
:1054A000884574D9DFF8A0C1BCF8000058820020FC
:1054B00008E03CF81020B3F812A0524500D95A82F7
:1054C000401CC0B2B042F4D3BCF8260018820020C1
:1054D00008E03CF81020B3F810A0524500D21A8220
:1054E000401CC0B2B042F4D3188A884200D8198256
:1054F000A678A8EB01000222B04229DD93F800C093
:10550000BCF1030F24D0598AB3F810A0A1EB0A0113
:10551000B14204DDA3F814A00320187060E066789F
:10552000B14204DDBCF1020F01D01A7058E02678B8
:10553000B14255DDBCF1010F52D007D9A6F10506E5
:10554000B04201DA1D704BE01A7049E01D7047E06F
:1055500094F801C0604521DDB0421FDA1E78022EAA
:105560001CD019D2598AB3F810A0A1EB0A0AE2455F
:1055700001DD1A7034E021788A4531DD012E2FD00B
:1055800008D9A1F10501884202DD1D7028E022E062
:105590001A7025E01D7023E01A7021E022789042F5
:1055A0000FDD60450DDA187801280AD010B117D93F
:1055B0001D7015E0588A198A401A904210DD1D703E
:1055C0000EE0A8EB0100521F904201DB884507D294
:1055D00083F8009004E018B187F80090A7F81C80C9
:1055E0003878032802D287F8019000E07D700E4ED3
:1055F000383640B1012857D0DFF850A002287CD0BF
:1056000003287BD002E123E014AE473F0AD7233FB3
:10561000FFFF37BCFF7F8C000000C842AE47213F30
:105620008FC2F53EF628DC3E2C020020000020410F
:105630000000484200003E408FC2F5285C8FEA3FE0
:105640000000A0418E010020B4110020000069403C
:10565000B7F81C90C84515D9207818F0A3FB04466C
:105660000D46A8EB09006421484318F084FB22464C
:105670002B4618F08FF900226A4B18F0CFF818F07B
:105680004DFBB881B889F9880844A0F5FA7080B25A
:10569000B8813188814202D8491EB981B6E06328B9
:1056A00001D86320B881B1E0B7F81C90C84520D973
:1056B000607894F800A0A0EB0A0018F05CFB0446A8
:1056C0000D46A8EB0900A0EB0A00C821484318F0DA
:1056D00052FB22462B4618F05DF904460D463088F1
:1056E00018F060FB22462B4618F098F818F016FBCD
:1056F000B881B889F988084401E00FE04AE0A0F5D4
:10570000FA7080B2B8817188814202D8491EB9818D
:105710007CE03188814279D3B98177E0B98BA07878
:10572000A8EB0109814523DD192821D988451FD916
:1057300094F80180A0EB080018F01DFB04460D460C
:10574000A9EB080018F017FB22462B4618F022F9A7
:105750000022534618F076FB04460D46708818F078
:1057600021FB22462B4618F059F818F0D7FAB881D9
:10577000B889F9880844A0F5FA7080B2B881B18878
:10578000814202D8491EB98140E0718881423DD3EF
:10579000B9813BE0B98BA078A8EB0109814523DDF5
:1057A000192821D988451FD994F80180A0EB080059
:1057B00018F0E1FA04460D46A9EB080018F0DBFAF0
:1057C00022462B4618F0E6F80022534618F03AFB22
:1057D00004460D46B08818F0E5FA22462B4618F02C
:1057E0001DF818F09BFAB881B889F9880844A0F52B
:1057F000FA7080B2B881F188814202D8491EB9811D
:1058000004E0B188814201D33088B88178890222CE
:1058100001B2B88900B2FFF7ABFA78817889024902
:10582000088124E600005940CC840020F0B50346EE
:105830000025084600260A2A01D00670F0BD002B7C
:105840001DD005DA4FF02D0200F8012BC3F1000343
:1058500042F210724FF00A0793FBF2F454EA050C7F
:1058600006D004F1300500F8015B04FB123301257A
:1058700092FBF7F2002AEFDC06700846F0BD3022FA
:10588000027046700846F0BD0FB430B585B00546CD
:105890000AA800900EE05C2914D025292CD0521CB7
:1058A00028460992FAF72EFF80212846FAF797FF3B
:1058B0000028F9D0099A11780029ECD105B030BC44
:1058C0005DF814FB521C099210786E280CD07228D7
:1058D00002D0521C0992E7E70D212846FAF712FF81
:1058E0000998401C0990DFE70A212846FAF70AFFC9
:1058F0000998401C0990D7E7521C09921078642837
:1059000019D0732802D0521C0992CDE7009810C814
:10591000009009E02846FAF7F5FE80212846FAF7BC
:105920005EFF0028F9D0641C21780029F2D1099883
:10593000401C0990B8E7009808C800900A2201A905
:105940001846FFF773FF01AC09E02846FAF7DAFEC4
:1059500080212846FAF743FF0028F9D0641C2178FB
:105960000029F2D10998401C09909DE708B54FF431
:10597000A060F2F7D5FE34208DF8000001208DF8EC
:10598000010000218DF802108DF803006846F2F73F
:10599000CCFE08BD10B586B00121C804F9F78EFE13
:1059A00001211020F9F77FFE4FF48060ADF814005C
:1059B00018208DF8170003208DF81600F94C05A962
:1059C0002046F3F72AFAE114ADF8141004218DF8FB
:1059D000171005A92046F3F720FA4FF4E1300190A3
:1059E0000020ADF80800ADF80A00ADF80C00ADF8E5
:1059F00010000C20ADF80E00EB4C01A92046FAF780
:105A0000A5FD012240F225512046FAF726FE01228B
:105A100040F224412046FAF720FEFFF7A7FF0121BC
:105A20002046FAF70EFE06B010BD08B510208DF81E
:105A3000030003208DF8020001210820F9F733FE4E
:105A40004FF48050ADF800006946D848F3F7E5F907
:105A500008BD10B5FFF7E9FFFFF79CFF02F045FA1C
:105A6000BDE810404FF48051D048F3F745BA70B507
:105A7000CE4D4FF4805421462846F3F73FFA4FF4B9
:105A8000FA7003F0F9FE21462846BDE87040F3F7AE
:105A900033BA2DE9F05F07460E4693469846002537
:105AA000DFF80CA3BAF800046FF30E00AAF80004A4
:105AB0000024DFF8F4920BE0395D4846FAF722FE45
:105AC00080214846FAF78BFE0028F9D0641CA4B266
:105AD0004445F1D3BAF800046FF30E00AAF80004AD
:105AE0009AF8010420F080008AF8010404E0012003
:105AF00003F0C2FEF9F79FFC9AF80104000604D4F3
:105B000028466D1CADB20528F1D3BAF80014002068
:105B1000C1F30E010AF8010086B1BBF1000F0DD0F0
:105B20003146A34815F062FC28B95946A04815F043
:105B30005DFC002800D00120BDE8F09F3EB1314659
:105B40009B4815F053FC0028F6D00120F4E7594695
:105B5000974815F04BFC0028EED00120ECE72DE92A
:105B6000F0410D4690461E460024024691A18E4803
:105B7000FFF78AFE55EA080011D08D4FB7F80004F0
:105B80006FF30E00A7F8000497F8010420F08000DE
:105B900087F801043220B6FBF0F086B207E001205E
:105BA000BDE8F081322003F067FEF9F744FC97F876
:105BB0000104000604D42046641CA4B2B042F1D310
:105BC000B7F800140020C1F30E0178547DB1B8F18C
:105BD000000F0CD02946764815F008FC28B941463C
:105BE000734815F003FC0028DAD00120D8E73DB156
:105BF00029466F4815F0FAFB0028D1D00120CFE7E5
:105C000041466B4815F0F2FB0028C9D00120C7E7D8
:105C100070B500244FF480516448F3F76DF94FF4E8
:105C20007A7003F029FE4FF4FA750CE02B4600223F
:105C300062A163A0FFF793FF08B1022070BDFFF7D8
:105C400016FF641CE4B20A2CF0D301D0012070BD11
:105C5000002070BD40F6C413002805D0012807D0ED
:105C6000022809D00020704756A254A158A076E718
:105C700054A252A159A072E752A250A15AA06EE7B5
:105C800000B59FB00B4602465AA101A815F080F955
:105C900041F28833002249A101A8FFF760FF1FB03D
:105CA00000BD00B59FB00B46024657A101A815F0F4
:105CB0006FF941F28833002240A101A8FFF74FFF9E
:105CC000EDE72DE9F041CEB0642135A815F060FC78
:105CD0000024534D13AE281906EB840190F86A0096
:105CE0000A22FFF7A3FD641CE4B2042CF3D30024C2
:105CF0000FAF281907EB840190F86E000A22FFF716
:105D000095FD641CE4B2042CF3D300240DF12C089F
:105D1000281908EB840190F872000A22FFF786FD2B
:105D2000641CE4B2042CF3D312A811A9CDE9081025
:105D300010AACDE906720EA80DA9CDE9041016A887
:105D400015A90CAACDE90010CDE90282331D13AAD2
:105D500034A135A815F01CF935AA3DA117A815F0F6
:105D600017F94FF47A63002214A117A8FFF7F7FE82
:105D70004EB015E700B59FB00B460092024639A120
:105D800001A815F005F94FF47A7300220BA101A8C0
:105D9000FFF7E5FE83E700B585B000286ED001224D
:105DA0006DE06BE000100140004C0040000C014031
:105DB0000412002025730D0A000000004F4B000064
:105DC000415400006E6F206368616E6765000000DB
:105DD00041542B43574D4F44453D310041542B43D3
:105DE000574D4F44453D320041542B43574D4F448E
:105DF000453D330041542B43574A41503D222573C2
:105E0000222C22257322000041542B43574A415033
:105E10005F4445463D222573222C22257322000033
:105E2000C82200202225732E25732E25732E25735C
:105E3000222C2225732E25732E25732E2573222CBA
:105E40002225732E25732E25732E25732200000024
:105E500041542B4349505354415F4445463D2573BB
:105E60000000000041542B43575341503D222573FD
:105E7000222C222573222C312C2564000022FDA126
:105E8000684615F085F84FF4FA730022AFF2D4019A
:105E90006846FFF764FE05B000BDF0B5B9B0044632
:105EA0000F4615461E46642120A815F071FB14B15B
:105EB000012C0FD107E03B46F2A2F3A120A80095E8
:105EC00015F066F806E03B46F3A2EFA120A8009586
:105ED00015F05EF8052E06D220AB3246EFA102A8DF
:105EE00015F056F804E020AAF1A102A815F050F828
:105EF0004FF47A63F2A2AFF23C1102A8FFF72FFE33
:105F000039B0F0BD2DE9F041BAB08046409F0E4651
:105F100015461C46642121A815F03AFBCDE9006521
:105F20004346DDA2EAA121A8029415F031F8052F1D
:105F300006D221AB3A46D9A103A815F029F804E00E
:105F400021AADBA103A815F023F84FF47A63DCA2A1
:105F5000AFF2981103A8FFF702FE3AB020E610B5A1
:105F60009EB04FF4FA7400280ED00B460122DDA13A
:105F7000684615F00DF823460022AFF2C0116846BE
:105F8000FFF7EDFD1EB010BD0B460022D5A16846FF
:105F900014F0FEFF23460022AFF2E0116846FFF73F
:105FA000DEFDEFE710B54FF4FA730022AFF2F41103
:105FB000D1A0FFF7D4FDD8B1D3A1D64815F016FA79
:105FC00008B1022010BDD4A1D24815F00FFA08B1D3
:105FD000032010BDD3A1CF4815F008FA08B1042062
:105FE00010BDD3A1CB4815F001FA08B1052010BDB2
:105FF000062010BD10B500244FF4FA730022AFF252
:106000004421BDA0FFF7ABFD00282DD0CBA1C14896
:1060100015F0ECF900B10124CCA1BE4815F0E6F969
:1060200010B144F0020401E024F00204CBA1B9480D
:1060300015F0DCF910B144F0040401E024F004048C
:10604000CAA1B44815F0D2F910B144F0080401E037
:1060500024F00804C9A1AF4815F0C8F910B144F004
:10606000100401E024F01004204610BD2DE9FC418D
:1060700006464FF4FA730022AFF2C021C3A0FFF727
:106080006EFD00250024C5A1A24815F0AFF918B196
:106090000B3000226F4602E00020BDE8FC81815CED
:1060A0003A2907D0052D01D3222926D0012C0ED95B
:1060B0000020F2E7022C06D19DF801109DF8003077
:1060C00001EB031171556D1CEDB2002411E0A1F13B
:1060D0003003092B04D82146641CE4B27B5408E049
:1060E000A1F16103052B04D857392346641CE4B29F
:1060F000F954521CD2B2282AD1D3022C06D19DF8D1
:1061000001009DF8001000EB011070550120C4E75C
:1061100010B592B041790279C3788478CDE9022133
:10612000CDE9004343780278A0A105A814F030FF20
:106130004FF47A730022AFF27C3105A8FFF70FFD10
:1061400012B010BDF8B54FF4FA730022AFF29431DB
:10615000A0A0FFF704FD0024A2A16E4815F046F9A7
:10616000A34D10B10C3000210AE0A2A1694815F03E
:106170003DF908B10220F8BD642028720020F8BD66
:10618000425C222A03D03F2C04D90020F8BD0844E9
:10619000401C08E023462B44641CE4B29A72491C5C
:1061A000C9B23C29ECD310B11530002101E0002028
:1061B000F8BD425C2C2A0ED0491CC9B20529F8D37F
:1061C000002100226C46835CABB12D2B06D0022946
:1061D00006D90020F8BD0844401CF1E7002106E084
:1061E000303B092B03D80E46491CC9B2A355521C9B
:1061F000D2B2052AE7D3012904D0022906D0032907
:106200000ED01BE09DF80000287217E09DF80000FA
:106210009DF8011000EB800001EB400028720DE0BA
:106220009DF80010642041439DF8010000EB8000C0
:1062300001EB40009DF80210084428720120F8BDCF
:106240002DE9FE4380460E4617464FF4FA794B4639
:106250000022AFF2984169A0FFF781FC00250024DD
:1062600069A12C4815F0C2F810B1C21D00200EE142
:10627000CEE0000041542B4349504D55583D256414
:106280000000000054435000222573222C22257365
:10629000222C2573000000005544500041542B432C
:1062A000495053544152543D25642C25730000003D
:1062B00041542B43495053544152543D25730000DF
:1062C000414C5245415920434F4E4E4543540000E6
:1062D000222573222C222573222C25642C25642C44
:1062E0002564000041542B434950534552564552B2
:1062F0003D25642C2573000041542B4349505354D1
:1063000041545553000000005354415455533A3200
:106310000D0A0000041200205354415455533A33DF
:106320000D0A00005354415455533A340D0A0000ED
:106330005354415455533A350D0A00002B434950EC
:106340005354415455533A302C0000002B434950CC
:106350005354415455533A312C0000002B434950BB
:106360005354415455533A322C0000002B434950AA
:106370005354415455533A332C0000002B43495099
:106380005354415455533A342C00000041542B438C
:1063900049505354414D41433F0000002B43495065
:1063A0005354414D41433A220000000041542B43D5
:1063B00049505354414D41435F4445463D22257861
:1063C0003A25783A25783A25783A25783A25782278
:1063D0000000000041542B43574A41505F4355523F
:1063E0003F0000002B43574A41505F4355523A004B
:1063F000C8220020627573790000000041542B43CD
:10640000494653520000000053544149502C220089
:106410000020BDE8FE83115C2E2907D0032D01D397
:10642000222936D0032C28D90020F2E7012C04D0F1
:10643000022C06D0032C0ED01BE09DF808107155DD
:1064400017E09DF808109DF8093001EB810103EB7E
:10645000410171550DE09DF8083064214B439DF8D2
:10646000091001EB810103EB41019DF80A30194449
:1064700071556D1CEDB2002407E0303923460DF153
:10648000080C641CE4B20CF80310401CC0B2B84203
:10649000C1D3012C04D0022C06D0032C0ED01BE05B
:1064A0009DF80800705517E09DF808009DF8091048
:1064B00000EB800001EB400070550DE09DF80810E6
:1064C000642041439DF8090000EB800001EB40008F
:1064D0009DF80A10084470554B460022AFF2247113
:1064E000AFF25810FFF73BFB00250024AFF2541128
:1064F000FE4814F07BFF20B100F10B0300206E4634
:106500002EE0002085E7195C3A2907D0052D01D33C
:10651000222927D0022C0FD900207AE7022C07D19C
:106520009DF801109DF8002001EB021108F80510FC
:106530006D1CEDB2002411E0A1F13002092A04D84B
:106540002146641CE4B2725408E0A1F16102052AFC
:1065500004D857392246641CE4B2B154401CC0B27E
:10656000B842D0D3022C07D19DF801009DF800104D
:1065700000EB011008F80500FFF7E4FD012048E7F3
:1065800010B54FF4FA7423460022AFF2D071D8A0B0
:10659000FFF7E5FA40B12346D9A2AFF2E071BDE8BA
:1065A0001040D8A0FFF7DBBA002010BD10B54FF4A3
:1065B0007A7003F061F9D6A1D648FFF765F9BDE816
:1065C00010404FF4FA7003F057B970B51446ADF5AA
:1065D000167D0E461A46002540F226218C4203D92C
:1065E00000200DF5167D70BD38B13246AFF2343162
:1065F000C848FFF749F9012520E0052A05D22346BE
:10660000C5A1684614F0C4FC04E02246C7A1684650
:1066100014F0BEFC684614F0FBFE81B211B1B1F576
:10662000077F01D90020DCE7684601F0A9FC0220C1
:1066300003F022F9A1B2304601F0A2FC2846D0E7CF
:1066400000B59FB0642106A814F0A2FF06AABBA162
:1066500001A814F09DFC4FF47A630022AFF6A40168
:1066600001A8FFF77CFA1FB000BD2DE9F047814675
:106670000027DFF87882B8F800046FF30E00A8F85E
:10668000000498F8010420F0800088F8010440F22A
:106690000241404614F05AFF00240026AC4D32E07F
:1066A000022003F0E9F82978182904D0192909D023
:1066B00016290ED025E0FFF704FB10B3FFF7D7F93A
:1066C0002E701EE0FFF7BCFFD8B1FFF7D0F92E7097
:1066D00017E04FF4FA730022AFF620119DA0FFF7E8
:1066E0003EFA00B12E7040219D4814F02FFF9C48C7
:1066F0002021403014F02AFF9A49012048710BF004
:1067000039F9F8F798FE98F80104000604D42046F9
:10671000641CA4B26428C3D3B8F80004C0F30E000C
:1067200008F80060B9F1000F01D0704F05E08EA1AC
:106730006E4814F05BFE00B16C4F3846BDE8F08740
:1067400070B5027A2C2A01D0002070BD827A3A2AD4
:1067500010D1437A303B092B0CD89BB2002205E0C4
:106760008418E47A01F8014B521C92B29A42F7D392
:10677000184670BDC37A6FF02F053A2B03D0047B07
:106780003A2C1AD03EE0437A303B092B3AD8302AD3
:1067900038D3392A36D803EB830305EB43031A4475
:1067A00093B2002205E08418247B01F8014B521CAF
:1067B00092B29A42F7D3184670BD447A303C092C05
:1067C00020D8302A1ED3392A1CD8302B1AD3392B83
:1067D00018D804EBC406303A06EB041402EB82022C
:1067E00003EB840305EB42021A4493B2002205E056
:1067F0008418647B01F8014B521C92B29A42F7D381
:10680000184670BD002070BD10B50446432158489D
:1068100014F09CFE564914B1012C03D004E065200D
:10682000088001E0672008801D20488051480278D8
:106830008A804278CA8082780A81C2784A813E2260
:106840008A818379CB81464A603214780C825478ED
:106850004C8294788C82D478CC8232F8684C0C8349
:1068600089244C83007A888343480068C0F3072456
:1068700044EA00244C8481F82430030C1B0243EAD0
:106880001060A1F83900002081F83B0032F8662C36
:106890008A8781F83E0081F83F000A2281F8402073
:1068A00081F8410081F8420034490120087010BD90
:1068B0000B0A0370417000218170C170110A0171CF
:1068C000427170472DE9FF4707464FF47A73002263
:1068D000AFF618312AA0FFF742F900250024A046A0
:1068E0008DF80E808DF80D8052E00000041200201B
:1068F00041542B4349504D4F44453D310000000069
:106900003E00000041542B43495053454E44000083
:106910002B2B2B00004C004041542B434950534536
:106920004E443D25642C25640D0A000041542B4340
:10693000495053454E443D25640D0A0041542B43B4
:1069400057444843505F4445463D312C31000000D8
:106950008503002041542B524553544F52450000AB
:10696000D2220020380400202B49504400000000AF
:10697000061600204D80002018000020E8020020AC
:1069800041542B4349505354415F4355523F0000FB
:106990008DF80C80DCA1DE4814F028FD20B1431DE9
:1069A000002002AA03AE02E0002004B0C6E6195C93
:1069B0002E2907D0032D01D3222934D0022C28D927
:1069C0000020F2E7012C04D0022C06D0032C0ED0BC
:1069D0001BE09DF80C10515517E09DF80C109DF828
:1069E0000D4001EB810104EB410151550DE09DF893
:1069F0000C4064214C439DF80D1001EB810104EB28
:106A000041019DF80E40214451556D1CEDB200240A
:106A100005E03039A446641CE4B206F80C10401CB2
:106A2000C0B22828C3D3012C04D0022C06D0032CDA
:106A30000ED01BE09DF80C00505517E09DF80C009F
:106A40009DF80D1000EB800001EB400050550DE06B
:106A50009DF80C10642041439DF80D0000EB800070
:106A600001EB40009DF80E1008445055DFF8A49249
:106A7000E7B19DF8080099F86A10884211D19DF895
:106A8000090099F86B1088420BD19DF80A0099F81B
:106A90006C10884205D19DF80B0099F86D10884262
:106AA00007D00298C9F86A0002207EE70298C9F868
:106AB0006A00002500248DF80E808DF80D808DF879
:106AC0000C8095A1924814F091FC20B100F10A03CA
:106AD000002001AA01E0002067E7195C2E2907D0F9
:106AE000032D01D3222934D0022C28D900205CE7C1
:106AF000012C04D0022C06D0032C0ED01BE09DF8F4
:106B00000C10515517E09DF80C109DF80D4001EB4D
:106B1000810104EB410151550DE09DF80C406421C9
:106B20004C439DF80D1001EB810104EB41019DF8F0
:106B30000E40214451556D1CEDB2002405E0303962
:106B4000A446641CE4B206F80C10401CC0B228280D
:106B5000C3D3012C04D0022C06D0032C0ED01BE092
:106B60009DF80C00505517E09DF80C009DF80D1095
:106B700000EB800001EB400050550DE09DF80C103B
:106B8000642041439DF80D0000EB800001EB4000C4
:106B90009DF80E1008445055E7B19DF8040099F88F
:106BA0007210884211D19DF8050099F8731088423F
:106BB0000BD19DF8060099F87410884205D19DF814
:106BC000070099F87510884207D00198C9F872003B
:106BD0000220EAE60198C9F87200002500248DF829
:106BE0000E808DF80D808DF80C804EA1484814F071
:106BF000FDFB20B100F10A0300206A4601E00020FD
:106C0000D3E6195C2E2907D0032D01D3222934D0D5
:106C1000022C28D90020C8E6012C04D0022C06D072
:106C2000032C0ED01BE09DF80C10515517E09DF879
:106C30000C109DF80D4001EB810104EB4101515511
:106C40000DE09DF80C4064214C439DF80D1001EBC4
:106C5000810104EB41019DF80E40214451556D1C0A
:106C6000EDB2002405E03039A446641CE4B206F815
:106C70000C10401CC0B22828C3D3012C04D0022C15
:106C800006D0032C0ED01BE09DF80C00505517E0E9
:106C90009DF80C009DF80D1000EB800001EB40000A
:106CA00050550DE09DF80C10642041439DF80D00F7
:106CB00000EB800001EB40009DF80E100844505599
:106CC000E7B19DF8000099F86E10884211D19DF847
:106CD000010099F86F1088420BD19DF8020099F8D5
:106CE0007010884205D19DF8030099F87110884210
:106CF00007D00098C9F86E00022056E60098C9F83F
:106D00006E00012051E600003A69703A220000004E
:106D100004120020C82200203A6761746577617907
:106D20003A2200003A6E65746D61736B3A2200007E
:106D300010B5FAF702F9FAF7B3F840B210BDFAF756
:106D40001DB92DE9F04104460E461746FAF77BF8C7
:106D50006006000EFFF7ECFF0546280001D0BDE8F5
:106D6000F081002409E0305DFFF7E2FF054615B130
:106D7000FAF77FF803E0641CA4B2BC42F3D3FAF73D
:106D800078F82846EBE72DE9F04104460D46164613
:106D9000FAF759F8012000EB4400C0B2FFF7C8FF32
:106DA00004461CB1FAF765F82046D8E70024771EA0
:106DB00009E0BC4201DA012000E00020FFF7BFFF3C
:106DC0002855641CA4B2B442F3D3FAF752F8002059
:106DD000C5E710B5814C07E000F0BDFB08B100200D
:106DE00010BD0A2000F0BCFB641EF5D1601E10BD72
:106DF00070B5064607244FF0FF3500F097FB26FAE2
:106E000004F0C00702D000F064FB01E000F074FB66
:106E1000052000F0A5FB00F04FFB052000F0A0FBD3
:106E2000FFF7D7FF08B1284670BD641E64B2002C7E
:106E3000E3DA00F07BFB00F04CFB052000F090FB58
:106E400000F03AFB052000F08BFBFFF7C2FF08B112
:106E5000284670BD00F065FB08B1012400E0002465
:106E600000F064FB204670BD70B50646002500F0BA
:106E700030FB0724052000F073FB00F01DFBFFF73B
:106E8000A8FF08B1FF2070BD00F04BFB08B1012145
:106E900000E00021A1402943CDB200F047FB641E71
:106EA00064B2002CE6DA16B100F026FB01E000F037
:106EB00010FB052000F054FB00F0FEFA052000F066
:106EC0004FFBFFF786FF08B1FF2070BD00F02EFBDF
:106ED00000F0FFFA284670BD10B500F0EDFAFFF79C
:106EE00078FF10B14FF0FF3010BD00F005FB05201A
:106EF00000F036FB00F01AFB052000F031FB00200B
:106F000010BD10B500F0F8FA052000F029FB00F0E4
:106F1000D3FA052000F024FB00F0DBFABDE81040B6
:106F2000052000F01DBB2DE9F04104460E46174632
:106F3000FFF7D2FF002806D16006000EFFF758FFCA
:106F40000546280000D00AE7002409E0305DFFF77D
:106F50004FFF054615B1FFF7D4FF03E0641CA4B250
:106F6000BC42F3D3FFF7CDFF2846F8E62DE9F04108
:106F700004460D461646FFF7AFFF00280AD1012050
:106F800000EB4400C0B2FFF733FF04461CB1FFF72B
:106F9000B8FF2046E3E60024771E09E0BC4201DA90
:106FA000012000E00020FFF75FFF2855641CA4B219
:106FB000B442F3D3FFF7A5FF0020D0E610B500F0F0
:106FC00095FA00F079FABDE8104000F082BA10B5E9
:106FD00000F072FABDE8104000F07BBAF049020000
:106FE0002DE9F04106463489600013F06FFF074633
:106FF0000021DFF8588406E008EB4100008C27F8F8
:107000001100491C09B2A142F6DB3089401E04B2CE
:10701000002515E030897168001B401E51F82010D2
:1070200037F81400096821B1884708EB4501088446
:1070300002E008EB45010884641E24B26D1C2DB2E9
:10704000002CE7DA3846BDE8F04113F06EBF70B5AA
:107050000546FE4C4FF0FF362078012801D030461F
:1070600070BDFA492A892031582000F00CFB08B184
:10707000304670BD2846FFF7B3FF0020207070BD7A
:1070800070B5044625686D1D6189582000F013FB1A
:1070900000280CD1284600F063FA208930B1EB4972
:1070A000012008702046BDE87040D0E7002070BD88
:1070B00030B5044600200021E44A9269938807E035
:1070C000106850F82100057BA54203D0491CC9B2C5
:1070D0008B42F5D88B4200D1002030BD10B5FFF7B0
:1070E000E7FF10B1BDE81040CAE74FF0FF3010BD18
:1070F0002DE9F0470188DFF85483A8F81010D44830
:10710000C8F818000022DFF84C932AE0D9F80000F4
:1071100050F82240002001F4704501F0E00601F033
:107120001F07B4F80CC018E0A36833F8103003F45C
:10713000704AAA450FD15FEAC15A0CD403F0E00AA5
:10714000B24508D103F01F03BB4204D8C8F8184069
:107150000020BDE8F087401C00B28445E4DC521CEE
:1071600012B2B9F804009042D0DC4FF0FF30F0E7E3
:107170001CB50446002020800120009001ABB64AD7
:1071800042F23201582000F0B1FA002807D1BDF8D0
:1071900004002080B0F5544F02D04FF0FF301CBDEA
:1071A00000201CBD10B50120FFF782FF50B14189BE
:1071B000582000F080FA002803D1A449012008706B
:1071C000002010BD4FF0FF3010BD70B504460D46D5
:1071D0000120FFF76DFF50B1FFF739FF002805D1FF
:1071E0009A48018C2180408C2880002070BD4FF08F
:1071F000FF3070BD70B504460D460120FFF76EFFED
:10720000002805D19148028C2280408C28800020E3
:1072100070BDC7E708B56946FFF7D7FF08BD08B5D9
:107220006946FFF7E7FF08BDBCE708B501466846B9
:10723000FFF7CBFF08BD08B501466846FFF7DAFF48
:1072400008BD70B504460D4684480078FFF746FF38
:10725000002805D17D48028C2280408C28800020A7
:1072600070BD10B57D480078FFF722FF50B141890D
:10727000582000F020FA002803D17449012008703A
:10728000002010BD4FF0FF3010BD70B504460D4614
:1072900072480078FFF70CFF50B1FFF7D8FE0028C6
:1072A00005D16A48018C2180408C2880002070BD67
:1072B0004FF0FF3070BD10B504460220FFF70EFFFF
:1072C000002807D16148418C008C41EA00402060D1
:1072D00008B1002010BD4FF0FF3010BD38B5010CD3
:1072E000ADF80010ADF802004FF0FF3400280AD0CE
:1072F0000320FFF7DDFE40B1418902236A46582092
:1073000000F0E6F938BD204638BD204638BD10B53E
:1073100004461620FFF7E2FE002803D14B48008CFC
:107320002080002010BD31B54FF0FF34BDF80000C3
:1073300000280BD04A480078FFF7BAFE40B14189D7
:1073400001236A46582000F0C3F938BD204638BDF5
:10735000204638BDF8B50646344600253B486F1E2A
:10736000007CC0F34210012801D03846F8BD3D48EA
:107370000078FFF79DFE20B1B6F57A3F03D9384675
:10738000F8BD3846F8BD38490022A4FB013605FB9C
:10739000016104FB02110A0242EA13610091418972
:1073A00001236A46582000F093F9F8BD2F48006881
:1073B000704758207047254A137C0380108A000BC1
:1073C0000870002070472149CA68896806C00020FB
:1073D0007047002082E6F8B51C4C20340021216063
:1073E00061601A4E00203070FFF7E8FD0320009026
:1073F00023464FF4FA7243F28261582000F076F986
:10740000002857D125460323002108E035F8112034
:10741000100240EA122025F81100491C89B2994255
:10742000F4D32088C0F3072141EA002220792168A3
:10743000030443EA1140C0F3072180B241EA00206F
:10744000616862F31F40C1F3072211E0A816002013
:1074500054590308F85B0308605B0300655903088F
:10746000645903086659030800894100E0020020BE
:107470000B0C42EA01221B0243EA116162F31F4135
:10748000090C41EA0041000CC6E9021001200090FD
:1074900023464FF47A7242F22F01582000F026F969
:1074A000002807D12046FFF723FE002802D1BDE8BF
:1074B000F8408EE7F8BD000008B54FF48060ADF8E5
:1074C000000004208DF8030069462648F1F7A5FC6A
:1074D00008BD08B54FF40060ADF8000004208DF839
:1074E000030069461F48F1F798FC08BD10B5FFF787
:1074F000F0FFBDE81040DFE738B54FF40064ADF8A9
:10750000004010208DF8030003208DF80200154D77
:1075100069462846F1F781FC21462846F1F7EEFC42
:1075200038BD4FF400610F48F1F7D2BC38B54FF4C5
:107530008064ADF8004010208DF8030003208DF822
:107540000200084D69462846F1F767FC21462846A7
:10755000F1F7D4FC38BD4FF480610248F1F7B8BCB4
:1075600002F06AB9000C01404178007841EA00203D
:107570007047C178027841EA02614278807812044B
:1075800042EA002008437047F3E770B50546FF2044
:107590000023312410E0EA5C50400822060603D59F
:1075A00084EA4000C0B201E04006000E521ED2B292
:1075B000002AF3D15B1C9BB28B42ECD370BD10B59B
:1075C0001446FFF7E2FFA04202D04FF0FF3010BD9B
:1075D000002010BD08B50620009001226946002059
:1075E000FFF7A1FC08BD2DE9F04105461746984676
:1075F000080A287002206970002415E037F814107A
:107600000A0A411C89B22A5417F814004A1C96B27F
:107610006854A819801E0221FFF7B7FF0146701CAD
:1076200080B2A955641CE4B24445E7D3BDE8F081BB
:107630002DE9F04391B00F4602EB42011FFA81F8A9
:1076400001AE42463146FFF791FC002818D10024D4
:10765000002512E03019814682780221FFF7AFFF42
:1076600000280DD1315D681C80B2795599F8012050
:10767000411C8DB23A54E41CA4B24445EAD3002024
:1076800011B0BDE8F08370B50C4615462A46214678
:10769000FFF7CEFF00280DD109E004EB4003597835
:1076A0001A7841EA022124F81010401CC0B2A84206
:1076B000F3D3002070BD38B5044600231A4668464F
:1076C000FFF791FF022269462046FFF72CFC38BDE8
:1076D00010B588B00446DBB26846FFF784FF024667
:1076E00069462046FFF71FFC08B010BDF8B50646F6
:1076F000069F14461D4600231A466846FFF773FF8F
:10770000022269463046FFF70EFC002808D114B16A
:107710002046FFF725FF3A4629463046FFF7B3FFDC
:10772000F8BD08B5009313460022FFF7DFFF08BD40
:1077300070B50024FD4D4FF4FA76FEF733FCA871C6
:10774000401E032808D3304602F096F8F7F773FE80
:10775000641CE4B20A2CF0D3A879032807D133467D
:10776000BDE870400022F2A1F2A0FEF7F8B970BDAA
:1077700070B500244FF47A7504E0F7F75CFE6420DE
:1077800002F07AF82B460022E9A1EEA0FEF7E7F915
:10779000002804D12046641CE4B21428EDD370BD47
:1077A00010B5002404E0F7F746FE642002F064F808
:1077B00064230022DEA1E6A0FEF7D1F9002804D15F
:1077C0002046641CE4B21428EDD310BD10B500248B
:1077D00004E0F7F730FE642002F04EF86423002244
:1077E000D3A1DFA0FEF7BBF9002804D12046641C1A
:1077F000E4B21428EDD310BD2DE9F047DC4E00258E
:107800007571DFF8289399F80600012874D099F86B
:10781000000050B135704FF4FA730022C4A1D0A01B
:10782000FEF79DF9C82002F027F899F801004FF4FF
:107830007A7701280ED1FEF744FA384602F01CF898
:107840003B46CCA2BAA1CDA0FEF789F9C82002F030
:1078500013F8757199F800004FF48068012824D15D
:107860000020FEF7F7F9C82002F006F8AF494A31C8
:10787000A1F14000FEF704FA002411E00020FEF719
:10788000F4FE01464246BF4813F0E1FDA8A1BE4800
:1078900013F0ACFD48B9F7F7CEFD384601F0ECFF28
:1078A0002046641CE4B20A28E8D399F801000128B4
:1078B0001ED10024FEF705FA384601F0DDFF11E085
:1078C0000020FEF7D2FE01464246AE4813F0BFFD4F
:1078D00097A1AD4813F08AFD48B9F7F7ACFD3846DB
:1078E00001F0CAFF2046641CE4B20A28E8D375718F
:1078F000BDE8F0471CE7FFE7BDE8F08710B59C4CFA
:10790000A079012805D1FFF777FFF1F719FC0020D6
:10791000A07110BD10B5002404E0F7F78CFD6420C1
:1079200001F0AAFF6423002281A198A0FEF717F9B5
:10793000002804D12046641CE4B20228EDD310BD17
:107940008EB01420089000274FF0000A884D0026C2
:107950002E70DFF8D881042088F80700B8F80200FC
:107960004FF6FF74002801D0A04203D14FF4FB7002
:10797000A8F802006D4898F80A100A300D90FF2907
:1079800007D198F80B00FF2803D140210D9813F080
:10799000DDFD664898F84A104A300C90FF2907D15F
:1079A00098F84B00FF2803D120210C9813F0CEFD4E
:1079B000AE71B8F8040008B1A04203D14BF6C02064
:1079C000A8F80400B8F802000A2206A9FDF72EFF65
:1079D0004FF4FA64204601F04FFFFEF73AF8FEF745
:1079E00046F8204601F048FFFEF712F983464F485B
:1079F0004FF0010976300B90BBF1020F02D088F8EE
:107A0000069055E0644C207808B1FF280BD16078CF
:107A100008B1FF2807D1A07808B1FF2803D1E0788A
:107A200088B3FF283CD040F2C240F9F7AAFB8DF89A
:107A30001000442831D018208DF81100FE208DF858
:107A40001200E078102803D210308DF8130001E006
:107A50008DF81300A078102803D210308DF8140090
:107A600001E08DF814006078102803D210308DF8F2
:107A7000150001E08DF815002078102804D2103090
:107A80008DF8160002E00BE08DF816000DF11100E4
:107A9000FEF73EFB85F8019002E00B98FEF7E6FA50
:107AA000052088F806000020FEF7D4F8FFF7A4FEB2
:107AB000052001F0E1FEBBF1020F0BD1687801282F
:107AC00008D10B98FEF7D2FA6E70442140F2C24002
:107AD000F9F758FBF7F7AFFCBBF1020F03D0FEF745
:107AE00097F88346E4E7A878142802D9AE70FDF72A
:107AF000BEFF98F8060002286FD001286DD098F8D4
:107B0000010038B988F86A6088F86B6088F86C60A2
:107B100088F86D60287840B94FF4FA73002204A108
:107B20000BA0FEF71CF800B138E039E0C8220020B5
:107B30004F4B000041542B434950434C4F53453D5C
:107B40003500000041542B524553544F524500001C
:107B500041542B43575354415254534D41525400B6
:107B600041542B435753544F50534D4152540000EE
:107B7000E4020020726561647900000041542B52D8
:107B800053540000E01600200412002041542B43FF
:107B900057514150000000004D80002085F80090B2
:107BA0002878C0B30024FEF7FDF988F806006420A9
:107BB00001F062FEF7F73FFC98F80600032804D9AD
:107BC0002046641CA4B2C828EDD3C82C06D3FFF706
:107BD00013FEA878401CA8706AE720E088F80060CF
:107BE00040210D9813F0B2FC20210C9813F0AEFC4C
:107BF000E94880F8059009F0BDFE4FF4FA730022C1
:107C0000AFF2D401AFF2A800FDF7A9FF642001F0A4
:107C100033FEFFF7F1FDC82001F02EFE48E7AE70FD
:107C2000687920B34FF480642146DC4813F08EFC61
:107C30002146DB4813F08AFC0020FEF716FD0146C2
:107C40002246D74813F003FCD548C0793038C4B277
:107C5000D249D348FEF774FD024610006BD0A01E37
:107C600002287DD8CD490878EE2865D073E0282217
:107C7000CC490B98FEF7E4FA68B198F86A0040B96D
:107C800098F86B0028B998F86C0010B998F86D0056
:107C9000E0B185F805900020FEF714FE4FF4FA7469
:107CA00023460022AFF27811BFA0FDF758FF012054
:107CB000FEF771F8F7F7BFFB23460022AFF29011F1
:107CC000AFF29010FDF74BFF002403E06E71E2E786
:107CD000F7F7B1FB0096B8F8041002230A46B6A0E5
:107CE000FEF710F920B92046641CA4B20528EFD392
:107CF000002401E0F7F79FFB40F2D24102230A463D
:107D0000ADA0CDF80090FEF7FDF820B92046641C28
:107D1000A4B20528EED3002401E0F7F78CFB08AAF3
:107D200006A90120FEF71BF9002804D12046641C97
:107D3000A4B20528F1D3ACE0487810280BD188789C
:107D400048B9C87838B9087928B9487918B988790C
:107D500008B9C87948B19C4A88799279904200E084
:107D60001FE00CD0FF2807D093E07F210B20F9F70C
:107D700009FAF1F7E5F98CE0C879192810D087499C
:107D8000052008F05FFB6A8942B185488F49C079B8
:107D90003038C3B20020FEF718FC6E81FFF7AEFD4D
:107DA00077E014B1012C23D073E0894C207898BB84
:107DB00084F800900023794901A8CDF800900CF0D8
:107DC00002FB0246501EB0F5FF7F0FD80123734916
:107DD00001A80DF073FE2A8942B171487D49C0792E
:107DE0003038C3B20020FEF7F0FB2E81267050E041
:107DF0006A49087864284CD185F80490002098F8E6
:107E00006A300A9398F86B4098F86CE098F86D1017
:107E1000C2F3850C099114E03BE060490A9A01EB3A
:107E200080014B7893420AD18A78A24207D1CA785E
:107E3000724504D10A7909998A4200D12E71401CF9
:107E4000C0B26045E9D3287918B30020FEF7DCFC06
:107E500061498E77CE7781F8206081F8216000201B
:107E6000594B1A180C1892F84D2384F82520401C01
:107E7000C0B21428F5D311F83E0F40F0020008708C
:107E8000474843225449C0793038C3B20020FEF736
:107E90009CFB50466421B0FBF1F20AF1010A01FBA0
:107EA00012001FFA8AFA60B9FEF74CF9C8B1022035
:107EB00088F80600EE70E878032802D388F8069068
:107EC0006E7138467F1CBFB2B0F5967F7FF699ADD4
:107ED00000270120FEF7F6FC02287FF492AD6E71B8
:107EE000E6E5E878401CE870E5E710B58CB00121C4
:107EF0000220F7F7CDFB394C2046F0F731FE4FF466
:107F0000167004901020039000210B91254A123224
:107F10000292089180220692202009903048019018
:107F20000791059180140A9001A92046F0F78FFE71
:107F30000CB010BD70B50446294D01222D1F8021C3
:107F40002846F8F7A5FB2146244C2046F0F7C0FE52
:107F500001212046F0F7A5FE224E3046F0F7BDFE87
:107F60000028FAD03046F0F7C7FE00212046F0F78F
:107F700098FE2846BDE8704000228021F8F788BBB3
:107F800010B50C46014607482246123013F05FFA3E
:107F90002046FFF7CFFF10BD38040020C81E002088
:107FA000E01600203223002041542B4349504D4F0E
:107FB00044453D30000000003235352E3235352E37
:107FC0003235352E323535004D800020D41C00204E
:107FD0000D000020E01A0020061600205804024080
:107FE000044C00400000021030B5B0F5FA7F6CD2AE
:107FF000454B1B78012B06D0022B09D0434B33F89D
:108000001000088062E0424B33F8100008805DE009
:108010003D4DAD1C2B88834208D900EBC00303EB18
:1080200040100A23B0FBF3F008804FE06C888442D4
:108030000CD9E41AC01A04EB84044FF4FA736400F8
:10804000584390FBF4F0323008803FE0AB88834225
:108050000CD91B1B001B03EB83034FF4FA745B006A
:10806000604390FBF3F0643008802FE0EC8884429A
:108070000CD9E41AC01A04EB84044FF4FA736400B8
:10808000584390FBF4F0963008801FE02B89834220
:108090000CD91B1B001B03EB83034FF4FA745B002A
:1080A000604390FBF3F0C83008800FE0C41A4FF42F
:1080B000FA704443C3F5FA7000EB8000400094FB73
:1080C000F0F000F59670088000E0088008883228FB
:1080D00002D20020107030BD642802D2012010703E
:1080E00030BD962802D20220107030BDC82802D2BE
:1080F0000320107030BDB0F5967F02D204201070BE
:1081000030BD0520107030BDF0020020EA5F03088A
:10811000005C03085648018941814FF47A718182DD
:10812000704770B540F2BE40F9F72BF8504CE08034
:108130001E2801D90720E08040F2BB40F8F77CFF01
:10814000054640F2BC40F8F777FF45EA0020208161
:10815000B0F5FA7F02D94FF4C870208140F2BF40D9
:10816000F8F76AFF207140F2BD40F8F765FFA07094
:108170000A2801D90120A07040F2BA40F8F75CFF4C
:10818000E0700021012800D9E170E078012803D0D7
:108190006182BDE87040BDE74FF49860F8F74CFF8E
:1081A000054640F2C140F8F747FF45EA00206082EB
:1081B000EFE710B504462E484482E1B24FF49860D0
:1081C000F8F7E0FFC4F30721BDE8104040F2C140DA
:1081D000F8F7D8BF70B526498A89521C8A818A8AE5
:1081E000002482420AD90B785B1CDBB20B700A2B8D
:1081F00004D90C708B78D21A8A828C818A8A4FF4C7
:10820000616302F10A05A84209D8143DA84206DBC1
:10821000C889401C80B2C881984200D34A818889AD
:1082200098420BD34878401CC0B248708C810A8AAF
:10823000521C0A820A79904200D34C70C8880A8A7C
:1082400000EB4000B2EBC00F10D30C8208894A89C2
:1082500000F10A018A4202D814398A4206DA101A59
:1082600000B2FFF7A6FFBDE8704053E770BD000005
:108270000203002008B5002142F2B112684600F066
:1082800044FB024669466220FEF75BFD00B200280F
:1082900004D14FF47A70FFF763F9002008BDFEB5F2
:1082A00006460D46144600214EF60542684600F08B
:1082B0002CFB024669466220FEF743FD00B200280F
:1082C00015D106226946622000F0A7FB00B2002803
:1082D0000DD16846FFF748F930806E46B01CFFF7B5
:1082E00043F92880301DFFF73FF920800020FEBDB4
:1082F0007CB50C4615466A4601A9FFF7D0FF002859
:1083000010D1BDF8040045F27351FF4A484302EB17
:1083100050302060BDF8000043F2D4014843400BC8
:10832000286000207CBD08B5002143F686726846AF
:1083300000F0EBFA024669466220FEF702FD00B249
:10834000002803D1F148FFF70BF9002008BD38B52C
:108350000446002142F21832684600F0D6FA02467E
:1083600069466220FEF7EDFC00B2002810D14FF400
:108370007A70FFF7F5F802226946622000F04DFBA3
:1083800000B2002804D16846FFF7EEF820800020F4
:1083900038BD38B504466846FFF7D9FF002807D135
:1083A000BDF8000045F273514843400B20600020A7
:1083B00038BD1CB50446002142F21D42684600F05B
:1083C000A4FA01462246684600F0CDFA82B2694618
:1083D0006220FEF7B6FC00B2002804D14FF47A7098
:1083E000FFF7BEF800201CBD45F6DE714843000CC7
:1083F000DFE738B50446002142F22232684600F039
:1084000084FA024669466220FEF79BFC00B200280F
:1084100010D14FF47A70FFF7A3F802226946622068
:1084200000F0FBFA00B2002804D16846FFF79CF880
:108430002080002038BD1CB50446002142F22742AE
:10844000684600F062FA01462246684600F08BFA60
:1084500082B269466220FEF774FC00B2002804D1A3
:108460004FF47A70FFF77CF800201CBD1CB5044661
:1084700000214FF46042684600F047FA0146224668
:10848000684600F070FA82B269466220FEF759FC35
:1084900000B2002804D14FF47A70FFF761F8002091
:1084A0001CBD7CB505460C46002143F22F62684690
:1084B00000F02BFA01462A46684600F054FA82B2D0
:1084C00069466220FEF73DFC00B200280FD19048BB
:1084D000FFF746F802226946622000F09EFA00B2D9
:1084E000002804D16846FFF73FF8208000207CBDBB
:1084F00038B50446002142F21332684600F005FA0E
:10850000024669466220FEF71CFC00B2002810D12A
:108510004FF47A70FFF724F802226946622000F0D7
:108520007CFA00B2002804D16846FFF71DF82080CD
:10853000002038BD1CB50446002142F216426846B0
:1085400000F0E3F901462246684600F00CFA82B2D8
:1085500069466220FEF7F5FB00B2002804D14FF413
:108560007A70FEF7FDFF00201CBD08B5002142F225
:10857000AC12684600F0C9F9024669466220FEF76F
:10858000E0FB00B208BD38B5044600214EF2B84207
:10859000684600F0BAF9024669466220FEF7D1FB50
:1085A00000B2002810D14FF47A70FEF7D9FF0222F2
:1085B0006946622000F031FA00B2002804D1684612
:1085C000FEF7D2FF2080002038BD08B5002143F21D
:1085D0001562684600F099F9024669466220FEF786
:1085E000B0FB00B2002803D14A48FEF7B9FF0020D3
:1085F00008BDFEB506460D461446002143F28262D0
:10860000684600F082F9024669466220FEF799FB4F
:1086100000B2002819D14FF47A70FEF7A1FF0622AC
:108620006946622000F0F9F900B200280DD16846D1
:10863000FEF79AFF30806E46B01CFEF795FF28804B
:10864000301DFEF791FF20800020FEBD38B50446A6
:10865000002143F23962684600F057F90246694644
:108660006220FEF76EFB00B200280FD12A48FEF709
:1086700077FF02226946622000F0CFF900B200289D
:1086800004D16846FEF770FF2080002038BD08B591
:10869000002143F23262684600F037F9024669462B
:1086A0006220FEF74EFB00B2002803D11948FEF706
:1086B00057FF002008BD08B5002143F24662684616
:1086C00000F023F9024669466220FEF73AFB00B249
:1086D000002804D144F62060FEF742FF002008BDC8
:1086E00008B5002142F29D12684600F00EF90246DC
:1086F00069466220FEF725FB00B2002803D1074837
:10870000FEF72EFF002008BD3850FFFF20A1070014
:10871000801A060000350C0080969800404B4C00F3
:1087200008B5002142F29612684600F0EEF80246C3
:1087300069466220FEF705FB00B20028E3D14CF247
:108740005030FEF70DFF0020DDE708B5002143F2B1
:10875000E062684600F0D9F8024669466220FEF7FA
:10876000F0FA00B20028CED14FF47A70FEF7F8FE8E
:108770000020C8E708B5002143F2F662684600F021
:10878000C4F8024669466220FEF7DBFA44F6206030
:10879000FEF7E6FE0020B6E72DE9FE43FEF70EFCED
:1087A000FFF7E8FFFFF7BFFDFFF785FF2D4900202A
:1087B00008702D4C012525816A4601A902A8FFF702
:1087C00018FF0226DFF8A480072708B1268103E0FE
:1087D0000320208188F80070FFF74CFD10B1E58080
:1087E000BDE8FE83E68088F80070F9E73EB51E49D3
:1087F000C88A401CC8821D480078072819D1194C26
:108800002078012816D06A4601A902A8FFF770FD5A
:1088100000280ED1BDF8080000280AD0009A642173
:1088200092FBF1F2019B92B293FBF1F189B2F2F764
:108830008DFE3EBDFFF777FD4FF47A75284601F0B7
:108840001BF80C4A0A491088FFF72BFE284601F056
:1088500013F8FFF70FFD41F2883001F00DF800200A
:1088600020703EBD18030020A6860020590100207C
:10887000A0030020A203002070B50546FF200023BE
:10888000312410E0EA5C50400822060603D584EA51
:108890004000C0B201E04006000E521ED2B2002AD3
:1088A000F3D15B1C9BB28B42ECD370BD10B5144668
:1088B000FFF7E2FFA04201D0012010BD002010BD53
:1088C0002DE9F041054617469846080A287002200F
:1088D0006970002415E037F814100A0A411C89B2A7
:1088E0002A5417F814004A1C96B26854A819801E1E
:1088F0000221FFF7C1FF0146701C80B2A955641C1C
:10890000E4B24445E7D3BDE8F08110B5140A4B1C2E
:108910009BB24454591C89B2C254084610BD70B56C
:10892000044615462A0E481C80B262542A0C411C8B
:108930008EB22254A019801E0221FFF79DFFA05580
:10894000761CB1B22A0A481C80B26254411C8EB215
:108950002554A019801E0221FFF78EFFA055761C1A
:10896000B0B270BDDBE730B50446130A481C80B2D4
:108970006354411C8DB222546019801E0221FFF7FE
:108980007BFF60556D1CA8B230BD92B2EBE770B5AD
:10899000044615462A0E481C80B262542A0C411C1B
:1089A0008EB22254A019801E0221FFF765FFA05548
:1089B000761CB1B22A0A481C80B26254411C8EB2A5
:1089C0002554A019801E0221FFF756FFA055761CE2
:1089D000B0B270BD2DE9F0410546084617469846ED
:1089E0005FEAC87101D004208DE7002412E03A5DEF
:1089F000411C89B22A5438194278481C86B26A54FC
:108A0000A819801E0221FFF737FFA855761CB0B2C7
:108A1000A41CA4B24445EAD375E72DE9F0470D46FE
:108A2000510801EB41018FB2D10702D00420BDE80B
:108A3000F0873A462946FEF7A6F9DFF8508028B1BC
:108A4000B8F82C10491CA8F82C10F0E700240026D8
:108A500017E02819814682780221FFF727FF28B105
:108A6000B8F82E10491CA8F82E10E0E7295D701CFC
:108A700080B2A95599F80120411C8EB22A54E41CF9
:108A8000A4B2BC42E5D30020D1E70000A6860020B6
:108A900070B50024F64D04EB840005EB800000F077
:108AA0004FFC641C0A2CF6D3F148C83000F048FC97
:108AB000EF48DC3000F044FCED48F03000F040FCC2
:108AC000EC4800F03DFCEB48143000F039FCE9497B
:108AD000E9483C3941631431816370BD70B5044687
:108AE0001546102204F1340012F079FD002084F8BC
:108AF00043000A2D00D30925E5626564201D00F0BE
:108B00002AFC04F1180000F026FC2461C5F10A00DB
:108B1000A061646270BD70B506460D46482000F045
:108B2000A5FC044644B1B60045B12846206348B1CF
:108B3000A522314612F002FD204670BD304600F0FD
:108B400095FCF3E7204600F0E7FC0024F4E72DE96C
:108B5000FF4F81B08246DDE90E68109917469B46AB
:108B60003846FFF7D8FF0446C34DECB3216B781E9F
:108B700001EB800020F00709009732462046119B48
:108B80000299FFF7ABFF5A465146484600F01EFCDB
:108B90002060B8F1000F01D0C8F8004000F041FC9F
:108BA000A868401CA860286810B1A86938B10BE01B
:108BB0002C60A868012807D1FFF76AFF04E0286845
:108BC000C06AB04200D82C60E06A2969884200D9A6
:108BD0002861E96A491CE9626969884200D96861CB
:108BE00000EB8001A24800E008E000EB8100211DBD
:108BF00000F0B4FB012400F01CFC01E04FF0FF3456
:108C0000012C07D1A86928B12868C06AB04201D2F6
:108C100000F001FC05B02046BDE8F08F70B50546B8
:108C200000F0FFFB944E3068854200D10025F5B17D
:108C30002C46201D00F0B8FBA06A18B104F1180002
:108C400000F0B2FB211D8B4800F088FB7068401CCF
:108C50007060F06A401CF06200F0EBFBB069002825
:108C600007D0002D05D1BDE8704000F0D4BB3468BA
:108C7000DFE770BD70B5804DE869002803D0286A31
:108C8000401C286270BDE868401CE860E8684FF04E
:108C9000FF3670B9686BA96B6963A863A86A401C4A
:108CA000A862686B0068A0B1686BC068C068406863
:108CB0002863E868296B8842E4D3686B006850B188
:108CC000686BC068C4686068E968814205D228633F
:108CD00070BD2E63EDE72E6370BD201D00F064FBB8
:108CE000A06A18B104F1180000F05EFBE06A69693F
:108CF000884200D968615E4900EB800001EB80008A
:108D0000211D00F02BFBD8E72DE9F041002700F0F2
:108D100088FB594EF069401EF061F069E8BBB0680D
:108D2000D8B30025DFF84C81A8F114081CE0D8F86E
:108D30000C00C46804F1180000F036FB201D00F0A0
:108D400033FBE06A7169884200D97061484900EBE1
:108D5000800001EB8000211D00F000FBE06A31681B
:108D6000C96A884200D30125D8F800000028DED166
:108D7000306A28B908E0FFF77DFF306A401E306294
:108D8000306A0028F7D10125012D02D0706A012830
:108D900006D101270020706200E001E000F03BFBFB
:108DA00000F047FB3846BDE8F08170B50446324D0F
:108DB00028684460E868844206D22968A86B091DC7
:108DC000BDE8704000F0D8BA2968686B091D00F052
:108DD000D3FA286B844200D22C6370BD2648C16947
:108DE000491CC161704770B503460C460022FFF76D
:108DF000F5FF186804442049CD68A84206D9A0426E
:108E00000AD9C868844207D9012205E0A04202D8E5
:108E1000C868844200D901221C6032B10868001D74
:108E200000F0C2FA2046FFF7C0FFFFF76DFF0028F1
:108E300003D1BDE8704000F0EEBA70BD10B5024637
:108E40000020002A0DD0FFF7C9FF0B48C1688C181D
:108E50000068001D00F0A8FA2046FFF7A6FFFFF704
:108E600053FF002803D1BDE8104000F0D4BA10BD74
:108E70009C250020A02600201C03002010B50446DD
:108E800000F0CFFA0CB9F7480468E46A00F0D1FAB0
:108E9000204610BD2DE9F04106460D4600270A2D5B
:108EA00000D3092500F0BDFADFF8B883D8F8000038
:108EB000864200D1002646B13446606CA8422ED0CE
:108EC000854205D936B1012704E0D8F80040F4E71F
:108ED00006B90127E26A904200D1E5626564C5F1F6
:108EE0000A01A161E04D00EB8000616905EB8000A3
:108EF000814210D1201D00F057FAE06AD8F8141012
:108F0000884201D9C8F8140000EB800005EB80000E
:108F1000211D00F023FA012F01D100F07CFABDE8F9
:108F2000F04100F086BACF49C869002802D001207C
:108F300048627047CC4A02E04869401E486148696F
:108F400000EB800052F820000028F5D0486900EBC3
:108F5000800002EB800042685268426000F1080322
:108F60009A4201D1526842604068C0680860704708
:108F700070B5054600F055FABA4E3068854200D10A
:108F80000025BDB12C46201D00F00EFAA06A18B1D4
:108F900004F1180000F008FA211DB44800F0DEF9D1
:108FA00000F047FA002D0ED1B06928B1BDE870403D
:108FB00000F031BA3468E6E7AC480068B16888422E
:108FC00002D10020306070BDBDE87040ABE70021E9
:108FD000A64B42699A4206D1806AA3F128029042C8
:108FE00001D000B901210846704770B50446002C35
:108FF00025D09C4D2868844221D000F012FA2046EA
:10900000FFF7E5FF012816D1201D00F0CDF9E06A39
:109010006969884200D96861934900EB800001EBDF
:109020008000211D00F09AF9E06A2968C96A884227
:1090300001D300F0F0F9BDE8704000F0FAB970BD5E
:1090400070B5044600252046FFF7C1FF012808D16E
:10905000844EF06938B1854804F11801283800F0D1
:109060007DF9284670BDE06A3168C96A884201D33B
:10907000012500E00025201D00F096F9E06A7169E5
:10908000884200D97061784900EB800001EB8000D4
:10909000211D00F063F9E4E710B50446206B00F0F1
:1090A0003BFA2046BDE8104000F036BA70B56D4D71
:1090B000686800281FD0FFF791FE6C4E143E3068A0
:1090C000B8B10024FFF720FE002C14D100F0A9F95C
:1090D000F068C468201D00F067F9A868401EA86009
:1090E0006868401E686000F0A4F92046BDE8704042
:1090F000D2E70124E6E770BD5B4CFFF7D7FF20689D
:109100000128FAD900F087F9F7E71FB50024009489
:10911000019402942346642255A157480394FFF713
:1091200016FD012809D1EFF7D3F84E4801218161DE
:10913000C460BDE81F4000F05AB91FBD10B5EFF77D
:10914000C7F8484900208861BDE8104000F062B9C6
:1091500010B500F066F94348C46800F06AF920468B
:1091600010BD10B5EFF7B4F83E48C468EFF7B7F894
:10917000204610BD3B488068704770B50D46394C9D
:109180002168183100F0F8F82068001D00F00CF993
:10919000681C04D0E0682844BDE8704005E62168FA
:1091A000BDE87040091D314800F0D8B870B5C068FE
:1091B000C46804F11800064600F0F6F8294DEA6983
:1091C0005AB12A483146283800F0C8F8E06A2968C0
:1091D000C96A884212D3012070BD201D00F0E4F856
:1091E000E06A6969884200D968611F4900EB800024
:1091F00001EB8000211D00F0B1F8E7E7002070BD11
:1092000018498A6A0260C9684160704770B50446AF
:109210000D4600F006F92868411C0AD0114B216860
:109220009A6A914207D06168DA68914203D80124B2
:1092300010E000240EE06268D968891A814208D2E1
:10924000D968891A401A28602046FFF7D9FF002400
:1092500000E0012400F0EDF8204670BD0149012036
:10926000486270471C0300209C250020B426002083
:1092700049444C4500000000F99001082E48006860
:10928000EFE72D488169002903D0C06918B1022099
:10929000E7E70020E5E70120E3E770B50446264D47
:1092A000E06A2968C96A884223D22868C06AC0F186
:1092B0000A00A061E06A214E00EB8000616906EBC4
:1092C0008000814212D1201D00F06EF82868C06A2B
:1092D000E0626969884200D9686100EB800006EBB2
:1092E0008000211DBDE8704000F038B82868C06AD1
:1092F000E06270BD10B5044600281BD0616CE06AC6
:10930000884217D0201D00F04FF8606CE062C0F179
:109310000A00A0610849E06A4A69904200D94861A0
:10932000064900EB800001EB8000211DBDE81040E4
:1093300000F014B810BD00001C0300209C25002084
:1093400000F1080141604FF0FF328260C1600161AD
:109350000021016070470021016170474268536835
:109360004B6043688B60536899605160416008614D
:109370000168491C0160704710B50B685A1C02D087
:1093800000F1080202E0026904E0526854682468AF
:109390009C42FAD953684B6099608A6051600861B9
:1093A0000168491C016010BDD0E901219160D0E93C
:1093B0000112516001694A68824201D182684A60A3
:1093C000002202610868401E0860704720384FF094
:1093D0008073C36181610021416140F82029704799
:1093E0004FF0E0201E49416107210161704710B52F
:1093F0001C48016841F47F010160016841F07F4130
:109400000160FFF7EDFF184900200860EEF738FF14
:10941000002010BD704713494FF080501C39086080
:10942000704710B5EEF754FF0F480168491C016002
:1094300010BD0D490868401E0860002801D1EEF7F4
:109440004EBF704710B507494FF080501C39086077
:10945000EEF73EFFFFF70EFCBDE81040EEF73FBF12
:109460003F19010020ED00E0580300202DE9F041F4
:1094700004460025FFF7B2FC384E06F1080170687B
:1094800001F1080360B936480860002048604FF4D5
:10949000A0425A6018603248426003600120706048
:1094A0003CB11034600704D004F00700C0F108009C
:1094B0000444601E44F6FF72904228D2274A0832C4
:1094C000096801E00A4601464868A04202D20868DD
:1094D0000028F7D199421AD0156810350868106035
:1094E0004868001B20280ED90B1958604C605C6836
:1094F0001A48083000E0104602685768A742FAD3BD
:1095000002681A60036048683168081A3060FFF723
:10951000FBFB2846BDE8F08110B5002818D01038B4
:109520000446FFF75BFC60680C49083100E0114617
:109530000A6853688342FAD3086820600C600748C1
:109540006168026811440160BDE81040FFF7DCBBB0
:1095500010BD024800687047704700005C0300209F
:10956000C82600207047704770B504469F4D4021C3
:109570002846F7F734F90028F9D0A1B22846F7F7C2
:10958000C1F8204670BD2DE9F04186B006460121A4
:1095900044F20400F6F787F8944D2846F6F78EFF5C
:1095A0006815ADF8140003208DF8160018208DF80A
:1095B0001700DFF83C8205A94046EFF72EFC2F1577
:1095C000ADF8147004208DF8170005A94046EFF798
:1095D00024FCAC15ADF8144010208DF8170005A937
:1095E0004046EFF71AFC21464046EFF785FC252060
:1095F0008DF8000000248DF8014001208DF8020054
:109600008DF803006846EFF790F801967948AA14A0
:109610000178022925D0012928D0ADF80C40ADF8F9
:10962000084075480178012927D0022928D003294C
:109630002BD0ADF80A40ADF810400C20ADF80E006C
:1096400001A92846F6F782FF012240F2255128465B
:10965000F7F703F801212846F6F7F3FF06B0BDE857
:10966000F081ADF80C70ADF80820DAE74FF4C06077
:10967000ADF80C00ADF80820D3E7ADF80A20DAE722
:109680004FF40050ADF80A00D5E74FF44050ADF864
:109690000A00D0E7F0B587B0054601212020F6F793
:1096A00002F801218804F6F709F801215348EFF781
:1096B00045FC534F3846F6F701FFB815ADF81800D2
:1096C00003268DF81A6018208DF81B004D4C06A952
:1096D0002046EFF7A2FB6015ADF8180048208DF882
:1096E0001B0006A92046EFF798FB27208DF8040001
:1096F00000248DF805408DF8066001208DF80700E4
:1097000001A8EFF712F80295ADF80C407814ADF807
:109710000E00ADF81040ADF814400C20ADF812006A
:1097200002A93846F6F712FF012240F225513846C9
:10973000F6F793FF01213846F6F783FF07B0F0BD37
:1097400070B586B0054601211020F5F7ACFF012168
:109750002020F5F7A8FF01210805F5F7AFFF2A4EF5
:109760003046F6F7ABFEB014ADF8140003208DF8C8
:10977000160018208DF8170005A92448EFF74DFBB7
:109780000420ADF8140048208DF8170005A91D48E5
:10979000EFF743FB35208DF8000000248DF80140E1
:1097A00002208DF8020001208DF803006846EEF7D4
:1097B000BCFF0195ADF808407014ADF80A00ADF893
:1097C0000C40ADF810400C20ADF80E0001A9304659
:1097D000F6F7BCFE012240F225513046F6F73DFF78
:1097E00001213046F6F72DFF06B070BD003801406C
:1097F000000801400B0000200C0000203000140085
:10980000004800400014014000500040001001409A
:109810004FF0E0210A6922F004020A61224AC008DE
:1098200010704FF47A7358430123538048610869DC
:1098300040F00100086170472DE9F04100244FF02D
:10984000E0277E690546184800784543FFF7E9FDA3
:10985000BA69B9699142FCD003D2A2EB0100044479
:1098600003E0A6EB0100104404440A46AC42F0D3E6
:10987000BDE8F041FFF7DDBD70B50446FFF701FD1F
:1098800060B1094D6888844203D3B4FBF0F0FFF760
:10989000D5FA6888B4FBF0F100FB11444FF47A70FC
:1098A0006043BDE87040C7E778030020F749FF2018
:1098B0000870F74908707047F64900200860F649BB
:1098C00048734876704710B5F34C207C801EC1B2B7
:1098D000F24806F0CBFFF149227C237C0A4412F8BF
:1098E000012C194411F8021C02EB0121814201D123
:1098F000012010BD002010BD2DE9F05FDFF8A0832E
:1099000040F225514046F6F775FFDFF898A301278E
:109910000026DFF89493E04C012833D040F22775FD
:1099200029464046F6F766FF01285FD18AF807709E
:1099300099F82B10032901D0002957D10CF039F9DF
:10994000228D501C2085D948815C4046F6F7DAFE0E
:10995000218DE08B814249D340214046F6F73FFFFD
:109960000028F9D040214046F6F740FF0022294662
:109970004046F6F772FE2685FFF79EFFBDE8F05FD2
:109980000CF017B999F82B1003290CD000292DD110
:109990000CF00FF94046F6F7B9FEC1B2BDE8F05F32
:1099A000C3480CF03CB8607BBC4D502807D2404601
:1099B000F6F7ACFE617B4A1C6273685401E0FFF766
:1099C0007BFF607B01280DD0607B042810D0607B7A
:1099D00007281CD0607BDFF8DC824FF003090628E3
:1099E00040D042E050202074207EE075BDE8F09F1A
:1099F000E878A97800EB01200A28F7D168780628D2
:109A0000F4D10C202074207E0830E075EEE76878F1
:109A1000032815D0062813D010281CD029785529E2
:109A2000E4D1FF28E2D1A8780128DFD168790028A5
:109A3000DCD1A8790028D9D1A7700520E070D5E73E
:109A4000E878A97800EB01200A28CFD008202074FC
:109A5000207EE075CAE7A87900F109012174083079
:109A6000E075C3E76878192828D0607B217C88429C
:109A7000BCD16878032803D0062801D01028B5D1BE
:109A80002878DFF834B2FF2803D09BF8061088420C
:109A90003DD1FFF718FFB0B32079012824D08AF810
:109AA00008709BF8D80030B18449C0EB00108000EA
:109AB000088083480670E67500201DE0A08B002812
:109AC00094D1E07A002891D0607B2074E67584F808
:109AD0001990002004E0295C08F80010401CC0B276
:109AE000217C8842F7D381E7BDE8F05FE4E6295C9A
:109AF00008F80010401CC0B2217C8842F7D384F8DB
:109B00001990A77272E7FFE7BDE8F05FD4E6BDE801
:109B1000F05FD1E670B56B4D40F225512846F6F75F
:109B200069FE694CB8B12846F6F7F0FDC2B2B4F848
:109B3000000440F2FF31C0F30E0088420BD2B4F8AB
:109B40000004B4F80034C0F30E01481C60F30E03A7
:109B5000A4F80034625440F224412846F6F74AFE45
:109B600001280AD194F8010440F0800084F801042F
:109B70002846BDE87040F6F7C9BD70BD2DE9F0413B
:109B8000524E40F225513046F6F734FE0025424C45
:109B900001281DD040F2277739463046F6F72AFED5
:109BA000012813D1628D208C82426DD34021304632
:109BB000F6F715FE0028F9D040213046F6F716FEDC
:109BC000002239463046F6F748FD6585BDE8F0814C
:109BD0003046F6F79BFDC0B2A17B3B29F6D23C4E46
:109BE0003249012332784E39012A04D0032AEDD1BB
:109BF0007E2831D032E07E2801D1A27C1AB1A27C2D
